:020000040040BA
:10400000C04E0020B1C34000ADC3400079E1400084
:10401000ADC34000ADC34000ADC340000000000090
:1040200000000000000000000000000051C7400038
:10403000ADC3400000000000B1C7400015C84000FB
:10404000ADC34000ADC34000ADC34000ADC34000B0
:10405000ADC34000ADC34000ADC340000000000050
:10406000ADC3400039E1400000000000799F4000EE
:104070008D9F4000BDBB4000ADC34000ADC34000BC
:10408000ADC34000ADC34000CDBB4000D97F400070
:104090004DE14000ADC34000ADC34000214C4000A5
:1040A000ADC34000ADC34000ADC34000ADC3400050
:1040B000ADC34000A94A4000ADC34000000000006D
:1040C00000000000000000000000000000000000F0
:1040D00000000000000000000000000000000000E0
:1040E00000000000000000000000000000000000D0
:1040F000000000000000000000000000ADC3400010
:104100008DB04000ADC34000000000000000000082
:10411000000000000000000000000000000000009F
:10412000000000000000000000000000000000008F
:10413000000000000000000000000000000000007F
:10414000000000000000000000000000000000006F
:104400001CF3000010B5054C237833B9044B13B1ED
:104410000448AFF300800123237010BDE80B002097
:10442000000000002C2741000C4B43B10C480D4903
:1044300010B5AFF300800C48036823B910BD0A48DB
:10444000036833B97047094B002BF7D0BDE8104023
:104450001847064B002BF5D0184700BF000000009E
:104460002C274100EC0B00202C274100000000000D
:104470000120704770470120704700207047704747
:1044800001207047014B1878704700BF0C0C0020CA
:104490007047000058B908B5054B1B78012B00D0B8
:1044A00008BD044B1B68002BFAD09847F8E770470B
:1044B000100C0020040C002008B50C4B9847C37862
:1044C0000B4A1370012B0CD101220A4B1A700022E7
:1044D000094B1A80094B9847094B1B681BB1984739
:1044E00001E0084B9847012008BD00BFC19B400078
:1044F0000C0C0020100C00200E0C00201DE14000D0
:10450000040C002029E1400008B5054B1B78012B65
:1045100000D008BD0022034B1A70034B9847F8E700
:104520000C0C0020100C002029E1400010B582B0D6
:10453000074B00930B46024600218420054CA04700
:1045400018B9054A13680133136002B010BD00BFEB
:1045500095444000C5B74000080C0020014B18608E
:10456000704700BF040C00202DE9F0474FF40046CF
:10457000BF4B5E600B20BF4CA0470C20A047BE4B3A
:104580004FF0400CC3F810C0C3F8A0C0C3F834C04B
:104590004FF0807EC3F810E0C3F8A0E0C3F834E029
:1045A000B64A01271761C2F8A0705763022414614C
:1045B000C2F8A04054631C61C3F8A0405C631F664E
:1045C000C3F890705F655F62C3F88070196F3943FC
:1045D0001967596F21F0010159675F604FF480310D
:1045E0001966C3F8901059655962C3F88010186FA6
:1045F00008431867586F20F48030586759601C6171
:10460000C3F8A0405C6304205861C3F8A00058665A
:10461000C3F8900058655862C3F88000196F21F004
:1046200004011967596F21F00401596718211966AF
:10463000C3F8901059655962C3F880101D6F25F0BA
:1046400018051D675D6F25F018055D675960082521
:104650001D66C3F890505D655D62C3F88050196FA8
:1046600021F008011967596F21F0080159675D6051
:1046700010211966C3F8901059655962C3F880106B
:10468000D3F8708028F01008C3F87080D3F87480D5
:1046900028F01008C3F8748059604FF48028C3F8DC
:1046A0001480C3F8A0804FF02009C3F81490C3F819
:1046B000A090C3F810C0C3F8A0C0C3F834C0C3F8BA
:1046C00010E0C3F8A0E0C3F834E01761C2F8A070AE
:1046D00057631461C2F8A04054634FF4007CC3F8E0
:1046E00060C0C3F890C0C3F854C0C3F824C0C3F876
:1046F00080C01C6F44EA0C041C675C6F24F40074D7
:104700005C67C3F804C04FF480641C66C3F8904033
:104710005C655C62C3F880401F6F27431F675F6F53
:1047200027F480675F675C604FF4006EC3F810E0A9
:10473000C3F8A0E0C3F834E04FF400275F61C3F88A
:10474000A0701F66C3F890705F655F62C3F88070E9
:104750001F6F27F400271F675F6F27F400275F672D
:104760004FF480175F61C3F8A0701F66C3F89070A4
:104770005F655F62C3F880701F6F27F480171F6743
:104780005F6F27F480175F674FF480575F61C3F84E
:10479000A0705F66C3F890705F655F62C3F8807059
:1047A0001F6F27F480571F675F6F27F480575F677D
:1047B0004FF400575F61C3F8A0704FF480775761E2
:1047C000C2F8A0704FF48048C3F86080C3F89080AE
:1047D000C3F85080C3F82480C3F88080D3F870A059
:1047E0002AF4804AC3F870A0D3F874A02AF4804A4F
:1047F000C3F874A0C3F81080C3F8A080C3F8308059
:104800005E61C3F8A0604FF400365E61C3F8A0603B
:104810001066C2F8900050655062C2F88000166FB2
:1048200026F004061667566F26F004065667506099
:104830001566C2F8905055655562C2F88050106FE9
:1048400020F008001067506F20F008005067556096
:104850000B4DD5F8140140F03000C5F8140151613A
:10486000C2F8A0105166C2F890105165516209E07B
:1048700050140E40F5C04000000E0E4000100E40D7
:1048800000020E40C2F88010116F21F01001116774
:10489000516F21F010015167C2F81090C2F8A0903A
:1048A000C2F83490C2F810C0C2F8A0C0C2F830C03C
:1048B0004FF400015961C3F8A0105966C3F8901075
:1048C00059655962C3F88010196F21F40001196706
:1048D000596F21F400015967C2F860E0C2F890E016
:1048E000C2F854E0C2F824E0C2F880E0116F21F46D
:1048F00000611167516F21F400615167C2F804E053
:104900001466C2F8904054655462C2F88040116F3A
:1049100021F480611167516F21F480615167546007
:104920001F66C3F890701F655F62C3F880701A6FCE
:1049300022F480721A675A6F22F480725A671F61DC
:10494000C3F8A0701F63BDE8F08700BF08B5034B34
:1049500053F8203003B1984708BD00BF180F00205E
:1049600010B582B0036B0193002400E00134172CD2
:1049700009D8064B53F82420019B1A42F6D0204652
:10498000034B9847F2E702B010BD00BFAC1E4100D8
:104990004D49400000230360064A4260064A826097
:1049A0004FF48022C2600222027442748374C37482
:1049B000037570470000DC05808D5B00036C1943B4
:1049C0000164704710B58B7C23B34FF000434A68F5
:1049D0008C686400B2FBF4F2013A120292B2134303
:1049E0000A7C120602F0706213434A7C120702F03E
:1049F00040521343CA6813434360CB7C63B14FF00A
:104A000080730A7D52B90022134303640968054B81
:104A1000984710BD0023DAE70023F2E74FF4801235
:104A2000F2E700BFBD49400008B5036B13F0807F7B
:104A300001D0192008BD01230360064B98470023CD
:104A400004E00021044A42F823100133172BF8D95F
:104A5000002008BDC5494000180F0020B1F1FF3FFC
:104A600004D0044B53F82130436270474FF0FF33BA
:104A700043627047AC1E410010B5084C44F8212039
:104A8000074A4FF00054C2F880411B01DBB282F8A4
:104A90001D331460034B984710BD00BF180F002052
:104AA00000E100E05D4A400008B50248024B98472B
:104AB00008BD00BF008003406149400010B51720C9
:104AC000234CA0471820A047224B4FF480321A668F
:104AD000C3F890205A655A62C3F88020196F1143B9
:104AE0001967596F21F4803159675A6001225A665B
:104AF000C3F890205A655A62C3F88020196F114399
:104B00001967596F21F0010159675A60A3F52063B5
:104B100040F21262DA644FF400621A600E4B0F4AE0
:104B20005A6041225A62052119600D4A5A644FF4B5
:104B3000F572DA6500229A6519640A4B1A700A4BFD
:104B40004FF400021A60702283F8172310BD00BFD3
:104B5000F5C04000000E0E400000014004060900B0
:104B600001C4000A7C0F002000E100E010B54FF402
:104B70000002124BC3F88020BFF34F8FBFF36F8F3B
:104B80000F4B4FF480321A66C3F890205A655A6270
:104B9000C3F88020196F21F480311967596F21F40F
:104BA000803159671A601A61C3F8A0205A63172030
:104BB000044CA0471820A04710BD00BF00E100E052
:104BC000000E0E4049C14000642800D964200F4AFD
:104BD000D36D03FB00F30E49A1FB03135B0993653F
:104BE00048B10A4B5A6C22F040625A645A6C42F047
:104BF00080625A6470471346526C22F040625A64D5
:104C00005A6C42F000625A64704700BF00000140D5
:104C10001F85EB51014B1888704700BF800F0020A3
:104C20000F4B1B6A13F0010F06D000220D490A70CA
:104C30000D490A600D490A6013F0400F0ED00122A1
:104C4000084B1A70064B9A69094BB3FBF2F3064AFC
:104C50001360C3EB03139A00044B1A60704700BF44
:104C6000000001407C0F0020780F0020800F002002
:104C70001F1A0500014B1870704700BFBC000020D0
:104C8000064B1B7823B94FF40062054B1A6370473B
:104C90004FF40062024B5A63704700BFBC00002013
:104CA000000E0E40064B1B7823B94FF40062054BF3
:104CB0005A6370474FF40062024B1A63704700BF9B
:104CC000BC000020000E0E402DE9F04186B0884661
:104CD00016461F46D0B9244B984705460024049435
:104CE00098238DF8043001238DF8053002238DF8C8
:104CF000063003238DF8083005AB03938DF8078049
:104D00008DF815402846194B984705E0184B9847F1
:104D10000546E3E70134E4B2B4421ED28DF81440F4
:104D20003B5D8DF81630322201A92846114B984779
:104D3000AB79DBB2022BEDD028460F4B98473222DD
:104D400001A928460B4B9847AB79DBB2022BE1D087
:104D500028460A4B9847002003E02846074B98470F
:104D6000012006B0BDE8F0810DE14000396440004B
:104D700015E1400065644000156640004D64400048
:104D80002DE9F04186B00F4616469846B8B9344B27
:104D9000984704460025049598238DF80430012394
:104DA0008DF805308DF8065002238DF8083005ABDC
:104DB00003938DF8075020462A4B98470EE02A4B64
:104DC00098470446E6E72046284B9847002044E0F1
:104DD0009DF8153008F805300135EDB2B54238D2EE
:104DE0008DF814708DF8155000238DF8063032229E
:104DF00001A920461E4B9847A379DBB2022B0BD0AA
:104E000020461C4B9847322201A92046184B984750
:104E1000A379DBB2022BD6D101238DF806303222E2
:104E200001A92046124B9847A379DBB2022BCFD0C1
:104E30002046104B9847322201A920460C4B984738
:104E4000A379DBB2022BC3D02046084B9847002041
:104E500003E02046054B9847012006B0BDE8F081ED
:104E60000DE140003964400015E140004D64400010
:104E7000656440001566400070B506460C46104B50
:104E8000AA221A7011225A700222F0210D4DA84751
:104E9000012801D0002070BD220AE4B2084B1A702C
:104EA0005C709A70DC701A715C7100229A719022A9
:104EB000DA7102221A720922C2213046A84770BD57
:104EC000840F0020C94C400010B50022054B1A7019
:104ED00029B91121034B0122034CA04710BD102119
:104EE000F8E700BF840F0020C94C400070B50446AD
:104EF0000022104B1A700D4639B129210D4B0122A9
:104F000020460D4EB04715B970BD2821F6E7094D72
:104F1000AA232B7011236B702B460222F02120460E
:104F2000B047FF232B702B460122C0212046B047FB
:104F3000EAE700BF840F0020C94C400010B539B922
:104F40000022044B1A7001223621034CA04710BDE9
:104F50000322F6E7840F0020C94C400038B505460F
:104F60000C4BAA221A7012225A700222F0210A4C0B
:104F7000A047012801D0002038BD064B0322BF21E5
:104F80002846064CA047012801D0002038BD014B1F
:104F9000987838BD840F0020C94C4000814D4000F6
:104FA00010B50B462C227021014CA04710BD00BF4C
:104FB000C94C40002DE9F04182B000238DF8073044
:104FC0000139032926D8DFE801F00602040B134D4E
:104FD00002E0134D00E0134D8046012000240BE059
:104FE000114DF9E70DF10703024640460F4EB04759
:104FF0003C44E4B20134E4B201280CD123462F5DD5
:105000004FB1621CA95C012FECD902332B44781EEE
:10501000C0B2E9E7002002B0BDE8F081801F410086
:105020000C1F4100A820410038204100C94C40001D
:1050300038B51D4C0025A572E572257340F2DC538E
:10504000A3806423E3802580214621F8085F0620A1
:10505000164B98476580164B98470121154B98478A
:10506000012802D0104B987A38BD0122A272104B51
:1050700098470521104B9847034650B10A4AD3720E
:10508000002BEFD00A4B98470C4B9847064B5880A3
:10509000E8E7074CA0472946064B9847A04703215D
:1050A000054B98470346E9E7C40F0020A16D400077
:1050B00015E140004D51400061534000F152400065
:1050C000014B987A704700BFC40F002008B5164BFB
:1050D0009B7A6BB9144B1B7BD3B1134A118893880D
:1050E000D2889B1A99421DDC00220F4B1A7308BD0F
:1050F0000E4B98470E4B98470B4B1B89984203D891
:105100000022094B1A80E5E7C01A074B1880E1E737
:10511000054A11889388D2881344994202DB012200
:10512000014B1A7308BD00BFC40F002015E14000F9
:1051300081524000014B187B704700BFC40F002014
:10514000014B1888704700BFC40F002030B587B0EE
:1051500005460C4600238DF8073072228DF8082092
:105160008DF80B3001228DF809208DF80C200DF1FF
:105170000702049202228DF80A2005933C4B9847BF
:10518000322202A928463B4B9847002C3BD10124F0
:1051900002238DF80A3080238DF80B3001238DF81F
:1051A00007309C423CD08F238DF80B3003238DF8C1
:1051B0000A30012C3BD09DF8073003F0F00343F098
:1051C00002038DF8073002238DF80A30012C35D008
:1051D00007238DF80730F9238DF80B30012C34D0DC
:1051E00005238DF8073080238DF80B30012C33D048
:1051F0002846214B9847012C35D000221F4B1A70AE
:10520000204607B030BDA8238DF80B3001238DF860
:105210000730322202A92846164B98470446B7E7C2
:10522000322202A92846134B98470446BBE7322294
:1052300002A928460F4B98470446BCE7322202A930
:1052400028460C4B98470446C2E7322202A928465A
:10525000084B98470446C3E7322202A92846054B6B
:1052600098470446C4E70122044B1A70C8E700BF00
:1052700039644000656440004D644000110C00201A
:1052800030B587B004460023059301AB0493722325
:105290008DF8083001238DF809309C238DF80B30F0
:1052A00002238DF80C3003238DF80A300C4B9847FD
:1052B000322202A920460B4B9847054620460A4B4E
:1052C0009847012D04D00020084B187007B030BD5E
:1052D0009DF804009DF8053000EB032080B2F5E74F
:1052E00039644000656440004D644000110C0020AA
:1052F00030B587B004460023059301AB04937223B5
:105300008DF8083001238DF80930C0238DF80B305B
:1053100002238DF80C3003238DF80A300C4B98478C
:10532000322202A920460B4B9847054620460A4BDD
:105330009847012D04D00020084B187007B030BDED
:105340009DF804009DF8053000EB032080B2F5E7DE
:1053500039644000656440004D644000110C002039
:10536000F0B587B00646002305930DF107030493BB
:1053700072238DF8083001238DF80930D9228DF879
:105380000B208DF80C3002238DF80A304901C9B288
:1053900041F010018DF80710214B9847322202A9E5
:1053A0003046204B98470546D7238DF80B302123F4
:1053B0008DF8073001280BD030461B4B9847DC2373
:1053C0008DF80B3003238DF80A300024274608E0BF
:1053D000322202A93046134B98470546ECE70134C8
:1053E000A4B2012D18D1BFB9092C15D819200F4B23
:1053F000984730460A4B9847322202A93046094B5B
:10540000984705463046084B98479DF8073013F0FB
:10541000010FE4D00127E2E7384607B0F0BD00BF36
:1054200039644000656440004D644000A5D34000ED
:10543000F0B587B00446002505958A238DF808301D
:1054400001268DF809608DF80C600DF107030493B7
:10545000254B984755238DF807308DF80B500223C4
:105460008DF80A30322202A92046204DA847032396
:105470008DF807308DF80B60322202A92046A8472C
:105480008DF8076004238DF80B30322202A92046E4
:10549000A84707238DF8073030238DF80B303222D0
:1054A00002A92046A8470F278DF8077031238DF8F1
:1054B0000B30322202A92046A8478DF80770322609
:1054C0008DF80B60324602A92046A8478DF8077078
:1054D00033238DF80B30324602A92046A8472046D8
:1054E000034B984707B0F0BD396440006564400045
:1054F0004D644000F0B587B004460E46234B9847F4
:10550000002304938A238DF8043001238DF805309D
:105510008DF808300DF11703039334278DF80770C9
:1055200002238DF8063033788DF81730322201A926
:105530002046174DA8478DF8077033788DF817303F
:10554000322201A92046A8478DF8077033788DF8DC
:105550001730322201A92046A84735238DF807309D
:1055600073788DF81730322201A92046A8473623D8
:105570008DF80730B3788DF81730322201A9204614
:10558000A8472046034B984707B0F0BD3964400058
:10559000656440004D64400030B587B00546102377
:1055A0008DF808302022584B1A630A20574B984731
:1055B0002846574B984700230593E7238DF80B3077
:1055C0000DF10703049301238DF80C308DF8093099
:1055D00003238DF80A30322202A928464D4B984702
:1055E00004469DF8073043F001038DF8073002238D
:1055F0008DF80A30012844D006238DF80B300323A0
:105600008DF80A30012C43D09DF8073063F07F03FA
:105610008DF8073002238DF80A30012C3FD000238B
:105620008DF807300C238DF80B30012C3ED00D2364
:105630008DF80B30012C40D00E238DF80B30012C4F
:1056400042D00F238DF80B30012C44D0E7238DF886
:105650000B3003238DF80A30012C43D09DF807301E
:1056600023F001038DF8073002238DF80A30012C56
:105670003FD02846284B9847012C41D0204607B000
:1056800030BD322202A92846224B98470446B3E790
:10569000322202A928461F4B98470446B4E732221B
:1056A00002A928461B4B98470446B8E7322202A9B4
:1056B0002846184B98470446B9E7322202A92846E3
:1056C000144B98470446B7E7322202A92846114BEB
:1056D00098470446B5E7322202A928460D4B984761
:1056E0000446B3E7322202A928460A4B98470446EB
:1056F000B4E7322202A92846064B98470446B8E789
:105700000122064B1A70B9E700100E40A5D34000E5
:1057100039644000656440004D644000120C002074
:10572000014B1878704700BF120C002030B587B0CD
:1057300004460D4600220592A8238DF80830012367
:105740008DF809308DF80B200DF1070204928DF8C9
:105750000C3002238DF80A30124B9847012D0ED0E1
:10576000022D15D000238DF80730322202A92046E1
:105770000D4B984720460D4B984707B030BD03238B
:105780008DF80730322202A92046074B9847F1E7EF
:1057900002238DF80730322202A92046024B984797
:1057A000E8E700BF39644000656440004D64400094
:1057B00030B587B072238DF8003001238DF80130A9
:1057C00000238DF802308DF8033008228DF8042074
:1057D00004AA029203938DF81000C0F307238DF8FA
:1057E0001130C0F307438DF81230000E8DF813000E
:1057F0008DF81410C1F307238DF81530C1F307435A
:105800008DF81630090E8DF81710084CA047084B7C
:105810009847A04732226946064B98470546A0475D
:10582000054B9847284607B030BD00BF0DE140004A
:1058300039644000656440004D64400030B587B075
:105840000D4672238DF8043001238DF805300023B6
:105850008DF806308DF8073004228DF8082005AA4F
:10586000039204938DF81400C0F307238DF81530CC
:10587000C0F307438DF81630000E8DF81700184C52
:10588000A047184B9847A047322201A9164B9847CA
:105890000446012808D0124B9847144B9847012C16
:1058A0000DD0204607B030BD01238DF806300C4BDB
:1058B0009847322201A90C4B98470446EBE79DF824
:1058C00014309DF8152003EB02239DF8162003EBFE
:1058D00002439DF8172003EB02632B60E1E700BF52
:1058E0000DE1400039644000656440004D644000B3
:1058F0002DE9F04E82B08246894693461BB11E4682
:10590000002501272FE00127012F40D0012F49D08A
:10591000012F4DD0012F51D04FF4000301932F4B95
:1059200098470446012F4FD1019B13F4000F4BD031
:105930000A9920462A4B984700284DD101A92948A9
:10594000294B98470746EDE7EA18B25C4FEAC30EC9
:1059500002FA0EF211440133DBB2A342F4D3012F59
:105960000DD02544EDB228464D45CDD2A9EB050416
:10597000042C28BF0424E4B200231946EDE700F10B
:10598000201000F58070194B98470746E9E74FEA69
:105990000A4101F4FE0101F500011248134B98473A
:1059A0000746B3E749461248104B98470746AFE70A
:1059B000594610480D4B98470746ABE7F2210E4871
:1059C0000A4B98470746A7E71FB9052002B0BDE874
:1059D000F08E9DF80700F9E70620F7E7916A40008E
:1059E000A96A4000100120003D584000B157400016
:1059F0001801200014012000FC00200010B584B024
:105A00000A4B93E8030002908DF80C1032230093A8
:105A100002AB002205210120054CA047034610B926
:105A20000121044A1170184604B010BD4021410004
:105A3000F1584000130C002070B5074D4FF480461C
:105A40006E630A20054CA0472E6340F21310A04756
:105A5000034B984770BD00BF000E0E40A5D3400019
:105A6000FD59400030B583B00D463223009300232A
:105A7000024604213120074CA047044610B12046BD
:105A800003B030BD29460448044B98470128F6D09E
:105A90000524F4E7F1584000200120003D58400063
:105AA00010B584B08DF80C100B0A8DF80D300B0C6E
:105AB0008DF80E30090E8DF80F103223009303ABD2
:105AC000024604212120024CA04704B010BD00BFB3
:105AD000F158400008B5044B1B780BB1002008BDFD
:105AE000024B984708BD00BF130C0020FD59400031
:105AF0002DE9F04383B059B1012904D00124204697
:105B000003B0BDE8F08340F65D0740F6050503E00D
:105B100040F2DD7740F2857580464FF000094C4633
:105B200001E0002CEBD1BD42E9D225F00306002CA8
:105B3000F7D101A93046164B984704460028F0D10A
:105B4000019B8DF80030C3F307228DF80120C3F3C9
:105B500007428DF802201B0E8DF80330E9B2F3B234
:105B6000C91AC9B2C1F10403BE1B9E4228BF1E461A
:105B7000042E28BF0426F6B23246694408EB090019
:105B8000044B984735444E445FFA86F9C9E700BF95
:105B9000655A400091F5400028B1012801D000204D
:105BA0007047094800E0094800B583B001A9084BD7
:105BB000984728B9019B13F4006F02D0012000E040
:105BC000002003B05DF804FB4000350040003100C8
:105BD000655A400010B52DED028B82B0044601A934
:105BE0003548364B98470346F8B14BB3002B32D0BB
:105BF000002B3BD0DFED328A002B49D09FED308A5D
:105C000073B9DDED017AB8EE677AC8EE077A9FEDD9
:105C10002D7A67EE877AFCEEE77A17EE902A62819A
:105C2000184602B0BDEC028B10BD02A951F8043D2C
:105C300023801B0C63802448204B98470346D4E7FD
:105C400002A951F8043DA3801B0CE3801F481B4BA5
:105C500098470346CAE702A951F8043D03F01F0321
:105C600023721B48154B98470346C1E702A951F818
:105C7000043DC3F3094308EE903AF8EE688A9FEDBD
:105C8000158A68EE888A14480C4B98470346B3E798
:105C900002A951F8043DDBB208EE103AB8EE488A8A
:105CA00028EE888ADFED077A28EE278A0B48034B17
:105CB00098470346A4E700BF30082200655A400019
:105CC000000000000000C8423808220054082200EA
:105CD0000800200000401C4604082200140822008E
:105CE00000B583B001A941F23070094B98470346D3
:105CF00018B1184603B05DF804FB019921F00601C4
:105D0000019141F23070034B98470346F1E700BF21
:105D1000655A4000A15A400030B583B015460C4A80
:105D2000A2FB01231B090F3300930023024611201D
:105D3000084CA047044610B1204603B030BD2946A8
:105D40000548064B98470128F6D00524F4E700BF24
:105D50001F85EB51F1584000200120003D584000C4
:105D600010B582B096230093134602462020024CC1
:105D7000A04702B010BD00BFF1584000072801D96C
:105D80000120704710B584B08DF80C0030238DF8D9
:105D90000D3041F28833009303AB0022022114201E
:105DA000014CA04704B010BDF1584000F0B583B0DD
:105DB000032832D8DFE800F00209050747F6F0763D
:105DC00004E0184E02E0184E00E0184E00240127AF
:105DD0003D4604E09CB10F2C11D00134E4B20F2CED
:105DE00013D801AA0121A019114B9847B8B9002D69
:105DF000F0D09DF80430FF2BECD00025EAE79DF8A9
:105E00000430002BE9D10027E7E717B11DB10020CE
:105E100006E0002004E0012002E0002000E0002075
:105E200003B0F0BDF0FF0100F0FF0300F07F0200BF
:105E3000195D400070B582B006460020114B9847AE
:105E400020B14FF4BE65002423460BE001200D4B2A
:105E5000984718B90323184602B070BD0A4DF2E7FF
:105E60000134E4B20E2CF6D8002BF9D101AA01219D
:105E70002819064B984703460028F1D19DF80420C5
:105E80003255EDE7AD5D4000F0050200195D4000C0
:105E900030B587B01D201C4B98471C4C236C23F455
:105EA0000013236468461A4B984769462046194BED
:105EB0009847636823F47F436360636843F47F43D8
:105EC0006360042323610823236101232361626843
:105ED00022F08F026260104A032120460F4DA8472E
:105EE000002120460E4B9847636813F0800F01D1C4
:105EF000082222600B4B4FF000521A60702283F888
:105F00001D2307B030BD00BFF5C040000080034036
:105F100095494000294A4000495F4000794A4000C5
:105F2000BD49400000E100E00222014B1A607047C9
:105F300000800340024B1880024B1980704700BF5D
:105F4000BE000020C000002010B5064C206D80B2BD
:105F5000054B9847A06DE16D89B280B2034B98471D
:105F600010BD00BF008003401D6F4000355F400042
:105F7000014B1888704700BFBE000020014B1888F5
:105F8000704700BFC00000200D4B1B8840F689629F
:105F9000934205D90B4A12883E2A01D80320704744
:105FA000084A128840F689618A4203D93E2B01D8FB
:105FB00004207047934201D80220704701207047A7
:105FC000BE000020C000002008B50120034B984708
:105FD000034B186000B1012008BD00BF75CC400024
:105FE000D40F002008B54FF0FF31024B1868024B68
:105FF000984708BDD40F002095CC400010B5002371
:106000001A46194602480068024CA04710BD00BF5E
:10601000D40F00203DCB4000154B98421BD003F518
:10602000A033984219D003F58043984217D0A3F5C6
:106030004043984215D003F58043984213D0A3F50E
:10604000A033984211D003F56033984201D032203A
:1060500070471620704708207047092070470E20AF
:10606000704713207047142070471520704700BFF9
:1060700000C000404900B0FBF1F00338002302E00B
:1060800040080133DBB2FF28FAD8020202F47F4253
:1060900052FA80F01B0403F4E02318447047000018
:1060A0002DE9F843D0F80090037ADBB2012B00F021
:1060B0009D80044609F5C065087908B9BDE8F883F4
:1060C00017460E46012323720023E371E1604B4B18
:1060D00098478046B378022B08D07378012B18D0EC
:1060E00033781B0403F4FE036B603CE07378012BF0
:1060F00009D033781B0403F4FE0303F580736B604F
:10610000F378EB602FE033785B081B0403F58073B2
:10611000F5E733785B081B04E6E70323A37100234C
:106120002372237A002B64D02B6A13F4807F3AD138
:1061300013F0040F3BD139464046314B98470028B5
:10614000F2D00523A371002323722E4BC9F8003629
:106150002DE00423A37100232372E2E73946404671
:10616000274B9847B8B93379E2799B1A002BD8DDD1
:106170002B6A13F4807FD0D113F4007FE9D113F0A0
:10618000040FEBD0B168E379DBB25A1CD2B2E271F2
:10619000CB5C6B63E2E70523A37100232372194BE9
:1061A000C9F80036BDE70323A37100232372237AC5
:1061B00013B30223C9F800362B6A13F0010F0ED176
:1061C000394640460E4B98470028F5D00523A37169
:1061D000002020720B4BC9F80036BDE8F88300237D
:1061E00023720223A3710120BDE8F8830020BDE8DB
:1061F000F8830020BDE8F88300205FE7916A400043
:10620000A96A4000028000052DE9F84FD0F800A0EF
:10621000037ADBB2012B00F099800AF5C0660B7996
:1062200013B91846BDE8F88F91460D460446012380
:1062300003720023C371E160464B98478046AB78F8
:10624000032B11D06B78012B21D02B781B0403F486
:10625000FE0303F5805373602F79012F1DD00123B6
:10626000CAF8003600274DE06B78012B09D02B7857
:106270001B0403F4FE0303F588537360EB78F360AB
:10628000EAE72B785B081B0403F58853F5E72B78C6
:106290005B081B0403F58053DDE70323CAF80036CF
:1062A00030E00323A37100232372237A002B4FD005
:1062B000336A13F0010F43D149464046264B9847B5
:1062C0000028F5D00523A37100232372234ACAF8BE
:1062D0000026A6E70423A37100232372E5E7052324
:1062E000A371002323721D4BCAF80036DDE71BF0B3
:1062F000020F07D0A968E379DBB25A1CD2B2E2716F
:10630000326BCA54E379DBB22A799342CDD2D6F804
:1063100020B01BF4807FC4D11BF4007FDAD1494642
:1063200040460D4B98470028D9D1002FDFD12B795B
:10633000E2799B1A012BDAD1022333600127D6E7D9
:10634000002323720223A37101236AE7002368E775
:10635000002366E7916A4000A96A400002800005B8
:106360002DE9F04106468846046820461B4B9847B5
:10637000312801D9BDE8F0810546194B9847032320
:1063800023602423C4F8003641461648164B98472C
:10639000C4F81006002333720123B3716BB2002BD3
:1063A00007DB5A0905F01F00012181400F4840F822
:1063B0002210002B0BDB03F1604303F56143202225
:1063C00083F8002301200A4B98473061D2E705F09B
:1063D0000F05084B20225A55F4E700BF1960400012
:1063E000F5C040000000DC057560400000E100E001
:1063F00075CC400014ED00E008B500680B4B9847E1
:10640000312811D843B2002B0CDB5B0900F01F01CF
:1064100001228A402033064941F82320BFF34F8FE1
:10642000BFF36F8F034B984708BD00BF1960400052
:1064300000E100E049C1400008B54FF0FF310069BC
:10644000014B9847C0B208BD95CC400010B5002361
:106450001A4619460069024CA047C0B210BD00BFE1
:106460003DCB400008B5837963B18B78032B0BD803
:10647000DFE803F002050205044B984708BD044B12
:10648000984708BD002008BD002008BDA16040005D
:106490000962400080797047F8B50646036803F545
:1064A000C064256AC76815F0040F0BD0E26A12F0C9
:1064B000040F07D0BA78002A4DD0022A4BD0BA7800
:1064C000032A5ED015F0020F08D0E26A12F0020F24
:1064D00004D0BA78012A73D0032A71D015F4807FD2
:1064E0000DD0E36A13F4807F09D040F20733A36232
:1064F000002333720323B371FB6803B1984715F48B
:10650000007F0DD0E36A13F4007F09D040F2073317
:10651000A362002333720423B371FB6803B198476D
:1065200015F0010F16D0E36A13F0010F12D0BB78FB
:106530000BB1022B09D140F20533A3620023337261
:106540000223B371FB6803B19847BB78012B54D089
:10655000032B52D0F8BDF279D2B239798A4208D2EF
:10656000B868F279D2B2511CC9B2F171825C62632F
:10657000A5E70222C3F80026012262620422A26279
:106580009DE77A78012A11D03A78120402F4FE02CB
:1065900002F5805262603A79012A0DD00122C3F8D7
:1065A00000260422A262022262628BE73A78520835
:1065B000120402F58052EDE70322C3F80026F0E74B
:1065C000B868F279D2B2511CC9B2F171216B815411
:1065D000F179C9B23A79013A91420AD0F379DBB242
:1065E0003A7993427FF47AAF012363620223A36274
:1065F00074E70222C3F80026F0E740F20333A362F7
:10660000002333720223B371FB68002BA2D098479A
:10661000A0E7000070B4056805F5C0660379202B7B
:106620000BD9A3F12001CBB21A4C01219940216072
:10663000216521612163002211E0174CF5E7013348
:106640009BB2B3F52F7FFAD36163002301E00133DE
:106650009BB2B3F52F7FFAD321630132D2B2092A5C
:1066600001D80023EDE76161616032698023C5F8DC
:106670000036002301E001339BB2B3F52F7FFAD33C
:1066800032612423C5F8003600230372012383718D
:1066900070BC704700100E40000E0E4070B590B0F8
:1066A00000248DF835408DF836408DF837408DF850
:1066B00039408DF83A40ADF83E400F238DF8343024
:1066C0000A23ADF83C3001258DF838500DAA0B494E
:1066D00007A80B4EB0470DAA0A4901A8B0471023DE
:1066E000079A1360019A1360074B1D70074B1C70CB
:1066F00047F6FF72064B1A8010B070BD00C0024012
:10670000DDBB400000000340140C0020B811002045
:106710008212002042B110B420B119B1034B58606D
:1067200099605A805DF8044B704700BF140C00203C
:10673000154B1B783BB3144B5B8823B3124A52684A
:106740000AB311498968F1B1F0B583B000920193A1
:106750000E4D6A46694628460D4FB8474FF48036BD
:106760002E62094B9B6800930A4C6A466946204694
:10677000B847266201212846074DA8470121204637
:10678000A84703B0F0BD7047140C002000C10240C0
:1067900019BB40000001034031BB40000223034A03
:1067A000136202F580421362704700BF00C10240CD
:1067B00010B58CB00A4B9847069A136823F0100363
:1067C0001360009A136823F0100313600D20054C2A
:1067D000A0471220A0470022034B1A700CB010BD36
:1067E0009D67400049C14000140C0020064B1B78F7
:1067F0003BB1054B5888054BD3F80431C01A80B221
:1068000070470020704700BF140C002000C00240F9
:10681000094AD36D23F4FF4323F07F03C0F30E0036
:106820000343D36502F58042D36D23F4FF4323F085
:106830007F031843D065704700C00240014B1880A9
:10684000704700BF82120020014B1870704700BFD4
:10685000B81100200048704784120020004870479B
:10686000D80F0020704770472DE9F8434C4B9847EC
:1068700005464C4B9847044678E0A0EB070E1FFAFC
:106880008EFE0EF1F00E1FFA8EFE7EE03121002307
:1068900008E02F21FBE744480078C0B2012831D03E
:1068A00001339BB2994252D9DA1992B2EF2A01D937
:1068B000F03A92B23C4800780028ECD13B48B0F95D
:1068C000000035F9126006FB00F6F6134FEA830864
:1068D000DFF8E0C00CF8236008F10109C6F30726D1
:1068E0000CF8096034F9122000FB02F2D21308F10F
:1068F00002000CF8002008F10308C2F307220CF88C
:106900000820CDE735F9120034F91220024402EBD9
:10691000D272521012F5004F05DBB2F5004F03DBC7
:1069200047F6FF7200E0224A98005FFA82FC214E8F
:1069300006F823C000F10108C2F3072206F8082078
:1069400000F1020806F808C003303254A8E71A4BD9
:10695000A3F800E07744BFB2184B1F80EF2F01D996
:10696000F03F1F8089001348154B98474FF0FF31C7
:106970000120144B9847144B9847104B1F88B8427E
:10698000FFF47BAFC01B1FFA80FEBEF1300F3FF655
:106990007DAFBEF12F0F7FF67CAF302177E700BFD0
:1069A000556840005D684000B81100208212002048
:1069B0000080FFFFBC11002080120020200C00206E
:1069C0002D45400055D84000ED674000F8B5084C13
:1069D0004FF4804666630A20064DA8474027676348
:1069E0000A20A84727630A20A8472663F8BD00BFEE
:1069F000000E0E40A5D34000F8B578B9114D4FF404
:106A000080736B630220104CA0474FF080736B6360
:106A10000420A04701220D4B5A63F8BD094E4FF4E4
:106A200080737363094F02253D632846064CA047D7
:106A300001233B630420A0474FF080733363284653
:106A4000A047F8BD000E0E40A5D3400000100E4038
:106A500010B5084C4FF4804363630020064B984701
:106A60000220064B98470222054B5A63402363637A
:106A700010BD00BF000E0E40F9694000A5D34000D4
:106A800000100E400322014B1A60704730140E4074
:106A9000044B986801E0034B9868024B9B6898424E
:106AA000F9D1704730140E4010B584B001900C46F7
:106AB000064B98470390039B019A9B1AA34202D26C
:106AC000002004B010BD0120FBE700BF916A400028
:106AD00030B585B01E4B1B68002B31D01D4B98473D
:106AE0004FF0FF311A4B18681B4B9847EFF3108398
:106AF000B3FA83F35B09039372B6BFF35F8F00228F
:106B0000164B1A70039D80230093154B15221421F8
:106B10001448154CA04704462DB101220F4B1A70A2
:106B2000BFF35F8F62B600231A4619460848006813
:106B30000E4DA8470E4B984744B1002005B030BD1C
:106B400001200C4B9847024B1860C7E70120F5E77E
:106B5000240C0020E55F400095CC40002A02002074
:106B600064140020000A0E40110000203DCB4000BC
:106B7000FD5F400075CC400010B5074B98470022E0
:106B800013210648064B98470446064B9847B4FA2B
:106B900084F0400910BD00BFE55F4000000A0E40D0
:106BA00055BE4000FD5F400038B5114B9847EFF3EC
:106BB000108404B972B6002308E09A0002F580023E
:106BC0000C4951F82310116001339BB27F2BF4D98B
:106BD000002212210848094B9847C5B204B962B691
:106BE000074B98470DB1002038BD012038BD00BFCC
:106BF000E55F400064140020000A0E4055BE4000CE
:106C0000FD5F400010B400240EE0400080F007005B
:106C1000C0B20133DBB2072B05D810F0800FF4D1DE
:106C20004000C0B2F5E70134944204D211F8013BB0
:106C300058400023EFE75DF8044B704770B50646F7
:106C4000002501E02C44A5B2B5F5007F15D20E4B0E
:106C5000E918EA5CFF2A14D06B1C0B481B5C033359
:106C6000DCB2B242EED1621EFF20084B98472B19CE
:106C7000074A9B5C9842E5D101E04FF6FF75284634
:106C800070BD4FF6FF75FAE764140020056C4000F4
:106C90006314002008B5094B1B781BB1022B01D0EF
:106CA000074808BD074B9847012804D10122034B30
:106CB0001A70034808BD002008BD00BF280C002042
:106CC00064140020D16A400008B5094B1B781BB141
:106CD000022B01D0074808BD074B9847012804D173
:106CE0000122034B1A70034808BD002008BD00BFF5
:106CF000280C002064140020D16A4000A8B108B517
:106D00000346B1F5007F12D28818B0F5007F01D993
:106D1000002008BD08461946064B1844064B984704
:106D20000222064B1A70012008BD00207047002087
:106D300008BD00BF6414002091F54000280C00201D
:106D400008B5064B1B78022B01D0002008BD044B70
:106D500098470128FAD1034B984708BD280C00201A
:106D6000796B4000A96B400090B110B504460268F1
:106D7000094B9A4201D0002010BD9A220146FF2003
:106D8000064B984794F89A30984203D0002010BDE3
:106D900000207047012010BD5FE1AD5A056C400036
:106DA00010B50C46084B9847B0F5007F01D3002082
:106DB00010BD811C054B5A1C125C19442046044B23
:106DC0009847012010BD00BF3D6C400064140020B6
:106DD00091F5400008B5054B9847B0F5007F02D209
:106DE000034BC05C08BD002008BD00BF3D6C4000E7
:106DF00065140020FF292FD02DE9F843D61CF6B2E8
:106E00008419B4F5007F03D94FF6FF70BDE8F8830D
:106E100017460C4605460221114A1170DFF84C80D6
:106E200000EB080900F80840421C02F8087008440A
:106E30003A46194640440B4B98477C190234721E5F
:106E40004946FF20084B984708F80400E81980B22B
:106E5000033080B2BDE8F8834FF6FF70704700BF83
:106E6000280C002091F54000056C400064140020BF
:106E700010B5A8B0224B98470446224B984708B952
:106E800028B010BD9B22214601A81F4B98474FF404
:106E90000072FF211D481E4B984702AB10220121B2
:106EA00000201C4CA0474FF6FF73984203D026AB3E
:106EB00003220221A0474FF6FF73984205D00DF13F
:106EC0009B0301220321134CA0474FF6FF73984206
:106ED00004D027AB012204210E4CA0474FF6FF73CC
:106EE000984205D00DF19D0301220521094CA047D0
:106EF0004FF6FF739842C3D0074B9847C0E700BFD7
:106F0000956C4000696D400091F5400064140020CC
:106F10008DF74000F56D4000416D4000044B188036
:106F2000044A1378591C1170034A22F81300704761
:106F300068180020290C00206816002008B5194B9D
:106F40001B8807EE903AF8EE677A9FED177A67EEA6
:106F5000877A164BC3ED007AF7EE006A76EEE76AA1
:106F600087EEA67ADFED126A67EE267A114BC3ED43
:106F7000007A86EEA77A17EE100A0F4B9847DFEDDE
:106F80000F7A07EE100A27EE277ADFED0D7A77EEFB
:106F9000C77ADFED0C6A86EEA77A0B4B83ED007A99
:106FA00008BD00BF68180020010880396416002061
:106FB00000401C46701800207DE1400033139543CB
:106FC00000F05745C47D7B496C180020BFF35F8FEC
:106FD000024B1868BFF35F8F704700BF6C1800202A
:106FE00068B90F4A1368B3F1FF3F0AD00320B3F129
:106FF000333F0ED013B9536803B902207047094AD2
:10700000F0E75168B1F1FF3F01D00320EFE7002026
:10701000EDE75168B1F1333FECD10120EAE700BF61
:1070200000C0470000E0470018B101280FD002203F
:1070300070470B4841F6F87383B130B4C518C45893
:107040008C4206D0083B002BF8D1012004E0054813
:10705000F0E76B681360002030BC70470120704778
:1070600000C0470000E0470070B505460020124C04
:10707000A04706460120A0471DB1012D12D00220D5
:1070800070BD022803D0022E07D0022070BD012E51
:1070900001D0012070BD002070BD012801D000206A
:1070A00070BD70BD022E05D0022801D0022070BD37
:1070B000012070BD002070BDE16F4000F8B50446AE
:1070C0000F461646450A094B984704F4FE7000F532
:1070D00080031F605E602A4601210548054B9847E2
:1070E0000446054B98472046F8BD00BFE55F4000C9
:1070F000000A0E4055BE4000FD5F4000012909D046
:1071000002290CD1002108B538B906480A46064BB9
:10711000984708BD4FF03331F5E70448F6E7012002
:10712000704700BF00C04700BD70400000E047004E
:1071300038B518B101280DD0022038BD0A4C0823FB
:10714000B3F5005F0ED2E018E558B5F1FF3F03D06C
:107150000833F5E7054CF2E7054B984708B10220E4
:1071600038BD38BD012038BD00C0470000E04700F1
:10717000BD70400010B568B140F2F234074B98473B
:10718000224607210648074B98470446064B984776
:10719000204610BD40F2E234F0E700BFE55F40005A
:1071A000000A0E4055BE4000FD5F400038B5044661
:1071B0000D460120034B98472A462146024B98472B
:1071C00038BD00BF6970400029704000F8B5044622
:1071D0000D4600200C4B984706462A4621460B4B8D
:1071E0009847012800D0F8BDB6FA86F77F093946DE
:1071F0003046074B984708B10220F4E72A4621465B
:107200003846024B9847F8BD697040003171400024
:107210009972400030B583B000230193044660B9F1
:10722000164D17490023B3F5006F24D251F82320DF
:10723000B2F1FF3F04D10133F5E7124D1249F1E7F6
:107240002046124B9847044610B1204603B030BD8B
:1072500001A928460E4B984740B9019901312846AB
:107260000C4B98470028F0D00124EEE70121284676
:10727000084B9847F6E70024E7E700BF0120FFFF2F
:1072800000C047000220FFFF00E04700757140008A
:10729000AD714000CD71400070B582B005460E461C
:1072A0000846284B9847012806D001213046264B36
:1072B00098470446002841D1002400E00134234BC4
:1072C0001B689C4215D201AA214B53F82410284672
:1072D000204B9847022830D00028EFD1019A1C4B50
:1072E00053F8241030461C4B98470028E6D0012460
:1072F00024E02846194B98470446F8B90221304645
:10730000114B98470446C8B985B9154D02A9002309
:1073100041F8083D2846134B984748B90099013178
:107320002846114B984748B1012407E00F4DEDE77F
:10733000012128460C4B9847F5E70124204602B06E
:1073400070BD00BFE16F4000FD704000D80000201C
:10735000C400002029704000317140007571400068
:107360000120FFFFAD714000CD7140000220FFFF02
:1073700010B500200E4B9847044608B1204610BDBA
:1073800001200B4B984704460028F7D10221094BF6
:10739000984704460028F1D101210748074B984738
:1073A00008B10124EAE701210548044B9847E5E7C5
:1073B00075714000FD7040000120FFFFCD7140005D
:1073C0000220FFFF38B50020284DA84704460120C1
:1073D000A847012C20D034B1022C35D0244B98473B
:1073E0000346184638BD012806D0022810D10020D7
:1073F000204B98470346F4E700201E4B984703466E
:107400000028EED1022101201B4B98470346E8E7F4
:10741000174B98470346E4E738B1022810D1002102
:107420000120164B98470346DBE70120114B984794
:1074300003460028D5D102210F4B98470346D0E7D9
:107440000B4B98470346CCE728B1022808D1084BDC
:1074500098470346C5E70120064B98470346C0E717
:1074600001210020054B98470346BAE7E16F400031
:107470007173400015724000FD7040009972400029
:1074800008B50A4B984708B1012008BD2022084BD7
:107490005A630A20074B9847074B9847074B984772
:1074A000012801D0002008BD08BD00BF21574000C1
:1074B00000100E40A5D3400015E140009955400052
:1074C00030B587B0174B984704468A238DF80830AB
:1074D0000025059501238DF809308DF80C300DF14C
:1074E00007030493104B98478DF80B5003238DF836
:1074F0000A30322202A920460C4B984720460C4BFA
:107500009847022806D0002520460A4B984728466F
:1075100007B030BD9DF80730092B01D00025F3E7F7
:107520000125F1E715E14000396440006564400041
:10753000956440004D64400030B587B01A4B9847C1
:10754000044600220592A8238DF8083001238DF807
:1075500009308DF80B2001AA049202228DF80C202C
:107560008DF80A30114B9847322202A92046104B61
:10757000984720460F4B9847022806D00025204602
:107580000D4B9847284607B030BD9DF8043033B9FD
:107590009DF8053013F0F80F03D00025EFE7002524
:1075A000EDE70125EBE700BF0DE140003964400045
:1075B00065644000956440004D64400008B5034B8D
:1075C000984708B1002008BD012008BDD55A4000E9
:1075D00030B587B0184B98470446002305937223B3
:1075E0008DF8083001238DF8093092228DF80B2098
:1075F0000DF1070204928DF80C3003238DF80A3048
:107600000E4B9847322202A920460D4B9847204640
:107610000C4B9847022806D0002520460A4B984775
:10762000284607B030BD9DF80730442B01D0002517
:10763000F3E70125F1E700BF15E1400039644000A0
:1076400065644000956440004D64400070B586B0AC
:10765000002832D11C4B98470446002505959823F5
:107660008DF8083001268DF809608DF80A50022344
:107670008DF80C3001AB04938DF80B502046134B62
:10768000984736238DF804308DF80550322202A930
:1076900020460F4DA8478DF80A60322202A92046E5
:1076A000A84720460B4B984702280AD000252046C1
:1076B000094B9847284606B070BD084B98470446CA
:1076C000CBE73546F3E700BF0DE1400039644000E9
:1076D00065644000956440004D64400015E1400041
:1076E00038B50020064CA04705460120A047012DD3
:1076F00001D0002038BD0128FCD0002038BD00BFDB
:107700004D7640002DE9F0473D4BD3F858801920C5
:107710003C4B98474FF496703B4B9847002409E048
:107720003A4B98473A4B23F814000320364B9847BE
:107730000134E4B21F2CF3D9364B98478246002619
:107740003746354634463FE0314931F813100A4494
:107750000133DBB21F2BF7D94FEA5219B9F10A0FE7
:1077600017D92A4B9847631CDBB2294A22F8140028
:107770001F2B1DD81C46A9F1FA0398421AD309F110
:10778000FA02904225D80135EDB2202D13D90126F9
:1077900011E0B8F1000F05D0194BC3F85880002054
:1077A000BDE8F0870020174B98470020BDE8F08720
:1077B0000024E0E700250320134B98474FF47A613B
:1077C0005046154B984707462FB926B900231A464D
:1077D000C0E70025EFE7B8F1000F07D0084BC3F86A
:1077E000588057B936B10120BDE8F0870020054B1D
:1077F0009847F6E70020BDE8F0870020BDE8F08755
:1078000000000140C94B4000A5D34000154C40008A
:1078100074180020916A4000A96A4000004870472F
:1078200048214100062070472DE9F84305460E46E1
:1078300017460A469C211E4B98470446451B40B1FB
:10784000731B052B05D94378552B07D010237B706C
:1078500001E000237B702046BDE8F88390F80280A9
:10786000C37888EA0303FF2B02D011237B70F2E771
:1078700090F80490437909EB03291FFA89F9B9F1CB
:107880003A0F06D84D440635AE4205D200237B7030
:10789000E1E712237B70DEE74A46811D381D054B68
:1078A0009847A7F8029087F8008001237B70D2E701
:1078B000F1F4400091F5400010B553889C1D8C42B6
:1078C00019D83A2B01D9002010BD11469C23037012
:1078D00055234370137883701378DB43C370937818
:1078E000037153881B0A4371528804310630034BDD
:1078F0009847012010BD002010BD00BF91F5400049
:1079000070B582B004460378253B332B00F2198210
:10791000DFE813F0450017021702170217023400C0
:10792000170217021702170217021702170217028F
:10793000170217021702170217021702170217027F
:107940001702170217021702170217023E01170249
:107950001702FA0017021702170217021702BA01DC
:1079600013015C0017021702170217021702170211
:10797000170265017900CB00A600E3009C4C2A2386
:1079800023709C4DA84760809B4B98470646A847AC
:1079900002463146201D994B984702B070BD012028
:1079A000974B984780B2924B588010B945221A7075
:1079B000F3E794490120944B984718B125228C4B4A
:1079C0001A70EAE745228A4B1A70E6E74388032BD0
:1079D00005D0874B00225A8045221A70DDE70379D3
:1079E0008DF8043043798DF8053083798DF80630B1
:1079F000864B984701A9864B98477D4B00225A80B9
:107A000024221A70C9E74388012B05D0784B002245
:107A10005A8045221A70C0E703790F2B05D9744BA1
:107A200000225A8045221A70B7E77A4B9847704A6D
:107A30005523137020235380237900EB43100668ED
:107A400045688468C16856609560D46011610669B4
:107A500045698469C16956619561D46111629CE789
:107A60004388212B05D0624B00225A8045221A7090
:107A700093E701790F2905D95D4B00225A804522F1
:107A80001A708AE7202249010530634B9847012884
:107A900005D0574B00225A8045221A707DE7544B7F
:107AA00000225A8024221A7077E743882BB1504B6A
:107AB00000225A8045221A706FE7584B98470128D8
:107AC00005D04B4B00225A8045221A7065E7484B7F
:107AD00000225A8024221A705FE743882BB1444B5E
:107AE00000225A8045221A7057E74D4B984728B913
:107AF0003F4B00225A8024221A704EE73C4B002252
:107B00005A8045221A7048E74388012B05D0384B2C
:107B100000225A8045221A703FE70079414B98476E
:107B200028B9334B00225A8024221A7035E7304B93
:107B300000225A8045221A702FE74388082B05D06F
:107B40002B4B00225A8045221A7026E7037942798E
:107B500003EB0223827903EB0243C079217A627A34
:107B600001EB0221A27A01EB0241E47A01AA01EBC6
:107B7000046103EB00602C4B984700287FF40DAFA5
:107B80001B4B019A5A604B221A7004225A8004E758
:107B90004388063B9BB21F2B05D9154B00225A8008
:107BA00045221A70F9E64379807903EB0023E079E6
:107BB00003EB0043207A04F10902217903EB006012
:107BC0001A4B984728B90A4B00225A8024221A706F
:107BD000E3E6074B00225A8045221A70DDE643880F
:107BE00033B3034B00225A8045221A70D5E600BFFA
:107BF000B4180020257840001D78400091F5400021
:107C0000D56D4000B8180020A16D400015E140007E
:107C1000F5544000C96C4000FD6C4000416D4000CF
:107C2000D55A40007D5D4000195D4000615D400017
:107C30000020474B1871474B984720B1444A1379AD
:107C400043F0010313710120424B984720B1404A91
:107C5000137943F00203137102203E4B984720B181
:107C60003B4A137943F0040313710320394B9847BF
:107C700020B1374A137943F008031371344B0122C2
:107C80005A8054221A7088E64388012B05D0304B65
:107C900000225A8045221A707FE60379463B102B5A
:107CA00049D8DFE803F03F480948484812484836B9
:107CB0002D48481B48482400274B9847244B1871EF
:107CC0004A221A7001225A8067E6244B9847204BBB
:107CD00018714A221A7001225A805EE6204B98479A
:107CE0001B4B18714A221A7001225A8055E61D4B0F
:107CF0009847174B18714A221A7001225A804CE695
:107D0000194B9847124B18714A221A7001225A8057
:107D100043E6164B98470E4B18714A221A700122FF
:107D20005A803AE6124B9847094B18714A221A704A
:107D300001225A8031E6064B45221A7000225A80F1
:107D40002BE6034B00225A8045221A7025E600BF1D
:107D5000B4180020AD5D400081744000C174400043
:107D600039754000BD754000D1754000E176400096
:107D70000577400000487047B4180020F0B583B084
:107D8000EFF31083B3FA83F35B09019372B6BFF389
:107D90005F8F0022364B1A70019E364B1B68364AA5
:107DA00015682B447F2B2AD8324B1C682246334956
:107DB00033482844334B98472C442F4B1C600022F7
:107DC0002C4B1A602EB10122294B1A70BFF35F8F22
:107DD00062B62D4A284B196829482C4B9847014612
:107DE000D0B1274BC31A284842881A44951D4478BD
:107DF000012C15D044BB802B1CD900242AE01D4A3D
:107E0000136814682C441B1B03F18004204A137868
:107E100043F001031370C9E70024174B1C6019E0FD
:107E20001748154F3E68761B32464119194B984743
:107E30003E600FE0104D2C68E41A22461048154BA6
:107E400098472C60002405E00133802B05D90024DD
:107E5000094B1C60204603B0F0BD0948064D2C6854
:107E6000E41A2246C1180B4B98472C600024F1E716
:107E70002A020020FC1B00200C1C0020541C0020A7
:107E8000FC1A002091F54000101C002029784000C9
:107E9000081C0020C5F6400010B5174B9847174B3B
:107EA00018600DE0164B195D1648174B98470134C2
:107EB000E4B2164B1B689C42F4D30022134B1A60A9
:107EC0000120134B9847134B98470128F8D11248CB
:107ED000124B9847124B9847024680210848114B95
:107EE00098470128ECD10E4B984743880633074A40
:107EF00013600024DDE700BF3DD64000001C0020D9
:107F00007C1B002000820140DFC24000041C0020D6
:107F1000A5D340007D7D4000101C00200179400069
:107F2000757D4000B978400030B583B0802422468A
:107F300000211B481B4DA847224600211A48A8478C
:107F400000231A4A13601A4A13601A4A13701A4A15
:107F500010215166C2F8901051655162C2F880102C
:107F6000116F21F010011167516F21F0100151675D
:107F7000124A4FF400211160202182F813130121CD
:107F80000F4A91600193009322460E490E480F4C10
:107F9000A047012802D00E480E4B984703B030BDD1
:107FA000541C00208DF740007C1B0020FC1B00208F
:107FB000041C0020081C0020000E0E4000E100E020
:107FC0000082014050214100997E4000EDD04000E8
:107FD000582141003DEF4000104B1B6913F0010F89
:107FE00012D00E4B5B6913F0010F0DD00C4B1B68C8
:107FF0007F2B0AD90B4A137843F001031370074B08
:108000009A69094B83F87F207047054A1368591C09
:108010001160024A9169044AD154704700820140BC
:10802000FC1B0020081C0020541C002070B50646D4
:108030000D46094B98470446002040B92946204682
:10804000064B984728B93046054B9847F5E701207D
:1080500070BD002070BD00BF916A4000A96A400059
:10806000E994400010B54FF47A722B4B1A8004E06B
:108070004022002129482A4B9847274B188880B274
:10808000284B9847254C2323237014236370264BD9
:108090009847C0F30F23A370E070244B9847C0F3B8
:1080A0000F2323716071224B9847C0F30F23A371F4
:1080B000E071204B9847C0F30F23237260721E4B70
:1080C0009847C4F80A001D4B1B7807EE103AB8EE2B
:1080D000477A9FED1B6A27EE067ADFED1A6A37EEC4
:1080E000667A17EE103AC4F80E30174B1B7807EE7D
:1080F000903AF8EE677A67EE867A77EEE67A17EED0
:10810000903AC4F81230114B98470028B0D0322171
:1081100020460F4B9847ABE73E1D0020F81C00207F
:108120008DF74000A5D34000154C40004151400060
:10813000715F40007D5F4000CD6F4000E100002096
:10814000B4C8363F6FDB4A42E200002035E1400010
:108150002D804000F0B583B0A04B9847A04B18602D
:10816000402200219F48A04B9847B2E19F4B98477F
:108170009F4BBB221A601A225A609E4A936823F0D2
:108180007F4323F4706343F0254343F470639360AB
:10819000994B1360A8E193490B462A2203F8012B5F
:1081A000964A1068C1F8010092889A809FE10120E8
:1081B000934B984728B98B4B45221A7002225A706C
:1081C00098E18849252301F8013B01208D4B984710
:1081D00090E108208A4B984728B9824B45221A70B3
:1081E00002225A7089E17F49262301F8013B0820C9
:1081F000844B984781E10920814B984728B9794BF6
:1082000045221A7002225A707AE176497E2301F8DB
:10821000013B09207B4B984772E1C4F30723012BF4
:1082200016D023B1022B11D04FF0FF3000E076487A
:10823000B0F1FF3F14D001A9744B984750B9694B76
:108240005A221A70019AC3F801205DE17048EFE7E5
:108250007048EDE7634B45221A7002225A7053E1D1
:10826000604B45221A7001225A704DE124225D4B69
:108270001A704CE15B4B45221A70674A12785A70AB
:1082800048E1664B1B780F2B05D9564B45221A70D7
:1082900001225A7041E1624B9847524A55231370AC
:1082A000202353705D4B1B7800EB4310D0F800E0A7
:1082B00047688668C168C2F802E0C2F80670C2F872
:1082C0000A60C2F80E10D0F810E047698669C169EB
:1082D000C2F812E0C2F81670C2F81A60C2F81E1096
:1082E0001BE1404B4B221A7004225A706A444D4BDA
:1082F00019684D4B18684D4B984720B9394B019A76
:10830000C3F802200CE10022494B1A6008E1354B0A
:1083100054221A7000205870464B984720B1314AB9
:10832000537843F0010353700120424B984720B12A
:108330002C4A537843F00203537002203D4B984778
:1083400020B1284A537843F0040353700320394B7B
:108350009847002800F0E780224A537843F008034A
:108360005370E0E0344B1878072805D91D4B45229F
:108370001A7001225A70D9E0304B984718B924225C
:10838000184B1A70D2E0174B45221A7003225A700C
:10839000CCE02B4A234B1968234B1868294B98478C
:1083A00018B924220F4B1A70C3E00E4B45221A70E5
:1083B00003225A70BDE00B484E2300F8013B224BCC
:1083C0009847002800F0B880204B4FF020321A6008
:1083D0005A609A60C3F80B20AEE000BF3DD6400063
:1083E0002C0C0020481D00208DF74000C1E040000B
:1083F00090140E4000140E40080000A5F02141002A
:10840000D56D4000A16D40000110FFFFAD7140002F
:108410000310FFFF0210FFFF401D00203C1D002045
:10842000C96C4000441D0020381D0020195D40002B
:108430004A1D0020AD5D4000D41C00207D5D400041
:10844000D81C0020615D4000355E4000491D0020C1
:108450004A223F4B1A70C4F30724463C102C2DD8F7
:10846000DFE804F0272C092C2C2C0E2C2C221D2CA0
:108470002C132C2C1800374B9847354B58705DE067
:10848000354B9847324B587058E0344B9847304B37
:10849000587053E0324B98472D4B58704EE0314B9B
:1084A00098472B4B587049E02F4B9847284B5870F2
:1084B00044E02E4B9847264B58703FE0244B452212
:1084C0001A7001225A7039E0402200212048284BBE
:1084D00098474FF0FF310120264B9847044600286B
:1084E000F7D042283FF442AE2A2C3FF454AE252C5C
:1084F0003FF45DAE262C3FF46CAE7E2C3FF47BAE99
:10850000E5B25A2D3FF489AE242C3FF4AFAE452C92
:108510003FF4B0AE552C3FF4B4AE4B2C3FF4E1AE7B
:10852000542C3FF4F4AE442C3FF41CAF412C3FF4E8
:1085300030AF4E2C3FF43FAF4A2D89D00E4B9847B9
:108540000028C1D0322102480C4B9847BCE700BF3D
:10855000481D002081744000C174400039754000FE
:10856000BD754000D1754000E176400005774000C0
:108570008DF7400055D8400035E140002D80400087
:1085800010B500230322014602480068024CA047B0
:1085900010BD00BF2C0C00207DD9400010B584B068
:1085A000002304AA42F8043D09490C680092032202
:1085B00001462046074CA047039B3BB14FF0805239
:1085C000054B1A60BFF34F8FBFF36F8F04B010BD20
:1085D0002C0C002029DA400004ED00E010B582B038
:1085E000002301930122009280220C490C480D4C7B
:1085F000A047012802D00C480C4B98470023019358
:108600000122009280220A490A48064CA04701280C
:1086100002D00948054B984702B010BD78214100AF
:1086200055814000EDD04000882141003DEF4000E1
:10863000B821410065804000C421410070B584B07C
:10864000044603782A2B5AD02378252B5BD0237835
:10865000262B5CD023787E2B5DD023785A2B5ED0DE
:108660002378532B62D02378472B6CD02378672B49
:108670007AD02378462B00F082802378522B00F0AA
:1086800085802378502B00F095802378492B00F0CB
:10869000AD802378422B00F0B3802378552B00F077
:1086A000B3802378572B00F0B6802378562B00F048
:1086B000C58023784C2B00F0C88023784B2B00F02A
:1086C000D2802378542B00F0EA802378442B00F0EA
:1086D000EA802378412B00F0ED802378592B00F0BD
:1086E0000B8123784E2B00F0208123784A2B00F059
:1086F00020812378402B00F04D8104B070BD2A20EA
:108700008F4B9847A0E725208D4B98479FE7262061
:108710008B4B98479EE77E20894B98479DE7607872
:10872000000240F05A00864B984799E7637833B9C6
:108730000120844B98472420814B984793E70020E1
:10874000804B9847F7E76378A07800EB032080B26E
:1087500010F4004F05D17C4B98472420784B984764
:1087600084E747F6FF70F6E76378A07800EB032014
:1087700000B2764B98472420714B984779E7607890
:10878000734B984724206E4B984776E76278A3781E
:1087900003EB02239BB2092B05D96E4A13802420D8
:1087A000674B98476DE701226B4B1A704520644B6D
:1087B000984766E763785BB1012B10D00022674BC6
:1087C0001A700122644B1A7045205D4B98475CE794
:1087D0000220634B98472420594B984755E70120C6
:1087E0005F4B98472420564B98474EE76278A37812
:1087F00003EB02235B4A13800520594B984748E757
:1088000042204F4B984748E76278574B1A705520E3
:108810004B4B984745E761780F2908D8202249013A
:10882000A01C524B98472420454B98473DE7012216
:10883000494B1A704520424B984736E70720484B72
:10884000984724203E4B984733E7494B62781A708B
:10885000A2785A70E2789A700620414B98472420FB
:10886000374B984729E76378A27803EB0223E27835
:1088700003EB0243227903EB02633E4A1360637900
:10888000A27903EB0223E27903EB0243227A03EBA2
:108890000263394A13604B20294B984711E7542053
:1088A000274B984711E76278344B1A704420244BC9
:1088B00098470EE76278531EDBB21F2B06D90122C0
:1088C000254B1A7045201E4B984706E72A4B1A6025
:1088D000A378E17803EB0123217903EB014361796C
:1088E00003EB016323490B60A11D2548254B9847E5
:1088F0004120134B9847F0E6002604AD45F8046D7F
:10890000214B984700953346012204211F4DA8476B
:10891000039B002B3FF4E5AE4FF080521C4B1A60D6
:10892000BFF34F8FBFF36F8FDBE64E20044B9847AA
:10893000DBE6607800024A30014B9847D9E600BF79
:108940009D85400049684000116840003D68400036
:10895000C94B40003E1D0020401D0020EF1D00209F
:10896000E99340000A1E00203C1D0020FD6C4000E1
:10897000EC1D0020381D0020441D0020D41C0020C8
:10898000D81C002091F54000CD8A400029DA400033
:1089900004ED00E001200C4B98470C4B984703ABCB
:1089A0000093002301220421094CA047039B002BC4
:1089B0003FF4A3AE4FF08052064B1A60BFF34F8FC7
:1089C000BFF36F8F99E600BF158F4000CD8A40003E
:1089D00029DA400004ED00E08388B3F59F5F0DD0F5
:1089E000B3F5706F17D0B3F5206F21D0B3F5A05F4A
:1089F0002AD0B3F5706F33D000207047C288B2F52B
:108A00001F6FEDD14289A2F5E752093A92B2C62A08
:108A1000E6D801207047C288B2F5F06FE3D14289F1
:108A2000A2F50B52053A92B2C62ADCD80220704752
:108A3000C288B2F5206FD9D14289A2F6553292B2DE
:108A4000C62AD3D804207047C288B2F5206FD0D18F
:108A50004289A2F6553292B2C62ACAD8042070477B
:108A6000C388B3F5F06F01D0002070474389A3F5A8
:108A7000B8530D3B9BB2C62B01D803207047002092
:108A800070470000F8B505460E460024204601E078
:108A90000134A4B22746B4EB960F14D215F8241073
:108AA00005EB84035A7801EB02219A7801EB02412D
:108AB000DB7801EB03610028EAD107F54060800014
:108AC000014B9847E4E7F8BDA15A4000014B1868F4
:108AD000704700BF340C0020014B1878704700BF6E
:108AE000330C0020F0B583B001238DF80330944B94
:108AF0009847944B18600023019306E04FF0FF3332
:108B000001AA00210846904CA047019B13F0010FD9
:108B1000F4D040F213108D4B98478D4B98474FF48B
:108B200080718C4B18688C4B984706E04FF0FF33F0
:108B300001AA00210846844CA047019B13F0020FB4
:108B4000F4D01920814B9847844B4FF480721A63FC
:108B5000DB6B13F4004F19D0814B98470F20814BEA
:108B6000984701467D48804B984700227F4B1A70FA
:108B70000DF1030104207E4B9847002834D09DF866
:108B8000033083F001038DF803302DE0794B9847D3
:108B9000E4E70022754B1A70704C4FF480756563E2
:108BA00019206A4B984725632FE0734B984743E0A1
:108BB000704B98470F206B4B9847014667486A4BAC
:108BC000984724206D4B9847684B1B78002B3BD16E
:108BD0006B4B984700284AD10022644B1A709DF8CD
:108BE0000330002B40F02F811420584B984700236E
:108BF00001AA04211846544CA047019B13F0040F0E
:108C0000E2D05A4B1B78002BC3D10F20554B98470D
:108C1000014652485B4B9847564B98475A4B9847EA
:108C20004B4B98474B4C4FF4807120684A4B984708
:108C30002268564B9A42B8D0484BDB6B13F4004F76
:108C4000B6D0474B9847B5E74D4B984718B1504BB6
:108C500098470028BCD10022444B1A703F4C4FF477
:108C6000807565631920394B98472563B0E7484BF9
:108C700098470028B0D03D4B1B78002BAFD1002087
:108C8000444DA847444C20700120A847434B18701E
:108C90002378002BA3D00028A1D00126334B1E70CF
:108CA0003F4C20463F4B984720463F4B984707464E
:108CB0004FF4FA70254B98470020A847364C207097
:108CC0003046A847354B1870237803B118B90022F5
:108CD000264B1A7083E739460020344CA0473946AA
:108CE0003046A0470A20324B9847002870D1314CBB
:108CF00000212046304B98472378112B79D0002152
:108D000008462E4CA04700210120A0479DF80330C3
:108D1000002B00F08D802A4B9847002800F08880B7
:108D2000284B1B78002B78D00124274B1C70214640
:108D30000020264DA84721462046A8474FE700BF00
:108D40003DD64000340C0020D9D84000A5D34000C7
:108D5000FD594000DC000020858A4000000E0E40D6
:108D6000A54C4000D3BC4000AFBC4000330C0020F9
:108D7000A16D4000814C4000E15C400081854000D5
:108D800061E14000B3BC4000395A4000F821410085
:108D90006DE14000995B4000310C0020320C002056
:108DA000E01D0020D55B4000D9894000B54F400050
:108DB000D56D4000881D0020F15A4000C94E40008A
:108DC000C1504000E0000020300C0020ED4E40007B
:108DD000002402A921F8084D0A20344B9847BDF819
:108DE00000102046324CA047BDF800103046A04786
:108DF0007DE76378002B82D1A378002B7FF47FAFCF
:108E0000E378892B7FF47BAF254621460020294C4F
:108E1000A04729460120A04771E70024264B1C707B
:108E200021462046254DA84721460120A847D6E6E1
:108E30000124214B1C7021460020204DA8472146CB
:108E40002046A847CBE61E4B1B78BBB11D4B98476D
:108E500000287FF4C9AE0022194B1A701A4B9847AC
:108E600000283FF4C1AE0024134B1C70214620465D
:108E7000124DA84721460120A847B5E6114B984757
:108E800000283FF4B1AE01220D4B1A700F4B1B7836
:108E9000002B3FF4A9AE1446074B1A701146002070
:108EA000064DA84721462046A8479DE6A16D4000F3
:108EB000794E4000A14F4000300C0020ED4E4000A4
:108EC000E000002035514000D98A4000330C0020DA
:108ED00010B582B000230193009380220549064813
:108EE000064CA047012802D00548064B984702B01F
:108EF00010BD00BFF8234100E58A4000EDD04000DE
:108F0000042441003DEF4000014B1878704700BF3A
:108F1000300C002018B9044A044B1A607047044A08
:108F2000024B1A60704700BFF8224100DC000020AD
:108F3000F821410008B5044B98476420034B98473B
:108F4000034B9847F7E700BF295F4000A5D34000D7
:108F50003D6F400070B584B050238DF80F30914BB9
:108F60009847914B1860914B9847914B9847012037
:108F7000904B984704A9002301F8023D05208E4B31
:108F8000984728B19DF80E3013B10020894B9847BF
:108F90008A4B98470DF10F010320874B9847884B68
:108FA00098479DF80F00874B9847874A874B1A6070
:108FB0000120874B9847044690B9834D854C0FCCD0
:108FC00028606960AA60EB60834B9847834B9847A1
:108FD0000222834B1A63834B98470546002416E010
:108FE0007A4B19680120744B984705E0774B1B6852
:108FF00000221A550134E4B20F2CF7D9E4E705201A
:10900000794B9847774B984705460134E4B20DB940
:10901000132CF4D9754B98472946754B9847754BD7
:109020009847754DA847002301221146734CA0476D
:109030000120734B9847A847002301220221A04733
:10904000704B9847644CA0476F4B98476F4B1B6819
:10905000ADF808301B0C8DF80A3002A90220564BDF
:109060009847A04702A96A4B984700252C466EE016
:109070001146002341F8043B6648674B984738B9CE
:10908000664B5968013159606248654B984768E002
:1090900001216048624B984763E01146002341F884
:1090A000043B60485C4B984738B95F4B59680131C5
:1090B00059605C485A4B984760E001215948584B29
:1090C00098475BE0134600221A605A6801325A60E2
:1090D00001A95648504B984750B9554B5968019BC8
:1090E000994201D8002513E04E484D4B9847F9E7C7
:1090F0004F4B59684B484A4B9847F3E74D4A136822
:1091000001331360052B41D90025494B1D601560C3
:10911000494BA3FB0423DB0803EB83035A0094426F
:1091200036D0464B9847002840F09E80444BA3FB26
:1091300004235B09642202FB1343002B00F0978099
:109140000A20294B98470134632C00D900240135AB
:10915000B5F57A7FDCD3314A1368013313603B2BBA
:1091600086D8384B98470028C8D00022314B1A6067
:109170002D4A1368013313603B2B8ED82C4A136899
:10918000013313603B2B9DD80025C1E70025BFE7C5
:109190002D4B984700285DD147232C4A13702C4A49
:1091A0001370BEE73DD64000580C0020C573400048
:1091B000716E4000754C4000A16D4000814C400034
:1091C000BD4A4000C94B4000101E0020F01D002089
:1091D000D56D4000A424410015E1400099554000A0
:1091E000000E0E40895F4000A5D340000DE1400015
:1091F0002D574000CD694000CD8A40007DD9400008
:10920000F969400031504000315440002C244100A5
:10921000F55440000110FFFFAD7140004C0C0020E0
:10922000CD7140000210FFFF3C0C00200310FFFF37
:10923000440C0020380C0020CDCCCCCCC1504000D8
:109240001F85EB51098F4000D98A4000E1000020C2
:10925000E20000200020074EB047074B18700120A5
:10926000B047064B18705CE7054B984768E7054B1D
:10927000984765E75D4F4000E1000020E2000020D4
:10928000CD5040003150400008B52A4B98472A4B3A
:10929000186009E000210846284CA0470021012061
:1092A000A0470022264B1A704FF0FF310120254BBA
:1092B0009847234B1B78013B062BF2D801A252F8AA
:1092C00023F000BFE19240009592400003934000DC
:1092D00013934000F1924000239340002F934000ED
:1092E00001210020154CA04701210846A047D8E7DE
:1092F000154D29880020154CA04729880120A0473A
:10930000CFE700210846124CA04700210120A047CA
:10931000C7E7012100200E4CA04701210846A047C5
:10932000BFE70C4B98470C490C4B9847B9E70C4BDF
:109330009847B6E73DD64000540C00203D4F400012
:10934000EF1D002055D840000A1E0020794E400035
:10935000ED4E400015E14000EC1D0020F5544000AA
:10936000416D400010B582B00023019303220092AA
:10937000802212491248134CA047012802D01248FB
:10938000124B984700230193009380221049114803
:109390000C4CA047012802D00F480C4B98470023E3
:1093A0000193009380220D490D48064CA0470128E7
:1093B00002D00C48054B984702B010BD3024410044
:1093C00089924000EDD04000342441003DEF400040
:1093D00050244100558F40005C244100842441000A
:1093E000358F40008824410000B583B00B4B1870C6
:1093F00002A9002341F8043D094B1868094B98471E
:10940000019B3BB14FF08052074B1A60BFF34F8F67
:10941000BFF36F8F03B05DF804FB00BFEF1D0020AA
:10942000540C002011DB400004ED00E00023044A4E
:109430001370044A13700120034B1870704700BF6B
:10944000640C0020600C00205C0C002070470020A1
:10945000704700000D4B5B881A0A032A01D00020D8
:10946000704713F0FF0F0ED1084BDB88402B01D063
:1094700000207047054B064A9A60064A1A6140224E
:109480009A81012070470020704700BF441E0020D1
:10949000680C0020C99440000122014B1A707047EB
:1094A0005C0C002010B5034B034A04490448054CEA
:1094B000A04710BD55944000B4010020600C00206E
:1094C000640C0020E995400008B5044B9B89402BB3
:1094D00000D008BD0248034B9847FAE7441E00201D
:1094E000680C00203D864000224B1B780BB91846C3
:1094F00070472DE9F04184B00746EFF31083B3FACB
:1095000083F35B09039372B6BFF35F8F00211A4B9D
:109510001970DDF80C80194D40222846184B9847E9
:109520003C4640372E4620686168A268E3680FC653
:1095300010343546BC42F5D1124B009340230F4AFC
:1095400000218120104CA04780F00100094B1870C9
:10955000B8F1000F05D00122074B1A70BFF35F8FDF
:1095600062B6044B1B7883F00103184604B0BDE8D3
:10957000F08100BF5C0C00202A020020A80C002013
:109580008DF7400099944000C5B7400010B50446DF
:10959000134B9847837A212B01D0002010BD00F196
:1095A0000902104B5B881B0A212B04D0C27B93421B
:1095B0000BD0002010BD0B4B9A60427AD9888A42AA
:1095C00028BF0A469A81012010BD064B9C60028A82
:1095D000D9888A4228BF0A469A81012010BD00BF5F
:1095E000C19B4000441E0020F8B5264C247865B28B
:1095F000002D07DB002D40DB04F06004202C22D07E
:109600000020F8BD14F0600603D11E4F7F78062FAE
:109610000BD0202EEED11B4A5278022A09D0032A01
:109620000CD0012AE6D19847F8BD1046164B984752
:10963000F8BD144B986001209881F8BD114B9960DA
:1096400001209881F8BD0F4A52780A2A07D00B2AC8
:109650000BD0092A01D00020F8BD9847F8BD094B6E
:109660005B881B0A03700120F8BD064BDB8833B909
:10967000044B5B880B700120F8BD0020F8BD002072
:10968000F8BD00BF441E00208D954000014B1868B6
:10969000704700BFF01D0020024B1B681B685888F4
:1096A00018447047F40C002038B504460D46094BA9
:1096B0009847024620782044904207D24378042BF2
:1096C00006D0AB4205D003781844F5E7002038BD3A
:1096D000002038BD9996400038B5144B1B780BB369
:1096E000134B1B681B681A7982421DD90D4604462C
:1096F000104A1360104B984703E01A7813440D4A40
:1097000013600C4B1B6898420AD95A78042AF4D18A
:109710009A789442F1D1DA78AA42EED1012038BD8C
:10972000002038BD002038BD002038BDF00C0020DE
:10973000F40C0020F80C002099964000084BDB88C0
:1097400063B9074B5B88012B01D000207047054AA5
:10975000138823F002031380012070470020704714
:10976000441E0020E80C002000207047044BDB88DA
:1097700023B9044A024B1A61012070470020704748
:10978000441E0020B19A400038B5134B1B7803B338
:10979000124B1C79124B1B681B681B799C4201D32E
:1097A000002317E0002120460E4B9847034688B15E
:1097B0000B4B1B685B6853F82450EB6898470146D5
:1097C0002046084B9847034620B1AB6898470346AC
:1097D00000E00023184638BDF00C0020441E002095
:1097E000F40C0020D996400038B5104B1B78D3B14B
:1097F00000240F4B1B681A681279944211D25B68DF
:1098000053F82450EB68984701462046094B984787
:10981000034648B1AB689847034628B90134E4B21F
:10982000E7E7002300E00023184638BDF00C0020D5
:10983000F40C0020D996400070B504460021114B6D
:109840009847054608B9284670BD0F4B1B685B68F2
:1098500053F82460F368984701462046094B98471F
:1098600005460028EFD0094B1C6805212046084B0F
:109870009847044618B18078064B9847F5E7736817
:109880009847E0E7D9964000F40C0020F80C00203F
:10989000A996400045B5400008B5064BDB88022B71
:1098A00001D0002008BD02210348044B9847012045
:1098B00008BD00BF441E0020E80C002029B4400071
:1098C00010B5184B9B78032B2AD8DFE803F005026C
:1098D000100B0720144C0CE004211448144B98473B
:1098E000002006E0134B98470446102001E01520A5
:1098F000114C08B1002308E0012010BDE15C0F4AC3
:1099000002EB430251800133DBB28342F6D3411CA8
:109910004900C9B209480170054B9847012010BDA4
:10992000002010BD441E00200C0200200802002070
:1099300029B440008D96400014020020DC01002074
:1099400008B5234B5B88DAB21B0A013B0E2B38D8D3
:10995000DFE803F00817313737373737373737370E
:1099600037372A001B4B186801781B4B9847184B58
:10997000DA889B899A4228D2154B9A81012318468E
:1099800008BD144B1B685B7C9A4201D30023F6E7A9
:10999000104B5B6853F8320041880F4B98470C4BD3
:1099A0009B6802225A70E2E70A4B986858B14188D6
:1099B000094B9847DBE7094B984703460028D6D167
:1099C000DDE70023DBE70023D9E70123D7E700BF6A
:1099D000441E0020E400002029B44000C19840004B
:1099E00008B5064BDB88012B01D0002008BD012102
:1099F0000348044B9847012008BD00BF441E0020C7
:109A0000F00C002029B4400038B5154BDB88012B41
:109A100002D00024204638BD124B1B78F3B1104B06
:109A20001D79114B1B681B681B799D4201D30024D3
:109A3000F0E7002128460D4B984704460028E9D05E
:109A4000094B1B685B6853F82530DB689847084B67
:109A5000187001211846074B9847DBE70024D9E727
:109A6000441E0020F00C0020F40C0020D996400089
:109A7000EC0C002029B4400008B5094BDB88022B10
:109A800001D0002008BD064B1879064B9847064BBD
:109A9000188002211846054B9847012008BD00BFD9
:109AA000441E002095B54000EA0C002029B4400077
:109AB00008B5034B588800F07F00024B984708BD5B
:109AC000441E0020D1B3400038B505460F4B9847DF
:109AD0000346C0B10E4B1C68052120460D4B98472C
:109AE000044640B18288C17880780B4B9847034682
:109AF0000028F1D107E0094B1B685B6853F825305B
:109B00001B6898470346184638BD00BFD9964000E9
:109B1000F80C0020A996400035B44000F40C002059
:109B200038B50C4BDB8893B90B4B1B780BB9002372
:109B30000EE0084B1C799D782046084B9847034659
:109B400030B129462046064B9847034600E00023E3
:109B5000184638BD441E0020F00C00203998400003
:109B6000C99A400008B5074BDB884BB9054B5B88A9
:109B70000BB1002008BD034B1879034B984708BD73
:109B8000002008BD441E0020D1B64000094BDB88F0
:109B90006BB9084B5B880BB10020704710B5054CC2
:109BA0002079054B98472079044B984710BD002039
:109BB000704700BF441E002041B94000D9B54000A5
:109BC000014B1868704700BFF80C002008B5014B26
:109BD000984708BD71B2400010B50B4B1B7863B1BC
:109BE000002404E02046094B98470134E4B2084BB6
:109BF0001B681B681B799C42F4D30022024B1A702D
:109C00000122044B1A8010BDF00C0020399840004E
:109C1000F40C0020E80C002008B5024B9847024BDA
:109C2000984708BD59B34000D99B40001C4BDB88C6
:109C300013B100231846704710B51A4B984750B31C
:109C4000174B9A78184B1B685B7C9A4201DD002306
:109C500022E0164B9847124B9B78154A1370EBB1D4
:109C6000114A526803F10053013B02EBC303114A4E
:109C7000136000240F4B1B681B681B799C4208D2A1
:109C8000002120460C4B9847034628B10134E4B22A
:109C9000F0E7012300E00023184610BD0123FBE795
:109CA000441E00200DB44000E4000020D99B400079
:109CB000F00C0020F40C0020C99A400008B5344B89
:109CC0001B7813F0800F0ED113F01F0343D1304ADD
:109CD0005278013A082A3ED8DFE802F0343D373D99
:109CE000313D3D3D3A002A4AD288002A4ED013F039
:109CF0001F0306D1264A5278062A0BD0082A0CD018
:109D00002AB1012B0CD0022B11D0002008BD214B11
:109D1000984708BD204B984708BD204B984708BD81
:109D20001B4A52780A2AEED11D4B984708BD184BA2
:109D30005B780BB1002008BD1A4B984708BD1A4B41
:109D4000984708BD194B984708BD194B984708BD5F
:109D5000184B984708BD012B03D0022B08D00020D8
:109D600008BD0B4A52780B2AF7D1134B984708BD10
:109D7000074B5B78012B03D0032B04D0002008BDD8
:109D80000E4B984708BD0E4B984708BD002008BDF4
:109D9000441E00209998400041994000E1994000FC
:109DA000099A4000799A40006D9740003D97400025
:109DB000699740002D9C4000219B4000659B40001E
:109DC0008D9B40000B4B1B7813B110B5002402E0B3
:109DD00070470134E4B2084B1B681A681279944248
:109DE00007D25B6853F824301B69002BF1D09847E9
:109DF000EFE710BDF00C0020F40C002008B5184B64
:109E000000229A811A615A611B7813F0800F11D1D8
:109E100013F0600F14D0124B1B7803F01F03012BBB
:109E200014D00F4B1B7803F01F03022B14D0002318
:109E3000184608BD0A4AD288002AE9D10023F7E76C
:109E4000084B984703460028E5D0F1E7064B9847B2
:109E500003460028E5D0EBE7044B98470346E7E7C5
:109E6000441E0020BD9C400089974000E9974000B7
:109E7000F8B504460E46114B984705462046104B50
:109E80009847054001D0002403E0F8BD0134062CBA
:109E900011D88DB123010B4AD058B042F6D102EB54
:109EA000041359680D42F1D01F46DB6898477B6860
:109EB00025EA0305EAE7F8BDF8BD00BFB7BC4000DE
:109EC000BBBC4000FC0C0020F8B5164C2768062FE0
:109ED00026D8002401E00134E4B2A446A7420AD304
:109EE000114E250106EB050E75598D42F3D1DEF8B2
:109EF00004509542EFD1CEF80010CEF80420CEF8F1
:109F000008300699CEF80C100137BC4505D0114633
:109F10001A46064B98470020F8BD02490F60F6E745
:109F20000120F8BD6C0D0020FC0C00207DBC400021
:109F30002DE9F04182B004460F4690460A4B9847FF
:109F400005462046094B984706462046084B984749
:109F5000CDF800803B46024631462846054CA047D6
:109F600002B0BDE8F08100BFBFBC4000CDBC4000E6
:109F7000D3BC4000C99E400008B50B210148024BEC
:109F8000984708BD000E0E40719E400008B50C2198
:109F90000148024B984708BD00100E40719E4000DA
:109FA000F8B506460C461546224B984707464FF033
:109FB000FF313046204B98473046204B9847002CC5
:109FC0000CDB630904F01F0101228A4020331C4985
:109FD00041F82320BFF34F8FBFF36F8F002C08DBB6
:109FE000630904F01F0101228A406033144941F8DB
:109FF0002320002C17DB2D01EDB204F1604303F5A3
:10A00000614383F80053002C08DB620904F01F044D
:10A01000012303FA04F40A4B43F822403946304640
:10A02000084B9847F8BD04F00F022D01EDB2064B26
:10A030009D54E8E7BBBC4000B3BC4000B7BC400047
:10A0400000E100E0AFBC400014ED00E082B0024649
:10A0500010B9244B1B783BB912B1224B1B780BB3C0
:10A06000204B1A7002B070471F4B1B7803B9FEE7F4
:10A07000EFF31083B3FA83F35B09009372B6BFF377
:10A080005F8F0021194B1970009817490B78013B1D
:10A090000B700028E0D00121144B1970BFF35F8FC3
:10A0A00062B6D9E7104B1B78FF2B19D0EFF3108362
:10A0B000B3FA83F35B09019372B6BFF35F8F00219C
:10A0C0000A4B1970019808490B7801330B7000286E
:10A0D000C6D00121054B1970BFF35F8F62B6BFE791
:10A0E000FEE700BF710D00205C1E00202A02002048
:10A0F00084B02A4B9A6842F480729A609A6822F07F
:10A100007F029A601A6B0192019A42F04F0201920B
:10A11000019A22F4074222F080020192019A42F44D
:10A1200000420192019A1A631C4B1B6B13F4004FFF
:10A13000FAD01A4A136B0293029B43F04F03029327
:10A14000029B43F400430293029B136300238DF8A8
:10A15000033006E000BF9DF803300133DBB28DF819
:10A1600003309DF80330DBB2132BF3D9EFF31083E8
:10A17000B3FA83F35B09039372B6BFF35F8F0022D8
:10A18000074B1A70039B0121044A116123B1044B50
:10A190001970BFF35F8F62B604B07047004004408F
:10A1A0002A020020034A0023136153619381024A6B
:10A1B00013707047441E0020760D002082B00522E7
:10A1C000104B1A70104A136B0193019B43F04F031D
:10A1D0000193019B43F020030193019B1363002330
:10A1E0008DF8033006E000BF9DF803300133DBB289
:10A1F0008DF803309DF80330DBB2132BF3D902B096
:10A20000704700BF760D00200040044082B003225A
:10A21000104B1A70104A136B0193019B43F04F03CC
:10A220000193019B43F010030193019B13630023EF
:10A230008DF8033006E000BF9DF803300133DBB238
:10A240008DF803309DF80330DBB2132BF3D902B045
:10A25000704700BF760D0020004004400422014BEF
:10A260001A707047760D002008B5024B1B6903B1C8
:10A27000984708BD441E002030B589B06A4B1B7852
:10A28000032B29D0694B9C89694B1B88E41AA4B223
:10A29000002C43D1674A11880B449BB21380634A58
:10A2A000D288934203D0644B1B78002B2CD0634B95
:10A2B0009847634A136B0393039B43F04F03039345
:10A2C000039B23F001030393039B13635C4B1B6B02
:10A2D00013F0010FFAD115E0594A136B0293029B58
:10A2E00043F04F030293029B23F001030293029B6E
:10A2F0001363534B1B6B13F0010FFAD1514B98476B
:10A30000514B984709B030BD484B5B6933B1984712
:10A3100020B10022464B1A80444B9C893F2C37D9F0
:10A320000022454B1A704024404B9A68404B1B88D2
:10A330001A44EFF31083B3FA83F35B09079372B601
:10A34000BFF35F8F0021414B197007983C4B1B6B8B
:10A3500013F0020F3ED028B101223C4B1A70BFF31C
:10A360005F8F62B60422304B1A70354A136B049328
:10A37000049B43F04F030493049B23F001030493D5
:10A38000049B13632E4B1B6B13F0010FFAD1B9E73B
:10A390000122294B1A70C7E7157829490D65013349
:10A3A000DBB2013299B28C42F6D8214B1A881444A0
:10A3B0001C80234A136B0593059B43F04F030593C1
:10A3C000059B43F010030593059B136300238DF851
:10A3D000073008E00023E5E700BF9DF807300133B0
:10A3E000DBB28DF807309DF80730DBB2132BF3D9C1
:10A3F000134A136B0693069B43F04F030693069B89
:10A4000023F001030693069B13630D4B1B6B13F0A4
:10A41000010FFAD100283FF475AF01220B4B1A70DF
:10A42000BFF35F8F62B66DE7760D0020441E0020FB
:10A43000720D0020740D0020700D00205DA2400000
:10A440000040044069A24000A5A140002A0200206B
:10A4500010B586B0654B1B78012B1ED0022B04D0A3
:10A46000042B02D0624B984701E0624B9847624A46
:10A47000136B0093009B43F04F030093009B23F06A
:10A4800002030093009B13635B4B1B6B13F0020FE3
:10A49000FAD15A4B984706B010BD574B186BC0F312
:10A4A0000A40574B9B89574A14882218934201DA75
:10A4B000181B80B2524B9A682244002305E04E4993
:10A4C000096D11700133DBB2013299B28842F6D8BE
:10A4D0000444A4B24B4B1C8040281BD0484B9C81A9
:10A4E0005B6913B19847002832D0434A136B02933B
:10A4F000029B43F04F030293029B23F0020302935B
:10A50000029B13633C4B1B6B13F0020FFAD13E4BC3
:10A510009847C0E73A4BDA883C4B1B8823449A4261
:10A52000DCDD374B9B899C4227D0334A136B059364
:10A53000059B43F04F030593059B23F0020305930E
:10A54000059B13632C4B1B6B13F0020FFAD1A2E790
:10A55000274B9847284A136B0193019B43F04F0305
:10A560000193019B23F002030193019B1363224B90
:10A570001B6B13F0020FFAD18DE7214B5B6953B1CE
:10A580009847E8B121491F4A0B88108803440B8083
:10A5900000231380C9E7164B9847174A136B0393A0
:10A5A000039B43F04F030393039B23F002030393A6
:10A5B000039B1363104B1B6B13F0020FFAD16AE776
:10A5C0000B4B98470C4A136B0493049B43F04F03C7
:10A5D0000493049B23F002030493049B1363064B30
:10A5E0001B6B13F0020FFAD155E700BF760D002068
:10A5F000BDA1400069A2400000400440A5A1400068
:10A60000441E0020720D00200DA24000740D002099
:10A610000023042B14D810B40A499A00D418A000BF
:10A6200004460844407C214400F083026FF3C712C3
:10A630004A740133DBB2042BEED95DF8044B70474A
:10A64000704700BF780D002038B5437C13F0100F21
:10A6500016D00D46437C6FF30413437404687CB139
:10A6600002F10C03074951F8233013F4806F01D035
:10A6700042F080028168012D14BF00200120A04714
:10A6800038BD00BF0040044010B500240BE0234655
:10A690000134E4B203EB8303980022460121034B0B
:10A6A0001844034B9847042CF1D910BD780D0020B5
:10A6B00049A6400010B500F00F02531E03EB8303C0
:10A6C0009C00012102482044024B984710BD00BF66
:10A6D000780D002049A6400030B482B00246441EE6
:10A6E0003B4900F10C0551F8253051F8251013F0C5
:10A6F000020302D001F0400151B9002B39D004EB24
:10A7000084039900334B0B44597C6FF383015974D4
:10A7100004EB840399002F4B0B445B7C13F00C0F6C
:10A7200032D12B4900F10C0551F825300093009BE4
:10A7300043F04F030093009B23F002030093009B20
:10A7400041F8253002F10C03214951F8233013F070
:10A75000020FF7D1002838D0032836D004EB840448
:10A76000A2001C4B13445A7C012161F383025A74EA
:10A770002BE004EB84039900164B0B44597C012514
:10A7800065F383015974C3E711490C3051F8203047
:10A790000193019B43F04F030193019B23F040037E
:10A7A0000193019B41F8203002F10C03084951F854
:10A7B000233013F0400FF7D104EB8404A200054BC3
:10A7C00013445A7C6FF383025A7402B030BC704752
:10A7D00000400440780D0020F0B4461EB30033441E
:10A7E00099002A4A0A445368D1680B449468641A51
:10A7F000128AC2F30902944209D31446002706EBD9
:10A8000086029500214A2A442144D1601EE0012796
:10A81000F5E71D781E4A00F1140142F821505D78D9
:10A8200042F821509D7842F82150DD7842F82150BD
:10A830001D7942F821505D7942F821509D7942F806
:10A840002150DD7942F82150083C0833072CE0D82C
:10A8500007E01D7800F114020D4941F82250013C37
:10A860000133002CF5D1094BB10088198200104644
:10A870001A44527CC2F3810203440132597C62F3D0
:10A88000830159743846F0BC704700BF780D002032
:10A890000040044070B582B0441E04EB84039A006B
:10A8A000364B13445B7CC3F3810328B1032801D0EA
:10A8B000022202E0012200E001229A4254DDA200BD
:10A8C000224495002D4B2B44DA689B689A4205D3AD
:10A8D0002A4B2B445B7C13F0400F48D00E460546B4
:10A8E000274B9847FEB1274A0C3552F82530019383
:10A8F000019B43F04F030193019B43F0100301932D
:10A90000019B42F8253000238DF8033006E000BF9C
:10A910009DF803300133DBB28DF803309DF803302E
:10A92000DBB2132BF3D940B104EB84039A00134B31
:10A9300013445A7C6FF386125A74A2002244910089
:10A940000E4B0B44DA689B689A4212D30B4B0B44B4
:10A950005B7C13F0400F0ED1084B0B445A7C42F045
:10A9600080025A74002000E0012002B070BD002077
:10A97000FBE70120F9E70120F7E700BF780D002091
:10A98000D9A74000004004402DE9F843054684461D
:10A99000471EBB003B449A002A4C1444A268E3685B
:10A9A000A2EB030EB4F81080C8F3090862681A44D9
:10A9B0000C30254951F82060C6F30A4666B3B64507
:10A9C0000BD9B6464FF0000907EB870188001D49F7
:10A9D00001447344CB6000210AE04FF00109F3E722
:10A9E0000CF11403184850F8233013700131013270
:10A9F0008E45F5D82846154B9847B9F1000F01D17F
:10AA0000B04507D905F10C030F4A52F8233013F073
:10AA1000200F04D0BDE8F8834FF00009EAE70123D6
:10AA2000AB405361074ABB00D81981000846114466
:10AA3000C968024491602A4600212046044B984789
:10AA4000E8E700BF780D002000400440D9A6400090
:10AA500049A640002DE9F0418CB00124ADE120462B
:10AA6000B34B98470120FAE1BB003B449900B14A3F
:10AA70000A44537CC3F38101033161F383035374AC
:10AA8000537C13F0200F00F0848013F00C0F3BD0A8
:10AA9000A94A04F10C0152F821300193019B43F0C3
:10AAA0004F030193019B43F010030193019B42F874
:10AAB000213000238DF8013006E000BF9DF8013001
:10AAC0000133DBB28DF801309DF80130DBB2132B7E
:10AAD000F3D9994A06F10C0152F821300293029BF6
:10AAE00043F04F030293029B23F001030293029B66
:10AAF00042F8213006F10C038F4A52F8233013F04C
:10AB0000010FF7D10120AAE18B4A04F10C0152F8A0
:10AB100021300393039B43F04F030393039B23F0E4
:10AB200001030393039B42F8213006F10C03824A90
:10AB300052F8233013F0010FF7D1114606F10C0340
:10AB400052F823200492049A42F04F020492049A8D
:10AB500042F020020492049A41F8232000238DF849
:10AB6000023006E000BF9DF802300133DBB28DF801
:10AB700002309DF80230DBB2132BF3D907EB8707C5
:10AB8000BA006C4B13445A7C6FF345125A7401207F
:10AB900065E113F0800F42D1BB003B449A00654B46
:10ABA0001344DA689B689A424CD307EB87039A00F8
:10ABB000604B13445B7C13F04C0F43D1EFF31083D5
:10ABC000B3FA83F35B090B9372B6BFF35F8F002276
:10ABD0005A4B1A700B9B584A55612BB10122574BA7
:10ABE0001A70BFF35F8F62B6534A06F10C0152F838
:10ABF00021300593059B43F04F030593059B23F0FC
:10AC000001030593059B42F8213006F10C034A4AE3
:10AC100052F8233013F0010FF7D101201FE1BB00E0
:10AC20003B449A00434B1344597C6FF3C71159744A
:10AC3000DA689A60404B5D61224600214046404BF5
:10AC40009847A9E7002C4AD0032C48D007EB87038C
:10AC50009A00384B13445B7C13F00C0F3FD0364AFC
:10AC600006F10C0152F821300693069B43F04F0386
:10AC70000693069B43F010030693069B42F821308F
:10AC800000238DF8033006E000BF9DF80330013348
:10AC9000DBB28DF803309DF80330DBB2132BF3D910
:10ACA000254A06F10C0152F821300793079B43F027
:10ACB0004F030793079B23F001030793079B42F879
:10ACC000213006F10C031C4A52F8233013F0010F17
:10ACD000F7D1002120461B4B98470120BFE0002CF4
:10ACE0004AD0032C48D001212046164B984758B330
:10ACF000114A06F10C0152F821300893089B43F0E9
:10AD00004F030893089B23F001030893089B42F824
:10AD1000213006F10C03084A52F8233013F0010FDA
:10AD2000F7D100212046074B9847012097E000BF4C
:10AD300089A94000780D0020004004402A0200202C
:10AD400049A6400095A840004749BB00D819820099
:10AD50000A4492F811E06FF3C71E82F811E0D2683E
:10AD60001F44BB0019448A60404B5D6122460021AC
:10AD700040463F4B9847BBE7012120463D4B984753
:10AD80003A4A06F10C0152F821300993099B43F02D
:10AD90004F030993099B23F001030993099B42F890
:10ADA000213006F10C03314A52F8233013F0010F21
:10ADB000F7D1012053E00134E4B2052C4ED82B4BDF
:10ADC0009B6926460125A5402B42F4D0671E07EB60
:10ADD00087029300244A02EB030804F10C03234A80
:10ADE00052F8233013F0420F7FF439AE04F10C0314
:10ADF0001E4A52F8233013F0010F7FF435AE04F1F0
:10AE00000C031A4A52F8233013F0080FD3D004F180
:10AE10000C0152F821300A930A9B43F04F030A9326
:10AE20000A9B23F008030A930A9B42F8213006F19B
:10AE30000C030E4A52F8233013F0080FF7D106F135
:10AE40000C0352F8233003F4E063B3F5807F09D09C
:10AE500006F10C0352F82330012000E000200CB072
:10AE6000BDE8F0810120FAE7780D002000400440A1
:10AE700049A6400095A8400000B587B0534B1B7809
:10AE8000E3B9534B1B6BC3F30A43082B3BD0504A27
:10AE9000136B0193019B43F04F030193019B23F03C
:10AEA00004030193019B1363494B1B6B13F0040FC5
:10AEB000FAD1484B984707B05DF804FB464B9847DA
:10AEC000464B9847DDE7424A116D454A9954013394
:10AED000DBB2072BF7D9434B9847B0B93C4A136B09
:10AEE0000293029B43F04F030293029B23F004035F
:10AEF0000293029B1363364B1B6B13F0040FFAD1C2
:10AF0000344B9847D7E70023E3E7354B93F90030FC
:10AF1000002B1EDB2E4A136B0593059B43F04F035A
:10AF20000593059B23F004030593059B1363284BAE
:10AF30001B6B13F0040FFAD1294BDB88002B42D096
:10AF40000023294A1380294A138001221F4B1A70BB
:10AF5000B1E71F4A136B0393039B43F04F03039323
:10AF6000039B43F080030393039B136300238DF83B
:10AF7000033006E000BF9DF803300133DBB28DF8EB
:10AF800003309DF80330DBB2132BF3D9104A136B57
:10AF90000493049B43F04F030493049B23F00403A6
:10AFA0000493049B13630A4B1B6B13F0040FFAD139
:10AFB00000230D4A13800D4A13800222034B1A709E
:10AFC0000B4B984777E70B4B984774E7760D0020BB
:10AFD00000400440BDA1400069A24000A5A140007E
:10AFE000441E0020FD9D4000740D0020720D0020C5
:10AFF00079A240000DA24000204BDB6913F0010F45
:10B0000037D000B583B01D4B1B6B13F0040F24D158
:10B010001A4B1B6B13F0010F23D1184B1B6B13F052
:10B02000020F22D1154B1B6B13F0080F23D0134ACC
:10B03000136B0193019B43F04F030193019B23F09A
:10B0400008030193019B13630C4B1B6B13F0080F58
:10B05000FAD1012003B05DF804FB094B98470120A9
:10B06000F8E7084B98470120F4E7074B9847012081
:10B07000F0E7002070470020ECE700BF00400440EC
:10B0800079AE400079A2400051A4400010B54C4B6D
:10B09000984720B94B4BDB6913F4807F10D03020E8
:10B0A000494B9847474B9B6913F4006F04D0454BBD
:10B0B000DB6913F4006F0AD1444B984770B110BD9F
:10B0C00072B6BFF35F8F0022414B1A7010BD4FF470
:10B0D00000623C4B1A623F4B984710BD3E4B98476D
:10B0E0000028ECD1374B9B6913F4005F04D0354B3B
:10B0F000DB6913F4005F3DD1324B9B6913F4007F91
:10B1000004D0304BDB6913F4007F33D12D4B9B69A6
:10B1100013F4806F04D02B4BDB6913F4806F29D1BB
:10B12000284B9B6913F4807F04D0264BDB6913F412
:10B13000807F2FD1234BDB6913F4805FBFD0214C7C
:10B140004FF480532362254B9847254B98476368FB
:10B1500023F001036360636823F002036360214B03
:10B160009847214B98474FF4807323614FF4006355
:10B170002361A4E7134C4FF4185323626361012049
:10B180001A4B98474FF48073236223614FF4006396
:10B19000236110BD0B4B4FF480721A625A614FF459
:10B1A00000521A614FF400721A614FF480621A6102
:10B1B00030200F4B984700200C4B984710BD00BF24
:10B1C0002DC2400000400440F5C04000F9AF4000EF
:10B1D0002A020020C59D400055AA400089A64000D3
:10B1E000D99B4000F1A04000A5A140004DA0400027
:10B1F00049C1400010B582B0EFF31083B3FA83F376
:10B200005B09019372B6BFF35F8F0022144B1A7073
:10B21000019C0120134B98473020134B9847134B48
:10B220005A6F22F480725A675A6F42F400725A675A
:10B230004FF480721A614FF400521A614FF4007299
:10B240001A614FF480621A614FF400621A612CB1E6
:10B250000122034B1A70BFF35F8F62B602B010BDBC
:10B260002A0200204DA04000F5C0400000400440EC
:10B2700030B583B0EFF31083B3FA83F35B09009327
:10B2800072B6BFF35F8F0024204B1C70009D204BD3
:10B29000984730201F4B98471F4B98471F4B502211
:10B2A00083F830234FF480325A601D4B98474FF497
:10B2B00080201C4B98471C4B1C701C4B1B78FF2B91
:10B2C00022D0EFF31083B3FA83F35B09019372B6D4
:10B2D000BFF35F8F00220D4B1A700199134A137848
:10B2E0000133137029B10122084B1A70BFF35F8F2D
:10B2F00062B60F4B98472DB10122044B1A70BFF371
:10B300005F8F62B603B030BDFEE700BF2A020020A7
:10B31000F9BA4000F5C04000E1BC400000E100E0A7
:10B3200011A6400019C24000710D00205C1E0020D3
:10B33000F5B1400008B5064B5A6F42F480725A6767
:10B340005A6F22F400725A670020024B984708BDDA
:10B35000004004404DA0400010B582B0EFF31083D0
:10B36000B3FA83F35B09009372B6BFF35F8F0022D9
:10B37000144B1A70009C144B9847144B1B7803B95C
:10B38000FEE7EFF31083B3FA83F35B09019372B620
:10B39000BFF35F8F00220B4B1A7001990B4A137891
:10B3A000013B137029B10122064B1A70BFF35F8F66
:10B3B00062B62CB10122034B1A70BFF35F8F62B6E5
:10B3C00002B010BD2A02002035B340005C1E0020F0
:10B3D0000D4B5A6822F001025A609A6822F480727A
:10B3E0009A60024670B1986820F07F0002F07F02F8
:10B3F000104398609A6842F480729A605A6842F0EA
:10B4000001025A60704700BF00400440054B5B6872
:10B4100013F0010F04D0034B986800F07F007047D1
:10B420000020704700400440014B986099817047AC
:10B43000441E0020F0B583B045B200F00F0005288F
:10B4400073D801F00306044600F10C033B4F57F894
:10B45000233013F4004F6BD1012E53D0031FDBB206
:10B46000012B54D94023934266DB461E06EB860728
:10B47000334B03EB870303F11007B3F810E062F3DB
:10B48000090EA3F810E05B7C03F07F036FF3451314
:10B490007B70002D3EDB294EB36A012282401343AC
:10B4A000B362264B9B6A1A42FBD0244B9E6A26EA63
:10B4B00002029A6200F10C0253F822300193019BC0
:10B4C00043F04F030193019B23F4074323F08003D0
:10B4D0000193002D23DB0A0202F4407242F4004281
:10B4E000019B1343019301990C30144B43F8201036
:10B4F00004F10C03114951F8233032EA0303F7D168
:10B50000012013E0B0B10328A8D100200EE04FF4D1
:10B510000073A8E77B786FF383037B70BBE70A02B5
:10B5200002F4407242F40442DAE7002003B0F0BDB6
:10B530000020FBE70020F9E70020F7E70040044087
:10B54000780D002000F00F03052B1ED810B582B037
:10B5500019460E4C0C3354F823200192019A42F004
:10B560004F020192019A22F400420192019A44F89A
:10B57000232001F10C03054A52F8233013F4004F45
:10B58000F7D1034B984702B010BD7047004004400C
:10B59000B5A6400000F00F00431E052815D803EBA8
:10B5A00083039A000A4B13445B7C13F0200F08D1ED
:10B5B0000C30084B53F8203013F0280F03D0012033
:10B5C000704701207047002070470020704700BF7F
:10B5D000780D00200040044010B485B044B200F063
:10B5E0000F00052865D8421EEFF31083B3FA83F3EA
:10B5F0005B09039372B6BFF35F8F0021314B197063
:10B600000399002C14DB304A00F10C0452F824306A
:10B610000293029B43F04F030293029B43F02003EB
:10B620000293029B42F8243000238DF807302EE06D
:10B6300000F10C03244C54F8233013F0100F09D1FF
:10B6400002EB82039C00214B23445B7CC3F3810308
:10B65000012BD8DD02EB820294001C4B23445A7C60
:10B6600042F020025A74012303FA00F0164B1861CD
:10B6700021B30120134B1870BFF35F8F62B619E03E
:10B6800000BF9DF807300133DBB28DF807309DF81D
:10B690000730DBB2132BF3D9012303FA00F00A4B76
:10B6A000186169B10120074B1870BFF35F8F62B654
:10B6B00000E0002005B05DF8044B70470120F9E779
:10B6C0000120F7E72A02002000400440780D002006
:10B6D00000F00F0005286CD830B583B00246441E38
:10B6E00004EB84039900354B0B44597C6FF34511EF
:10B6F000597400F10C03324951F8233013F0200F34
:10B7000059D000F10C0551F825300093009B43F00F
:10B710004F030093009B23F020030093009B41F80C
:10B72000253002F10C03264951F8233013F0200F85
:10B73000F7D10D468B6A012181400B43AB62204B50
:10B740009B6A1942FBD01E4B9D6A25EA0101996252
:10B750000C3053F820100191019941F04F010191F3
:10B76000019921F008010191019943F8201002F19B
:10B770000C03134951F8233013F0080FF7D104EBF1
:10B7800084039A000D4B13445B7C13F0100F01D11E
:10B79000012011E00949A200101983000B44587CD4
:10B7A0006FF3041058741444A300CB589847012039
:10B7B00002E000207047012003B030BD780D00206A
:10B7C00000400440F0B583B000F00F04052C00F2F7
:10B7D000A28047B2651E04F10C00554E56F82000B9
:10B7E00010F4004F00F09A8005EB8500514E06EBF7
:10B7F0008000407C10F0200F40F0928004F10C009B
:10B800004B4E56F8200010F0200F40F08B80EFF3E5
:10B810001080B0FA80F04009009072B6BFF35F8FDD
:10B82000002645480670DDF800E005EB8500414E36
:10B8300006EB8000407C10F0100F0AD0BEF1000F24
:10B8400072D001223C4B1A70BFF35F8F62B60020AA
:10B8500062E005EB8500374E06EB8000467C46F043
:10B8600010064674BEF1000F05D00126324806705E
:10B87000BFF35F8F62B6DFF8BCE005EB85008000A8
:10B880000EEB00067260B3600022F260089A4EF878
:10B89000002011B95BBB012000E00120254AA9006E
:10B8A0004B1902EB83035B7C60F386130D4402EBC0
:10B8B00085026FF3C7135374EFF31083B3FA83F366
:10B8C0005B09019372B6BFF35F8F00221A4B1A70A7
:10B8D000019D0123A340164A1361002F09DB2DB3FC
:10B8E0000120154B1870BFF35F8F62B614E0002083
:10B8F000D4E704F10C0352F8233013F0110FEED10A
:10B90000012120460D4B98470028E8D00021204611
:10B910000A4B9847E3E7002003B0F0BD0020FBE7A7
:10B920000020F9E70020F7E70020F5E70120F3E722
:10B9300000400440780D00202A02002095A8400015
:10B9400070B586B000F00F04052C00F2C98042B239
:10B95000EFF31083B3FA83F35B09059372B6BFF379
:10B960005F8F00215F4B1970059B26460125A5407E
:10B970005D494D612BB101215A4B1970BFF35F8FA7
:10B9800062B6002A80F2948004F10C03564A52F801
:10B99000233013F0100F64D0002C49D0032C47D073
:10B9A00004F10C0152F821300193019B43F04F0345
:10B9B0000193019B23F010030193019B42F8213076
:10B9C00006F10C03484A52F8233013F0100FF7D158
:10B9D00006F10C03444A52F8233013F0100FF7D14C
:10B9E00004F10C0152F821300293029B43F04F0303
:10B9F0000293029B43F010030293029B42F8213012
:10BA000000238DF8033006E000BF9DF803300133BA
:10BA1000DBB28DF803309DF80330DBB2132BF3D982
:10BA200006F10C03304A52F8233013F0100FF7D010
:10BA30002D4A04F10C0152F821300393039B43F08B
:10BA40004F030393039B23F010030393039B42F8DC
:10BA5000213006F10C03244A52F8233013F0100F62
:10BA6000F7D1214A04F10C0152F821300493049BD0
:10BA700043F04F030493049B23F001030493049BBE
:10BA800042F8213006F10C03174A52F8233013F024
:10BA9000010FF7D1621E02EB82029100134B0B449F
:10BAA0005A7C6FF383025A740AE02046104B984781
:10BAB00006F10C030C4A52F8233013F0420FF4D174
:10BAC000094A936A2B439362074B9B6A1D42FBD042
:10BAD000054A936A23EA050595622046054B984777
:10BAE00006B070BD2A02002000400440780D0020FE
:10BAF000D9A64000B5A64000064BD3F8142122F485
:10BB00004062C3F81421D3F8202142F00102C3F8A7
:10BB10002021704700020E400B4619B109680160F0
:10BB20005B6843601AB113680361536843617047EF
:10BB300021F0FE01C905C90D0162704710B51E4B09
:10BB400053F820402268536A13F0805F11D002231B
:10BB5000C2F8203123684FF0FF32DA6100232375E9
:10BB6000236913F0010F26D0636823B3204698475A
:10BB700010BD13F0006F13D00223C2F820312368E8
:10BB80004FF00062DA61236913F0020F03D0A3685B
:10BB90000BB12046984723680122C3F8202110BD2D
:10BBA00013F0007F07D0236913F0040F03D0E3687C
:10BBB0000BB12046984710BDDC0D002008B50020D1
:10BBC000014B984708BD00BF3DBB400008B50120B0
:10BBD000014B984708BD00BF3DBB400070B505460E
:10BBE0000E461446016001230B60214B99422BD075
:10BBF0000D20204B9847204B1D6023781B0203F437
:10BC0000FE43736063782BBB0022A3780BB142F034
:10BC10000402E3780BB142F0080223790BB142F041
:10BC2000100263791B0203F47063A179090389B2DE
:10BC30000B431343B3652389C3F30E03628943EABD
:10BC40000243F36500230CE012200A4B98470A4B8D
:10BC50005D60D2E70222D8E705EB83020021516044
:10BC60000133022BF8D900202861287570BD00BF70
:10BC700000000340F5C04000DC0D002012F0100F62
:10BC800012D0C0F8B01012F0200F07D0C0F8D410B6
:10BC900012F0400F05D0C0F8C0107047C0F8D010A7
:10BCA000F6E7C0F8C4107047C0F8B41070470164DC
:10BCB000704741647047C06C7047806C70474009A2
:10BCC00000F5001000F207704002704740090B3089
:10BCD000704700F01F00012303FA00F070470000D6
:10BCE00008B500200A4B98470A4B98470028FBD01C
:10BCF000094B9847094A0A4BDA620A4B98470028D1
:10BD0000FBD00020084B9847084B984708BD00BF60
:10BD100071C0400095C04000D9C04000013FB80547
:10BD200000040E40E5C04000F9C140000DC24000D3
:10BD300010B5A2B01848194B98470020184B9847E7
:10BD4000184B98470028FBD0174B9847174A184BB9
:10BD50009A62184B98470028FBD00020164B984752
:10BD6000164B984716480D4B9847164B1A68164BBA
:10BD70001344164A934201D922B010BD20230093E8
:10BD800002AB0F220E211248124CA047BDF84810FA
:10BD90001148124B9847EFE7000E270765C5400092
:10BDA00071C0400095C04000BDC04000013FB70BCE
:10BDB00000040E40C9C040001DC0400071C44000D6
:10BDC0000000DC052C020020C0D3BDF980C3C901EE
:10BDD000000A0E401100002010140E403DC2400029
:10BDE00070B50D461446064658B14FF0FF360AE0CE
:10BDF000064B1868064B1B682946984701350136E3
:10BE0000013C002CF4DC304670BD00BF6C1E0020ED
:10BE1000641E002070B5013802280FD81446002592
:10BE20008CB10A4B18684E1C094B1B68097898475F
:10BE3000002806DB0135013C3146F1E74FF0FF35C4
:10BE400001E04FF0FF35284670BD00BF6C1E00209A
:10BE5000681E0020A1F10E03012B02D84FF0FF3025
:10BE6000704710B582B0EFF31083B3FA83F35B0928
:10BE7000019372B6BFF35F8F00240B4B1C70019CC3
:10BE8000120222F07F4222F0FF02C9B2114341F0B8
:10BE9000B441064B98472CB10122034B1A70BFF3F3
:10BEA0005F8F62B602B010BD2A0200207900002028
:10BEB0004C4B1B78FF2B31D000B583B0EFF31083D0
:10BEC000B3FA83F35B09019372B6BFF35F8F00226D
:10BED000454B1A700199434A13780133137029B105
:10BEE0000122414B1A70BFF35F8F62B63F4A904206
:10BEF00015D03F4A904220D03E4A90422BD03E4A35
:10BF0000904236D03D4A904241D03D4A90424CD07A
:10BF10003C4A904257D003B05DF804FBFEE7162080
:10BF2000394B98470720394B984700210720384B59
:10BF300098470720374B9847EDE71520324B984735
:10BF40000720324B984700210720314B98470720A4
:10BF5000304B9847DFE714202B4B984707202B4B9B
:10BF60009847002107202A4B98470720294B9847DC
:10BF7000D1E71320244B98470620244B98470021F3
:10BF80000620234B98470620224B9847C3E70E20F4
:10BF90001D4B984706201D4B9847002106201C4B3F
:10BFA000984706201B4B9847B5E70920164B984742
:10BFB0000620164B984700210620154B984706206F
:10BFC000144B9847A7E708200F4B984706200F4BC4
:10BFD0009847002106200E4B984706200D4B9847A6
:10BFE00099E700BF5C1E00202A02002000000440E8
:10BFF0000080004000C0014000800140004002403D
:10C000000000024000C00040F5C04000E5C1400013
:10C010009DC14000D1C1400001607047134A136BBD
:10C0200023F07003184310634FF400630F4A926EBD
:10C0300012F0080F02D1A3B1013BF7E70B4A136BD3
:10C0400023F0030343F0020313634FF40063074A32
:10C05000926E12F0080F02D12BB1013BF7E70020DE
:10C060007047012070470120704700BF00040E4058
:10C07000012803D0054A064B1A607047044A9368AA
:10C0800043F0254343F480139360F3E7080000A5D1
:10C0900010140E40074B5B6913F0800F06D0064B5F
:10C0A0009B6E13F0800F03D1002070470020704773
:10C0B0000120704710140E4000040E400022014B76
:10C0C0009A62704700040E40024B986E00F0020026
:10C0D000704700BF00040E400022014BDA62704737
:10C0E00000040E40024B986E00F00400704700BF41
:10C0F00000040E4032281ED81F280CD8114B9A6914
:10C1000001238340934318D0012303FA00F00D4B21
:10C1100018610020704720380A4BD3F8082101230A
:10C12000834093430BD0012303FA00F0054BC3F87F
:10C130000001002070470120704700207047002058
:10C14000704700BF00040E40322822D81F280ED8A6
:10C15000114B9A6901238340934301D0002070471B
:10C16000012303FA00F00C4B58610020704720387F
:10C17000094BD3F8082101238340934301D00020C9
:10C180007047012303FA00F0034BC3F804010020B9
:10C1900070470120704700BF00040E4041F00401C9
:10C1A00000F11002094B43F822104FF40062074BD4
:10C1B000996E4FF480738340194202D11AB1013A4B
:10C1C000F5E7002070470120704700BF00040E40D3
:10C1D0004FF4807303FA00F0014B1860704700BF02
:10C1E00000040E404FF4807303FA00F0014B5860D6
:10C1F000704700BF00040E40000200F4706040F081
:10C200000100014B9863704700040E408022014BEF
:10C210001A60704700040E40C0F31200024B1A6F00
:10C2200010431867704700BF00040E40024B187897
:10C2300080F00100704700BFE40D0020C36923F4C3
:10C24000F053490201F4F051194341F0B44141F473
:10C250008071C161704730B4B2EB011F17D3102455
:10C2600001FB04F14B0803EBC202B2FBF1F2D3086D
:10C270005D1E4FF6FE718D4210D8082C09D01204B5
:10C2800002F4E0221A430262002030BC7047082406
:10C29000E6E7416841F400214160F0E70120F4E75E
:10C2A00040230360704788230360704710230360B6
:10C2B00070472423036070474FF480730360704716
:10C2C0004FF4002303607047436913F0020F04D05A
:10C2D000C1F30801C1610020704701207047436924
:10C2E00013F0020FFBD0C1F30801C16100207047B9
:10C2F000436913F0010F05D08369C3F308030B6092
:10C300000020704701207047014BC0F8E4307047AF
:10C310000041535510B50446094B9847002363600C
:10C320006362A3622046074B98472046064B984716
:10C330002046064B98472046054B984710BD00BF46
:10C3400009C34000A7C24000B3C24000B9C24000C8
:10C35000C1C2400070B505460C461646104B9847C2
:10C360000022104B1A60B4B13246216828460E4BA9
:10C370009847024688B96368A1680B4321690B435B
:10C38000E1680B430749086803430B6069680B4386
:10C390006B60104670BD0122FBE70122F9E700BF88
:10C3A00015C34000E80D002057C24000FEE7000022
:10C3B00000B583B0234B244A9A4209D0214B224A2C
:10C3C00003E0116819600433043220498B42F8D32A
:10C3D0001F4B02E000221A6004331E4A9342F9D335
:10C3E0001D4A22F07F011D4B9960EFF31083B3FAD1
:10C3F00083F35B09019372B6BFF35F8F0021184B83
:10C400001970019817490B6843F470030B60BFF370
:10C410004F8FBFF36F8F28B10121114B1970BFF3FC
:10C420005F8F62B602F16042B2F5203F04D20B4A40
:10C43000936843F0005393600B4B98470B4B98471E
:10C44000FEE700BF100000202C274100E80B002071
:10C45000E80B0020C01E00200040400000ED00E07E
:10C460002A02002088ED00E0EDEE4000CDDE400025
:10C47000344B1B6B03F00303012B20D083B1022B41
:10C4800039D0304B1B6B03F07003702B51D02D4B08
:10C490001A6BC2F302122C490B68D3400B60704731
:10C4A0002A4B5B6913F0800F04D04FF40042264BF7
:10C4B0001A60E6E74FF4FA42234B1A60E1E7214B9A
:10C4C0001B6A13F0807F03D0214A1F4B1A60D8E704
:10C4D000204A1D4B1A601B4B1B6A03F07003102B84
:10C4E00005D0202BCDD11C4A174B1A60C9E71B4A37
:10C4F000154B1A60C5E7154B5B6913F0800F13D01D
:10C500004FF40042104B1A600E4B1B6B03F00303F9
:10C51000022BB6D10B4B9A6AC2F30C420A490B6844
:10C5200002FB03330B60ACE74FF4FA42064B1A6090
:10C53000EAE7054A13680A49A1FB03135B08136085
:10C54000704700BF00040E402C02002010140E4063
:10C55000001BB70000127A0000366E010024F400C0
:10C56000ABAAAAAA144B98420FD9144B984211D9DE
:10C57000134B984212D9134B984213D9124B98423D
:10C5800014D9124A124B1A6070474FF08062104B58
:10C590001A6070470F4A0E4B1A6070470E4A0C4BD8
:10C5A0001A6070470D4A0A4B1A6070474FF0042218
:10C5B000074B1A60704700BFFF2C3101FF59620220
:10C5C000FF869303FFB3C404FFE0F50500050004F4
:10C5D000000A0E40000100040002000400030004F1
:10C5E0000A4B1B6853B1094B1B681A180849914242
:10C5F00008DB1046054A106018467047054A034B91
:10C600001A60F0E74FF0FF30704700BFEC0D0020DC
:10C61000FC7F0220C04E00204FF0FF3070474FF4E7
:10C6200000534B6000207047012070470020704786
:10C6300000F1080343604FF0FF328260C360036182
:10C6400000230360704700230361704743684B6019
:10C650009A688A609A68516099600861036801333A
:10C660000360704730B40D68B5F1FF3F02D000F1B0
:10C67000080202E0026904E01A4653681C68A542F9
:10C68000FAD253684B6099608A6051600861036810
:10C690000133036030BC7047036942688168916070
:10C6A0008268416851605A68904206D00022026157
:10C6B0001A68013A1A601868704782685A60F5E78C
:10C6C00082B0002301934FF0500383F31188BFF32E
:10C6D0006F8FBFF34F8F019B002BFCD002B07047D0
:10C6E00008480068006880F308884FF0000080F375
:10C6F000148862B661B6BFF34F8FBFF36F8F00DF50
:10C7000000BF000008ED00E0DFF80C00016841F414
:10C71000700101607047000088ED00E04FF0807309
:10C7200040F8043C21F0010140F8081C054B40F89A
:10C730000C3C40F8202C6FF0020340F8243C4438B5
:10C74000704700BFC1C640000000000000000000AC
:10C75000074B19680868B0E8F04F80F30988BFF309
:10C760006F8F4FF0000080F311887047AFF30080A7
:10C77000F00D00204FF0500383F31188BFF36F8F4B
:10C78000BFF34F8F024A136801331360704700BF35
:10C7900030020020034A1368013B13600BB983F396
:10C7A00011887047300200200000000000000000E7
:10C7B000EFF30980BFF36F8F154B1A681EF0100F4F
:10C7C00008BF20ED108A20E9F04F10602DE9090024
:10C7D0004FF0500080F31188BFF34F8FBFF36F8F7E
:10C7E00000F03CFE4FF0000080F3118809BC19688E
:10C7F0000868B0E8F04F1EF0100F08BFB0EC108AC8
:10C8000080F30988BFF36F8F704700BFAFF30080DC
:10C81000F00D002008B54FF0500383F31188BFF3EB
:10C820006F8FBFF34F8F054B984718B14FF0805271
:10C83000034B1A60002383F3118808BDD9D140004F
:10C8400004ED00E0054B00221A6005490A60054925
:10C85000054A116007221A60704700BF10E000E02F
:10C8600018E000E0FF7F010014E000E010B50E4B7F
:10C870001A6842F470021A601A6842F070421A6034
:10C880000A4B984700240A4B1C600A4B98470A4AF7
:10C89000136843F040431360084B9847084B984790
:10C8A000084B9847204610BD20ED00E045C84000E9
:10C8B0003002002009C7400034EF00E0E1C640002C
:10C8C0005DD44000C1C6400010B50446044B9847F3
:10C8D0002046044B98470446034B9847204610BD1A
:10C8E000C9D1400065EF4000CDD2400048B110B53D
:10C8F0000446044B98472046034B9847034B984700
:10C9000010BD7047C9D1400075EF4000CDD2400046
:10C91000436A23B1036B1868C0F10500704700201B
:10C920007047000010B50446064B9847A26BE36BB6
:10C930009A4204D00024044B9847204610BD01249D
:10C94000F9E700BF75C7400095C7400010B5044621
:10C95000054B9847A36B23B10024044B984720460E
:10C9600010BD0124F9E700BF75C7400095C740001E
:10C9700070B504461646856B026C5AB903681BB144
:10C9800000200135A56370BD4068174B9847002310
:10C990006360F6E76EB98068144B9847226CA36811
:10C9A0001344A3606268934219D32368A3600020F4
:10C9B000E7E7C0680D4B9847226C5242E368134486
:10C9C000E36021688B4202D263681A44E260022E5F
:10C9D00001D00020D5E725B1013D0020D1E700209E
:10C9E000CFE70020CDE700BF11D7400091F5400010
:10C9F00038B505461A4B984795F8454064B201E0B2
:10CA0000013C64B2002C0ADD6B6A43B105F12400DD
:10CA1000144B98470028F3D0134B9847F0E7FF23B7
:10CA200085F84530114B98470D4B984795F8444091
:10CA300064B201E0013C64B2002C0ADD2B6943B111
:10CA400005F11000074B98470028F3D0064B984794
:10CA5000F0E7FF2385F84430044B984738BD00BF0A
:10CA600075C7400035D5400031D6400095C740001D
:10CA700038B504460D46144B98472168E26B236C89
:10CA800003FB021060600020A063A160013A02FB7A
:10CA90000313E360FF2384F8443084F8453055B92C
:10CAA00023691BB9094B9847012038BD04F11000D8
:10CAB000074B9847F6E704F11000064DA84704F12C
:10CAC0002400A847EEE700BF75C7400095C74000A7
:10CAD00035D5400031C6400038B51D46049C0B4694
:10CAE00049B12260E063236401212046034B98474B
:10CAF00084F84C5038BD2460F4E700BF71CA400090
:10CB0000F0B583B0054617460E4689B100FB01F02B
:10CB10005030084B9847044638B100903B4600F12E
:10CB2000500231462846044DA847204603B0F0BDC8
:10CB30000020EDE7C9C84000D9CA4000F0B585B073
:10CB400004460F4601921E46002526E0324639462D
:10CB50002046354B9847636A23B9344B98470120E8
:10CB600005B0F0BD04F12400314B9847F5E72F4B99
:10CB700098470020F4E702A82E4B9847012519E0BA
:10CB8000002384F8443021E0002384F8453023E07A
:10CB90002046294B9847294B9847294B9847A26B29
:10CBA000E36B9A42D2D3022ED0D0019B002BDED071
:10CBB000002DE0D01D4B9847224B9847204B9847BB
:10CBC00094F844305BB2B3F1FF3FD9D094F84530CC
:10CBD0005BB2B3F1FF3FD7D0144B984701A902A82D
:10CBE000194B9847C8B92046184B98470028CFD012
:10CBF000019904F11000164B984720460E4B9847B8
:10CC00000E4B98470028C8D14FF08052114B1A6044
:10CC1000BFF34F8FBFF36F8FBFE72046064B984798
:10CC2000064B984700209BE771C9400095C740001C
:10CC300035D54000B5D54000F1C94000CDD2400007
:10CC400075C74000C9D14000CDD5400025C940007E
:10CC500011D5400004ED00E048B110B5002141605D
:10CC60000160C1600B460A46014CA04710BD7047E9
:10CC70003DCB400010B5024600210120034B9847F0
:10CC80000446034B9847204610BD00BF01CB40002F
:10CC900059CC400070B584B0044601910026354659
:10CCA0003EE0013BA36323683BB123694BB9444B8E
:10CCB00098470126304604B070BD424B98476060EB
:10CCC000F3E704F11000404B9847F0E73C4B9847DE
:10CCD0000026EFE702A83D4B984701252AE00023F4
:10CCE00084F8443032E0002384F8453034E0384B97
:10CCF00098476068374B98470646314B98473BE06A
:10CD00002046354B9847354B984709E02046324B33
:10CD10009847324B98472046314B9847002840D1DE
:10CD20002B4B9847A36B002BBBD1019B002BCDD085
:10CD3000002DCFD0224B98472A4B9847244B984739
:10CD400094F844305BB2B3F1FF3FC8D094F845305B
:10CD50005BB2B3F1FF3FC6D0194B984701A902A8B7
:10CD6000214B98470028D1D120461D4B98470028D9
:10CD7000C6D02368002BBAD0019904F124001B4BC4
:10CD800098472046144B9847144B98470028C7D122
:10CD90004FF08052164B1A60BFF34F8FBFF36F8F67
:10CDA000BEE7002E86D00A4B98472046114B984785
:10CDB00001466068104B9847014B9847002679E779
:10CDC00095C7400039D8400035D54000B5D5400062
:10CDD00075C7400049D64000F1C94000CDD240009F
:10CDE0004DC94000C9D14000CDD5400011D540000B
:10CDF00004ED00E011C9400099D74000F0B5036888
:10CE00004BB343685B68436000F10807BB4204D042
:10CE10004368D3F80CE0002609E05B684360F7E75D
:10CE20005B68436008E02E46B6B9AE4514D043684F
:10CE30005B6843609F42F3D04368DD6800230F2B9B
:10CE4000F2D8EA1892F83420CC5CA242ECD1002A45
:10CE5000E9D00133F3E700263046F0BD0A4B1B68EA
:10CE60001B684BB901234BB9074B1B68DB68DB68B8
:10CE70005A68064B1A6070470023F4E74FF0FF3200
:10CE8000024B1A60704700BFF40D0020A00E002076
:10CE90002DE9F84F81460D4617469A460A9EDDF861
:10CEA0002C800C9C9200A521206B1D4B9847236B76
:10CEB00007F18042013A03EB820727F007070023BE
:10CEC0000F2B07D8E95CE21882F83410EA5C0AB14B
:10CED0000133F5E7002384F84330042E00D90426FB
:10CEE000E662E66400252565201DDFF83CB0D847E2
:10CEF00004F11800D8472461C6F10506A6616462F2
:10CF0000656584F85850524649463846054B98475F
:10CF10002060B8F1000F01D0C8F80040BDE8F88FDC
:10CF20008DF740001DC7400047C6400070B5002483
:10CF300007E004EB840293000B4818440B4B98471E
:10CF40000134042CF5D90A4E3046084CA047094D4F
:10CF50002846A0470848A0470848A047084B1E603D
:10CF6000084B1D6070BD00BFFC0D002031C64000A5
:10CF7000740E0020880E0020A80E0020C00E002095
:10CF8000F40D0020F80D002010B504461C4B984706
:10CF90001C4A1368013313601B4B1B68002B26D0FF
:10CFA0001A4B1B683BB9184B1B68DA6AE36A9A4252
:10CFB00001D8154B1C60164A136801331360636473
:10CFC000E36A01229A401349086802430A6003EBAE
:10CFD00083039A00211D10481044104B9847104BB2
:10CFE00098470A4B1B680BB1074B1B6810BD064BDB
:10CFF0001C601368012BDED10A4B9847DBE700BFAA
:10D0000075C74000600E0020F00D0020BC0E00200F
:10D010006C0E0020700E0020FC0D00204DC640005C
:10D0200095C740002DCF400070B504460E461D4BFD
:10D030001D681D4B186804301C4B984750B91A4B9B
:10D040001B68DA6A012303FA02F219490B6823EA22
:10D0500002030B60B4F1FF3F13D02C44124B1B684A
:10D060005C60A54216D8134B18680F4B1968043141
:10D07000114B9847114B1B689C4201D20F4B1C600F
:10D0800070BD002EE9D0084B196804310C480D4BD7
:10D09000984770BD0C4B1868034B19680431064B58
:10D0A000984770BDD40E0020F00D002099C64000B6
:10D0B000700E0020F40D002065C64000A00E002078
:10D0C000C00E00204DC64000F80D002008B54FF0FE
:10D0D0008052044B1A60BFF34F8FBFF36F8F024B28
:10D0E0009847F4E704ED00E0C9DE40002DE9F04385
:10D0F00085B006460F46154698469000144B984753
:10D1000000B381465C20124B98470446B0B1C0F88A
:10D110003090CCB10023039302940D9B01930C9BA0
:10D12000009343462A46394630460A4DA8472046D2
:10D13000094B9847012005B0BDE8F0834846074BEE
:10D140009847E6E70024E4E74FF0FF30F3E700BF3D
:10D15000C9C8400091CE400089CF4000EDC84000D2
:10D1600010B582B0104B01930023009346220F4963
:10D170000F48104CA047012801D002B010BD4FF05D
:10D18000500383F31188BFF36F8FBFF34F8F4FF0BE
:10D19000FF32094B1A600122084B1A600022084B2B
:10D1A0001A60084B9847E8E79C0E0020B82441001D
:10D1B000CDD04000EDD04000A00E0020BC0E0020DD
:10D1C000D40E00206DC84000024A1368013313607A
:10D1D000704700BF680E002070B52F4B1B68002BF6
:10D1E00052D12E4B1E6801361E604EB12C4B1B686F
:10D1F0009E422FD22B4B1B68002B42D0002070BDCB
:10D20000294A1168294B186810601960284A136868
:10D2100001331360274B9847E8E7012320E04FF0E4
:10D22000FF321F4B1A60E5E71D4A1360E2E704F185
:10D230001800214B9847E36A01229A401F49086869
:10D2400002430A6003EB83039A0029461C481044FA
:10D250001C4B9847144B1B681B68002BDDD0002328
:10D26000002BDCD1104B1B68DB68DC6863689E42D6
:10D27000DAD3251D2846104B9847A36A002BD6D138
:10D28000D9E7114B9847B9E7064A13680133136091
:10D290000D4B9847B2E700BF680E0020D40E002067
:10D2A000A00E0020640E0020F40D0020F80D0020D8
:10D2B000A40E00205DCE400099C64000700E0020F4
:10D2C000FC0D00204DC64000CBDE400070B5274B62
:10D2D0009847274B1A68013A1A601B68002B32D115
:10D2E000244B1B68002B2ED00024234B1B6813B348
:10D2F000214BDB68DC6804F11800204EB047251D87
:10D300002846B047E36A01229A401D490868024353
:10D310000A6003EB83039A0029461A4810441A4B0B
:10D320009847E26A194B1B68DB6A9A42DDD30122F7
:10D33000174B1A60D9E70CB1164B9847164B1C686F
:10D340003CB9134B1B68154B9847002070BD013C3E
:10D3500007D0134B98470028F9D001220C4B1A60D4
:10D36000F5E700220C4B1A60EBE700BF75C74000E1
:10D37000680E0020600E0020A80E002099C6400014
:10D38000700E0020FC0D00204DC64000F00D002066
:10D39000D80E00205DCE4000640E002095C74000EE
:10D3A000D9D1400010B550B9002038B94FF08052A3
:10D3B000084B1A60BFF34F8FBFF36F8F10BD044649
:10D3C000054B984700212046044B9847044B98474B
:10D3D000EBE700BF04ED00E0C9D1400029D04000D8
:10D3E000CDD2400070B50646154B98470524013C48
:10D3F00004EB84029300314612481844124B9847BC
:10D40000054608B9002CF2D12DB15DB18DB10F4B9D
:10D410009847284670BD0E4B186831460A4B98470E
:10D420000546F2E70B4B18683146074B984705460F
:10D43000ECE731460848044B98470546E7E700BF4C
:10D44000C9D14000FC0D0020FDCD4000CDD24000F0
:10D45000F40D0020F80D0020C00E0020264B1B68A4
:10D46000002B2FD110B50022244B1A60244B1B68CF
:10D470001B6B1A68B2F1A53F28D0214B18681968B8
:10D480003431204B9847204B1B68B3FA83F3DBB24F
:10D49000C3F11F031D489A00D418A10001444C6831
:10D4A00064684C601A4491000831084484421AD0E0
:10D4B00003EB83039A00154B13445B68DA68104B47
:10D4C0001A6010BD01220D4B1A6070475A68B2F104
:10D4D000A53FD2D19A68B2F1A53FCED1DB68B3F1B6
:10D4E000A53FCAD1CFE7606803EB83029100074AEA
:10D4F0000A445060DCE700BF680E0020D80E002010
:10D50000F00D0020B1DE4000700E0020FC0D002068
:10D5100010B50C46044B19681831044B984701218B
:10D520002046034B984710BDF00D002065C6400013
:10D5300029D0400038B5C368DC6804F118052846D6
:10D54000144B9847144B1B68E3B9251D2846114B13
:10D550009847E36A01229A401049086802430A602A
:10D5600003EB83039A0029460D4810440D4B98475E
:10D57000E26A0D4B1B68DB6A9A4208D901200B4B0B
:10D58000186038BD29460A48064B9847F0E7002046
:10D5900038BD00BF99C64000680E0020700E002004
:10D5A000FC0D00204DC64000F00D0020D80E0020DC
:10D5B000A80E0020034B1B680360034B1B684360ED
:10D5C000704700BFA40E0020D40E0020F8B504461A
:10D5D0000D46124B9847124B19686268881A2B68DF
:10D5E000B3F1FF3F16D027680E4E3668B74201D020
:10D5F000914211D2984206D300232B6001240A4B9A
:10D6000098472046F8BD1B1A2B602046074B9847C9
:10D610000024F4E70024F2E70124F0E775C7400096
:10D62000D40E0020A40E002095C74000B5D54000C0
:10D630000122014B1A607047D80E0020014B186878
:10D64000704700BFF00D0020002854D038B50446C4
:10D65000C26A2A490968C96A8A4242D28169002994
:10D6600005DB26490968C96AC1F105018161606964
:10D6700002EB82029100224A0A44904207D0002223
:10D680003AB91E4A1268D26AE262012038BD01220C
:10D69000F6E7251D28461B4B984768B9E36A03EB5C
:10D6A00083018A0016498A5832B901229A401649E4
:10D6B0000B6823EA02030B60104B1B68DB6AE36212
:10D6C000012404FA03F21049086802430A6003EBDC
:10D6D00083039A0029460A4810440C4B9847204679
:10D6E00038BDC26C054B1B68DB6A9A4201D201202F
:10D6F00038BD002038BD0020704700BFF00D00206D
:10D70000FC0D002099C64000700E00204DC6400060
:10D71000002834D038B50446026D013A0265C06A6B
:10D72000E16C88422DD00AB1002038BD251D284665
:10D73000154B984768B9E36A03EB83018A001349E4
:10D740008A5832B901229A4011490B6823EA020330
:10D750000B60E36CE362C3F10502A261012404FAE9
:10D7600003F20B49086802430A6003EB83039A0043
:10D77000294606481044074B9847204638BD0020EC
:10D780007047002038BD00BF99C64000FC0D002046
:10D79000700E00204DC64000002843D038B5044626
:10D7A000C26C8A4200D20A46E16A8A4202D0206DE7
:10D7B000012800D038BDE262A069002802DBC2F176
:10D7C0000502A261636901EB81018800164A0244E7
:10D7D000934225D00022002AECD0251D2846134B69
:10D7E000984768B9E36A03EB83018A000E498A58B7
:10D7F00032B901229A400E490B6823EA02030B60FA
:10D80000E36A01229A400A49086802430A6003EB6E
:10D8100083039A00294604481044064B9847C9E7F9
:10D820000122D8E7704700BFFC0D002099C64000D8
:10D83000700E00204DC64000054B1B6823B1044B01
:10D840001A68136D01331365014B1868704700BFE8
:10D85000F00D002038B505460C461A4B98471A4B78
:10D860001B685B6D2BB9184B1B68012283F858208D
:10D87000ACB9164B9847134B9847134B1B685C6D1C
:10D8800024B1CDB9104B1B68621E5A650E4B1B6844
:10D89000002283F858200D4B9847204638BD11468A
:10D8A00020460B4B98474FF080520A4B1A60BFF34B
:10D8B0004F8FBFF36F8FDCE7034B1B6800225A6565
:10D8C000E4E700BF75C74000F00D002095C7400099
:10D8D00029D0400004ED00E0F8B507460D46144697
:10D8E0001E46214B9847214B1B6893F85830DBB2FA
:10D8F000022B0AD01D4B1A68506D20EA07005065B4
:10D900001B68012283F85820CEB9194B9847164B53
:10D9100098471CB1154B1B685B6D2360134B1B684C
:10D9200093F85830DBB2022B16D000240F4B1B6843
:10D93000002283F858200E4B98472046F8BD114628
:10D9400030460C4B98474FF080520B4B1A60BFF398
:10D950004F8FBFF36F8FD8E7044B1A68536D23EADC
:10D96000050555650124E1E775C74000F00D00206D
:10D9700095C7400029D0400004ED00E0F8B504460A
:10D980000F4615461E46214B98470EB1636D336016
:10D9900094F85830DBB2022284F858206A1E032A19
:10D9A0001AD8DFE802F0020C1114626D17436765A4
:10D9B0000125012B14D0164B98472846F8BD626DFF
:10D9C000013262650125F4E767650125F1E7022B65
:10D9D00004D067650125ECE70125EAE70025E8E7C3
:10D9E000261D30460B4B9847E36A01229A400A49AC
:10D9F000086802430A6003EB83039A003146074834
:10DA00001044074B9847074B1B68D4E775C7400085
:10DA100095C7400099C64000700E0020FC0D002004
:10DA20004DC64000F00D0020F8B5EFF311854FF022
:10DA3000500484F31188BFF36F8FBFF34F8F0BB186
:10DA4000446D1C6090F85830DBB2022480F85840D6
:10DA5000013A032A1AD8DFE802F0020C1114426DD1
:10DA6000114341650126012B14D085F311883046FE
:10DA7000F8BD426D013242650126F4E74165012699
:10DA8000F1E7022B04D041650126ECE70126EAE725
:10DA90000026E8E70446164B1B68F3B9071D384615
:10DAA000144B9847E36A01229A40134908680243DD
:10DAB0000A6003EB83039A00394610481044104B68
:10DAC0009847E26A0F4B1B68DB6A9A42CDD9069BE6
:10DAD0004BB10123069A1360C7E700F118010A4809
:10DAE000074B9847EDE70122084B1A60BDE700BFDE
:10DAF000680E002099C64000700E0020FC0D00202A
:10DB00004DC64000F00D0020A80E0020D80E0020C9
:10DB1000F8B5EFF311854FF0500383F31188BFF38D
:10DB20006F8FBFF34F8F90F85830DBB2022280F82E
:10DB30005820426D01324265012B02D085F31188D5
:10DB4000F8BD0E460446154B1B68E3B9071D384661
:10DB5000134B9847E36A01229A401249086802432E
:10DB60000A6003EB83039A0039460F4810440F4BB9
:10DB70009847E26A0E4B1B68DB6A9A42DED946B1CF
:10DB800001233360DAE700F118010A48074B984790
:10DB9000EFE70122084B1A60D0E700BF680E0020B3
:10DBA00099C64000700E0020FC0D00204DC64000BC
:10DBB000F00D0020A80E0020D80E0020064BDB6BD5
:10DBC000C3F30023054A1370054BDB6BC3F34033EB
:10DBD000044A1370704700BF00100E40DC0E002096
:10DBE000000E0E40DD0E002008B5054BDB6B13F474
:10DBF000004F02D1034B984708BD034B984708BD1F
:10DC0000000E0E40814C4000A54C400030B583B062
:10DC100004460D46002301932E4B984213D02E4B01
:10DC20009C421AD02D4B9C4221D02D4B9C4228D097
:10DC30002C4B9C422FD02C4B9C4236D02B4B9C42E1
:10DC40003DD003B030BD01A92046294B984700289C
:10DC5000F9D19DF804302B70E1E701A92046244B4F
:10DC600098470028F9D19DF804302B70DAE701A914
:10DC700020461F4B98470028F9D19DF804302B709F
:10DC8000D3E701A920461A4B98470028F9D19DF8FF
:10DC900004302B70CCE701A92046154B984700288B
:10DCA000F9D19DF804302B70C5E701A92046104B2F
:10DCB00098470028F9D19DF804302B70BEE701A9E0
:10DCC00020460B4B98470028F9D19DF804302B7063
:10DCD000B7E700BF00C2004000020240004202401D
:10DCE0000082014000C20140008200400002044066
:10DCF000F1C2400038B504460D46274B984213D078
:10DD0000264B984218D0264B98421DD0254B98425E
:10DD100022D0254B984227D0244B98422CD0244B1C
:10DD2000984231D0002038BD29462046214B9847E3
:10DD30000028F9D1012038BD294620461D4B9847BF
:10DD40000028F9D1012038BD29462046194B9847B3
:10DD50000028F9D1012038BD29462046154B9847A7
:10DD60000028F9D1012038BD29462046114B98479B
:10DD70000028F9D1012038BD294620460D4B98478F
:10DD80000028F9D1012038BD29462046094B984783
:10DD90000028F9D1012038BD00C200400002024035
:10DDA000004202400082014000C201400082004067
:10DDB00000020440C9C2400000B583B002A900239C
:10DDC00041F8043D084B1868084B9847019B3BB14C
:10DDD0004FF08052064B1A60BFF34F8FBFF36F8F27
:10DDE00003B05DF804FB00BFE00E002011DB400033
:10DDF00004ED00E070B58AB01D4B0FCB0AAC04E90E
:10DE00000F001C4D1C4B1D601C4A1D4B1A601D4A07
:10DE10001D4B1A60069B0093079B0193089B02937E
:10DE2000099B039300240494184E3046184B9847DE
:10DE300001213046174B9847174A69462846174B29
:10DE400098472846164B98472846164B9847164E33
:10DE5000336821469868154DA847336821465868AD
:10DE6000A847336821469868A8470AB070BD00BF2C
:10DE7000C0244100008201406C1E0020F5DC4000FF
:10DE8000681E00200DDC4000641E00200080014060
:10DE9000B1BE400019C040000000DC0555C3400081
:10DEA000A1C24000ADC240003802002065F8400029
:10DEB00008B50A4601460248024B9847FEE700BFF4
:10DEC000782541003DEF4000704770472DE9F04351
:10DED00083B04A4B98474A4A936843F0254343F43A
:10DEE00080139360474B9847474B9847474B984759
:10DEF000474B9847474B9847474B98470446474BF3
:10DF00009847F02201462046454B9847454B984795
:10DF10004548464B03602223037123234371444D3C
:10DF20002946444CA0474448444B03602B230371CB
:10DF30002A2343712946A047414B9847414B9847B4
:10DF40004148424B98474248424CA04742494348C7
:10DF5000A04743494348A047434A44494448A0474F
:10DF600000230193042200924FF4807241494248F9
:10DF7000424CA047012802D04148364B98473D48C3
:10DF8000404B9847404B1860404B9847404B984750
:10DF9000404B9847404B9847404A00210F20404E45
:10DFA000B047404C03220B2120463F4DA847DFF8E5
:10DFB00008914A4600212820B0473C4F03220C21FB
:10DFC0003846A8472820DFF8F480C0470146384685
:10DFD000374FB8474A4600210D20B04703220B2196
:10DFE0002046A8470D20C04701462046B847314B80
:10DFF0009847002003B0BDE8F08300BF69454000AA
:10E0000010140E4031BD4000856A4000C95F4000D9
:10E01000F5DD40009D664000556840005D684000A9
:10E020001567400031674000841E00200000024058
:10E03000A086010061634000701E002000C0014006
:10E04000CD9B4000915E4000B9DD40005D45400041
:10E05000D02441003DEF4000E8244100FC24410071
:10E06000F0214100082541001C25410028254100E0
:10E07000342541004C25410069684000EDD0400046
:10E0800054254100E5D34000E00E0020DD8540002E
:10E0900065934000D18E4000297F4000E9DB4000BD
:10E0A000319F4000000E0E40A19F400000100E4026
:10E0B000AFBC400061D14000BDDB4000D3BC40009C
:10E0C00010B50A4B984772B609480A4CA0470A484F
:10E0D000A0470A4B98470A4B98470A4B98470A4A69
:10E0E000136823F00103136010BD00BF516A4000A4
:10E0F000841E0020F9634000701E00206D4B40001C
:10E10000199C4000B167400010E000E000487047F3
:10E11000841E002000487047701E002008B5014B87
:10E12000984708BD6568400008B5014B984708BD91
:10E13000676840000120704708B50248024B9847C5
:10E1400008BD00BF841E00209964400008B5024845
:10E15000024B984708BD00BF701E00209964400024
:10E16000014B1878704700BFDD0E0020014B187876
:10E17000704700BFDC0E002000BEFEE770B58AB01D
:10E18000044600F06FF8324B93F900506B1C0646C2
:10E1900009D02146204600F08DFE20B900212046FE
:10E1A00000F07EFE10B130460AB070BD294B0890D9
:10E1B0002046019300F006FBCDE90401CDE9020100
:10E1C0002046CDB9244B4FF060420021CDE9062313
:10E1D00000F03EFE002833D002230093684600F092
:10E1E00085F9A8B1089BC3B9DDE9060100F03EFB43
:10E1F000064630460AB070BD184B00220021CDE91A
:10E20000062300F025FE68B102239D420093E5D16C
:10E2100000F066FE22230360E4E700F061FE089B45
:10E220000360E1E70123022D00930BD100F058FEBB
:10E23000212303600A4800F05BF9CDE90601D1E72C
:10E2400001230093684600F051F90028F2D1EDE770
:10E250003402002090254100FFFFEFC70000F0FFCF
:10E26000B42441002DE9F84F30F000432DD00028B0
:10E27000014604464ADBB0F1FF4F3BDAB0F5000F30
:10E280003CDB00268D4AC4F316052A4402F4000242
:10E29000E41582F07E507F3C34444FF07E51284399
:10E2A00004EBD25400F036FB05F10F03C3F3160361
:10E2B0000F2B064631DC002100F0CAFD002800F0DB
:10E2C00094804CB90020BDE8F88F00214FF04C40FD
:10E2D00000F0DEFCBDE8F88F204600F0D1FB784965
:10E2E000054600F021FC77490446284600F01CFC56
:10E2F0000146204600F010FBBDE8F88F4FF0984132
:10E3000000F012FC6FF018060446BBE700F002FBB9
:10E31000002100F0BDFCBDE8F88F4FF0804100F017
:10E32000FBFA0146304600F0B3FC8046204600F080
:10E33000A7FB41468146404600F0F6FB0146834676
:10E3400000F0F2FB6049DFF8A0A1074600F0ECFB0B
:10E350005E4900F0E1FA394600F0E6FB5C4900F066
:10E36000DBFA394600F0E0FB5A4900F0D5FA59468D
:10E3700000F0DAFB58498346384600F0D5FB574990
:10E3800000F0CAFA394600F0CFFB554900F0C4FA54
:10E39000394600F0C9FB0146584600F0BDFAC5F504
:10E3A0005713AA4403F5227343EA0A03002B0746D6
:10E3B00065DD4FF07C51304600F0B6FB314600F091
:10E3C000B3FB0546002C32D12946384600F0A4FAAA
:10E3D000414600F0A9FB0146284600F09BFA0146A1
:10E3E000304600F097FABDE8F88F3E49304600F01D
:10E3F0009BFB01464FF07C5000F08CFA31460546FD
:10E40000304600F091FB0146284600F08DFB0546A2
:10E41000002C2ED0204600F033FB2949074600F09F
:10E4200083FB28490446384600F07EFB14E024496B
:10E43000484600F079FB29460446384600F06CFA5D
:10E44000414600F071FB1F490746484600F06CFB4F
:10E450000146384600F060FA0146284600F05AFAB4
:10E46000314600F057FA0146204600F053FABDE865
:10E47000F88F0146304600F04DFABDE8F88F7CB1C8
:10E480000F49484600F050FB39460446304600F03C
:10E4900041FA414600F048FB0A4905464846C3E7B1
:10E4A0000146304600F036FA414600F03DFB014699
:10E4B000304600F02FFABDE8F88F00BF20FB4A007D
:10E4C0008071313FD1F717379788173E25333A3E91
:10E4D0002549923EABAA2A3F4FD01C3E298E633E6F
:10E4E000CDCCCC3EABAAAA3E305CCFFF002070471B
:10E4F00000200149704700BF0000F87F81F0004113
:10E5000002E000BF83F0004330B54FEA41044FEA18
:10E51000430594EA050F08BF90EA020F1FBF54EAB3
:10E52000000C55EA020C7FEA645C7FEA655C00F04F
:10E53000E2804FEA5454D4EB5555B8BF6D420CDD20
:10E540002C4480EA020281EA030382EA000083EAA3
:10E55000010180EA020281EA0303362D88BF30BD43
:10E5600011F0004F4FEA01314FF4801C4CEA113199
:10E5700002D0404261EB410113F0004F4FEA0333F8
:10E580004CEA133302D0524263EB430394EA050F83
:10E5900000F0A780A4F10104D5F1200E0DDB02FAF2
:10E5A0000EFC22FA05F2801841F1000103FA0EF286
:10E5B000801843FA05F359410EE0A5F120050EF14C
:10E5C000200E012A03FA0EFC28BF4CF0020C43FA7D
:10E5D00005F3C01851EBE37101F0004507D54FF08A
:10E5E000000EDCF1000C7EEB00006EEB0101B1F5DA
:10E5F000801F1BD3B1F5001F0CD349085FEA300020
:10E600004FEA3C0C04F101044FEA445212F5800F2A
:10E6100080F09A80BCF1004F08BF5FEA500C50F1C7
:10E62000000041EB045141EA050130BD5FEA4C0CAA
:10E63000404141EB010111F4801FA4F10104E9D133
:10E6400091F0000F04BF01460020B1FA81F308BF2A
:10E650002033A3F10B03B3F120020CDA0C3208DDF6
:10E6600002F1140CC2F10C0201FA0CF021FA02F1D1
:10E670000CE002F11402D8BFC2F1200C01FA02F141
:10E6800020FA0CFCDCBF41EA0C019040E41AA2BF66
:10E6900001EB0451294330BD6FEA04041F3C1CDA2E
:10E6A0000C340EDC04F11404C4F1200220FA04F04E
:10E6B00001FA02F340EA030021FA04F345EA0301F8
:10E6C00030BDC4F10C04C4F1200220FA02F001FABA
:10E6D00004F340EA0300294630BD21FA04F029463C
:10E6E00030BD94F0000F83F4801306BF81F48011D5
:10E6F0000134013D4EE77FEA645C18BF7FEA655C48
:10E7000029D094EA050F08BF90EA020F05D054EA19
:10E71000000C04BF1946104630BD91EA030F1EBF1E
:10E720000021002030BD5FEA545C05D14000494122
:10E7300028BF41F0004130BD14F580043CBF01F515
:10E74000801130BD01F0004545F0FE4141F47001FB
:10E750004FF0000030BD7FEA645C1ABF19461046D6
:10E760007FEA655C1CBF0B46024650EA013406BFD7
:10E7700052EA033591EA030F41F4002130BD00BF96
:10E7800090F0000F04BF0021704730B54FF4806453
:10E7900004F132044FF000054FF0000150E700BFD4
:10E7A00090F0000F04BF0021704730B54FF4806433
:10E7B00004F1320410F0004548BF40424FF0000120
:10E7C0003EE700BF42004FEAE2014FEA31014FEA63
:10E7D00002701FBF12F07F4393F07F4F81F06051B2
:10E7E000704792F0000F14BF93F07F4F704730B521
:10E7F0004FF4607401F0004521F0004120E700BFB4
:10E8000050EA010208BF704730B54FF000050AE03A
:10E8100050EA010208BF704730B511F0004502D53B
:10E82000404261EB41014FF4806404F132045FEA3D
:10E83000915C3FF4DCAE4FF003025FEADC0C18BFE2
:10E8400003325FEADC0C18BF033202EBDC02C2F1D8
:10E85000200300FA03FC20FA02F001FA03FE40EA6A
:10E860000E0021FA02F11444C1E600BF4FEA410252
:10E87000B2F1E04324BFB3F5001CDCF1FE5C0DD91E
:10E8800001F0004C4FEAC0024CEA5070B2F1004F68
:10E8900040EB830008BF20F00100704711F0804F6B
:10E8A00021D113F13872BCBF01F00040704741F430
:10E8B00080114FEA5252C2F11802C2F1200C10FA34
:10E8C0000CF320FA02F018BF40F001004FEAC12318
:10E8D0004FEAD32303FA0CFC40EA0C0023FA02F3BC
:10E8E0004FEA4303CCE77FEA625307D150EA013392
:10E8F0001EBF4FF0FE4040F44000704701F0004062
:10E9000040F0FE4040F40000704700BF80F000403F
:10E9100002E000BF81F0004142001FBF5FEA4103F7
:10E9200092EA030F7FEA226C7FEA236C6AD04FEAF7
:10E930001262D2EB1363C1BFD2184140484041403C
:10E94000B8BF5B42192B88BF704710F0004F40F4EE
:10E95000000020F07F4018BF404211F0004F41F40A
:10E96000000121F07F4118BF494292EA030F3FD0D6
:10E97000A2F1010241FA03FC10EB0C00C3F12003E9
:10E9800001FA03F100F0004302D5494260EB400078
:10E99000B0F5000F13D3B0F1807F06D340084FEAE3
:10E9A000310102F10102FE2A51D2B1F1004F40EBD8
:10E9B000C25008BF20F0010040EA03007047490040
:10E9C00040EB000010F4000FA2F10102EDD1B0FA0B
:10E9D00080FCACF1080CB2EB0C0200FA0CF0AABF00
:10E9E00000EBC25052421843BCBFD040184370479E
:10E9F00092F0000F81F4000106BF80F400000132A4
:10EA0000013BB5E74FEA41037FEA226C18BF7FEA7A
:10EA1000236C21D092EA030F04D092F0000F08BFBC
:10EA20000846704790EA010F1CBF0020704712F0A3
:10EA30007F4F04D1400028BF40F00040704712F1E2
:10EA400000723CBF00F50000704700F0004343F047
:10EA5000FE4040F4000070477FEA226216BF08467D
:10EA60007FEA23630146420206BF5FEA412390EA40
:10EA7000010F40F4800070474FF0000304E000BF36
:10EA800010F0004348BF40425FEA000C08BF7047E7
:10EA900043F0964301464FF000001CE050EA0102AB
:10EAA00008BF70474FF000030AE000BF50EA0102C0
:10EAB00008BF704711F0004302D5404261EB4101AD
:10EAC0005FEA010C02BF84460146002043F0B643D2
:10EAD00008BFA3F18053A3F50003BCFA8CF2083AF7
:10EAE000A3EBC25310DB01FA02FC634400FA02FC00
:10EAF000C2F12002BCF1004F20FA02F243EB020007
:10EB000008BF20F00100704702F1200201FA02FC68
:10EB1000C2F1200250EA4C0021FA02F243EB02005B
:10EB200008BF20EADC7070474FF0FF0C1CEAD0529F
:10EB30001EBF1CEAD15392EA0C0F93EA0C0F6FD060
:10EB40001A4480EA010C400218BF5FEA41211ED03E
:10EB50004FF0006343EA501043EA5111A0FB01312A
:10EB60000CF00040B1F5000F3EBF490041EAD371FF
:10EB70005B0040EA010062F17F02FD2A1DD8B3F17B
:10EB8000004F40EBC25008BF20F00100704790F0EA
:10EB9000000F0CF0004C08BF49024CEA502040EA3C
:10EBA00051207F3AC2BFD2F1FF0340EAC250704702
:10EBB00040F400004FF00003013A5DDC12F1190F40
:10EBC000DCBF00F000407047C2F10002410021FAB2
:10EBD00002F1C2F1200200FA02FC5FEA310040F1CA
:10EBE000000053EA4C0308BF20EADC70704792F043
:10EBF000000F00F0004C02BF400010F4000F013A7B
:10EC0000F9D040EA0C0093F0000F01F0004C02BF75
:10EC1000490011F4000F013BF9D041EA0C018FE7E4
:10EC20000CEAD15392EA0C0F18BF93EA0C0F0AD0EA
:10EC300030F0004C18BF31F0004CD8D180EA010010
:10EC400000F00040704790F0000F17BF90F0004FA9
:10EC5000084691F0000F91F0004F14D092EA0C0F8B
:10EC600001D142020FD193EA0C0F03D14B0218BF1E
:10EC7000084608D180EA010000F0004040F0FE4064
:10EC800040F40000704740F0FE4040F44000704700
:10EC90004FF0FF0C1CEAD0521EBF1CEAD15392EA7F
:10ECA0000C0F93EA0C0F69D0A2EB030280EA010C6F
:10ECB00049024FEA402037D04FF0805343EA111108
:10ECC00043EA10130CF000408B4238BF5B0042F166
:10ECD0007D024FF4000C8B4224BF5B1A40EA0C000B
:10ECE000B3EB510F24BFA3EB510340EA5C00B3EB3D
:10ECF000910F24BFA3EB910340EA9C00B3EBD10F2B
:10ED000024BFA3EBD10340EADC001B0118BF5FEA7C
:10ED10001C1CE0D1FD2A3FF650AF8B4240EBC250A5
:10ED200008BF20F0010070470CF0004C4CEA502066
:10ED30007F32C2BFD2F1FF0340EAC250704740F4B5
:10ED400000004FF00003013A37E792F0000F00F0A7
:10ED5000004C02BF400010F4000F013AF9D040EA25
:10ED60000C0093F0000F01F0004C02BF490011F4B9
:10ED7000000F013BF9D041EA0C0195E70CEAD153B1
:10ED800092EA0C0F08D142027FF47DAF93EA0C0F98
:10ED90007FF470AF084676E793EA0C0F04D14B027C
:10EDA0003FF44CAF08466EE730F0004C18BF31F02E
:10EDB000004CCAD130F000427FF45CAF31F0004328
:10EDC0007FF43CAF5FE700BF4FF0FF3C06E000BFC1
:10EDD0004FF0010C02E000BF4FF0010C4DF804CDE4
:10EDE0004FEA40024FEA41037FEA226C18BF7FEAF4
:10EDF000236C11D001B052EA530C18BF90EA010FF6
:10EE000058BFB2EB030088BFC81738BF6FEAE17084
:10EE100018BF40F0010070477FEA226C02D15FEA20
:10EE2000402C05D17FEA236CE4D15FEA412CE1D08C
:10EE30005DF8040B704700BF844608466146FFE753
:10EE40000FB5FFF7C9FF002848BF10F1000F0FBD35
:10EE50004DF808EDFFF7F4FF0CBF012000205DF82E
:10EE600008FB00BF4DF808EDFFF7EAFF34BF0120B3
:10EE700000205DF808FB00BF4DF808EDFFF7E0FF4C
:10EE800094BF012000205DF808FB00BF4DF808ED9D
:10EE9000FFF7D2FF94BF012000205DF808FB00BF00
:10EEA0004DF808EDFFF7C8FF34BF012000205DF8E2
:10EEB00008FB00BF4FEA40024FEA41037FEA226CA1
:10EEC00002D15FEA402C08D17FEA236C02D15FEACD
:10EED000412C02D14FF0000070474FF00100704705
:10EEE000014B1868704700BF3802002070B50F4E04
:10EEF0000F4D761BB61018BF002405D0013455F80D
:10EF0000043B9847A642F9D10A4E0B4D761B03F0FD
:10EF1000F7FBB61018BF002406D0013455F8043BA7
:10EF20009847A642F9D170BD70BD00BF0C274100C3
:10EF30000C274100142741000C2741000FB400B5F5
:10EF4000074983B004AB086853F8042B8168019328
:10EF500000F024FE03B05DF804EB04B0704700BF7E
:10EF600038020020024B0146186800F00BB800BFC1
:10EF700038020020024B0146186801F02BBF00BF89
:10EF8000380200202DE9F04F01F10B06162E83B058
:10EF9000054640F29E8036F0070600F1BD80B14282
:10EFA00000F2BA8000F040FCB6F5FC7FC0F093821E
:10EFB000730A00F0B880042B00F27981B30903F1E1
:10EFC000390003F1380EC300BF4F3B44A3F10801E1
:10EFD0005C68A14206D10CE0002A80F2AA80E468B5
:10EFE000A14206D0636823F003039A1B0F2AF3DDC6
:10EFF00070463C69DFF8E4E2744500F0AB81636879
:10F0000023F003039A1B0F2A00F39081002AC7F80C
:10F0100014E0C7F810E080F29D80B3F5007F80F027
:10F020006181DB0803F1010C99107A6857F83C8084
:10F03000C4F8088001238B4007EBCC011343083947
:10F04000E1607B6047F83C40C8F80C408210012426
:10F0500094409C4200F28B801C4206D120F00300B9
:10F0600064001C4200F10400FAD007EBC009CC4652
:10F070008046DCF80C309C4507D16DE1002A80F217
:10F080007B81DB689C4500F06781596821F00301B2
:10F090008A1B0F2AF2DDD3F80CC0D3F80880009346
:10F0A0009C19284646F0010642F001055E60C8F84A
:10F0B0000CC0CCF808807C613C61C4F80CE0C4F85A
:10F0C00008E065605A5000F0B5FB009B03F10804AE
:10F0D0001EE0102920D800F0A7FB102618230220DC
:10F0E000794F3B44A3F108025C68944200F03D81F3
:10F0F0006368E168A66823F00303234428465A683E
:10F10000F16042F001028E605A6000F093FB083417
:10F11000204603B0BDE8F08F00240C2320462B606E
:10F1200003B0BDE8F08F40204FF400734FF03F0E66
:10F130004AE72344E1685A68A66842F00102F16098
:10F1400028468E605A6000F075FB0834204603B0F4
:10F15000BDE8F08F234428465A6842F001025A6005
:10F1600000F068FB0834204603B0BDE8F08FBC68AF
:10F17000636823F00308B04504D3A8EB06030F2B04
:10F1800000F38580DFF85891504BD9F800201B68B8
:10F190000132334404EB080A00F0558103F5805333
:10F1A0000F3323F47F6B2BF00F0B5946284600F0EA
:10F1B00047FB411C024600F0FC80824500F2F780CC
:10F1C000434B19685944196000F04D81D9F800008B
:10F1D00001301BBFA2EB0A0A5144C9F80020196094
:10F1E00012F0070100F01581C1F10800C1F580514E
:10F1F0000244083102EB0B09C9F30B09A1EB090921
:10F20000494628460193009200F01AFB431C9DE8F2
:10F210000C0000F04381801A484440F00100196856
:10F22000BA604944BC425060196017D0B8F10F0F62
:10F2300040F2FB806068A8F10C0222F0070204EBA8
:10F24000020E00F001004FF0050C10430F2A606021
:10F25000CEF804C0CEF808C000F217811D4BBC6880
:10F260001A68914288BF19601B4B1A689142626804
:10F2700088BF196022F003029642A2EB060301D870
:10F280000F2B04DC284600F0D5FA002440E7A21931
:10F2900043F0010346F0010666602846BA605360F9
:10F2A00000F0C8FA0834204603B0BDE8F08F142BF4
:10F2B00071D9542B00F2A380330B03F16F0003F1DB
:10F2C0006E0EC30080E600BF68060020140F002009
:10F2D000E40E00200C0F0020100F0020700600200C
:10F2E000700A00205A0A042A5BD9142A00F2AE8060
:10F2F00002F15C01C9005B3207EB010C7958ACF1FB
:10F30000080C8C4500F088804A6822F00302934282
:10F3100073D289688C45F7D1DCF80C207B68E260F9
:10F32000C4F808C09460CCF80C408FE6A11946F0F0
:10F33000010C42F00106C4F804C028467961396125
:10F34000C1F80CE0C1F808E04E60E25000F072FA3B
:10F350000834DDE67B6879E608F1010818F0030F50
:10F360000CF1080C7FF485AE2DE0DC68A34208BFE9
:10F3700002303FF43EAEBBE619441C464A68DB68E7
:10F3800054F8086F42F001024A602846F3609E601C
:10F3900000F050FABCE603F15C0003F15B0EC30021
:10F3A00012E69A0902F13901C9003832A4E7BC42D9
:10F3B00054D0BC68626822F003025DE759F808394E
:10F3C000994540F0868010F0030F00F1FF30F5D131
:10F3D0007B6823EA04037B6064009C423FF6C7AE6F
:10F3E000002C3FF4C4AE1C4240467FF43EAE6400A5
:10F3F0001C4200F10400FAD037E68C468CE7B3F5E6
:10F40000AA7F15D8F30B03F1780003F1770EC30040
:10F41000DAE54FF48051EDE67B689210012101FAA4
:10F4200002F213437B60624679E70123536029E7C8
:10F4300040F25452934222D8B30C03F17D0003F101
:10F440007C0EC300C0E503F1100BAEE6542A29D8A8
:10F450001A0B02F16F01C9006E324DE7204B19689B
:10F4600059441960B2E6CAF30B0000287FF4AEAE2F
:10F4700008EB0B03BA6843F001035360EEE67F200C
:10F480004FF47E734FF07E0E9EE504F1080128468E
:10F49000009301F09FFC009B1968DFE601204FF00C
:10F4A0000009BCE6B2F5AA7F05D8DA0B02F17801B3
:10F4B000C900773220E740F254518A4205D89A0CAD
:10F4C00002F17D01C9007C3216E74FF47E717E2285
:10F4D00012E77B6880E7F00806F1080300E600BF4A
:10F4E000E40E00200000000000000000000000000A
:10F4F00001F0FF01102A2BDB10F0070F08D010F8E5
:10F50000013B013A8B422DD010F0070F42B3F6D1E8
:10F51000F0B441EA012141EA014122F007047FF001
:10F5200000070023F0E80256083C85EA010586EA58
:10F53000010685FA47F5A3FA87F586FA47F6A5FA94
:10F5400087F68EB9EED1F0BC01F0FF0102F00702A0
:10F5500032B110F8013B013A83EA010313B1F8D14B
:10F560000020704701387047002D06BF354603382C
:10F57000073815F0010F07D1013015F4807F02BF65
:10F58000013015F4C03F0130F0BC0138704700BFB6
:10F59000844641EA000313F003036DD1403A41D39E
:10F5A00051F8043B40F8043B51F8043B40F8043B5D
:10F5B00051F8043B40F8043B51F8043B40F8043B4D
:10F5C00051F8043B40F8043B51F8043B40F8043B3D
:10F5D00051F8043B40F8043B51F8043B40F8043B2D
:10F5E00051F8043B40F8043B51F8043B40F8043B1D
:10F5F00051F8043B40F8043B51F8043B40F8043B0D
:10F6000051F8043B40F8043B51F8043B40F8043BFC
:10F6100051F8043B40F8043B51F8043B40F8043BEC
:10F62000403ABDD2303211D351F8043B40F8043B8C
:10F6300051F8043B40F8043B51F8043B40F8043BCC
:10F6400051F8043B40F8043B103AEDD20C3205D39C
:10F6500051F8043B40F8043B043AF9D2043208D094
:10F66000D2071CBF11F8013B00F8013B01D30B8806
:10F6700003806046704700BF082A13D38B078DD0E4
:10F6800010F003038AD0C3F10403D21ADB071CBFB6
:10F6900011F8013B00F8013B80D331F8023B20F820
:10F6A000023B7BE7043AD9D3013A11F8013B00F859
:10F6B000013BF9D20B7803704B7843708B788370E1
:10F6C000604670478842F0B50DD98B1898420AD22F
:10F6D0008418002A51D0224613F8014D02F8014D3A
:10F6E0009942F9D1F0BD0F2A48D941EA00039B079E
:10F6F00046D100F1100401F11003154653F8106CC7
:10F7000044F8106C53F80C6C44F80C6C53F8086C0B
:10F7100044F8086C103D53F8046C44F8046C0F2D49
:10F7200003F1100304F11004E8D8A2F1100323F050
:10F730000F0302F00F0E1033BEF1030F1944034400
:10F7400021D91E1F0D467446043C55F8047B46F82B
:10F75000047F032CF8D8AEF1040424F0030404342D
:10F760002144234402F0030262B1013B0A4411F830
:10F77000014B03F8014F8A42F9D1F0BD0346F3E78C
:10F780000346F2E7F0BD7246EEE700BF70B48607AD
:10F7900046D0541E002A41D0CAB2034602E014F1FA
:10F7A000FF343BD303F8012B9D07F8D1032C2ED94E
:10F7B000CDB245EA05250F2C45EA054519D903F1D7
:10F7C00010022646103E0F2E42F8105C42F80C5CE8
:10F7D00042F8085C42F8045C02F11002F2D8A4F18D
:10F7E000100222F00F0204F00F041032032C134415
:10F7F0000DD91E462246043A032A46F8045BFAD87D
:10F80000221F22F003020432134404F003042CB13B
:10F81000C9B21C4403F8011B9C42FBD170BC704769
:10F8200014460346C2E700BF014801F06DBD00BFAA
:10F83000A81E0020014801F069BD00BFA81E0020DD
:10F8400038B5074C0023054608462360FCF7C8FE80
:10F85000431C00D038BD2368002BFBD02B6038BD83
:10F86000BC1E002000290CBF022200224FF480633E
:10F8700000F000B82DE9F043614C256883B00446E0
:10F880000F4690461E4615B1AB6B002B64D0B8F105
:10F89000020F06D0B8F1010F00F29F80002EC0F2D7
:10F8A0009C80636ED80734D52146284601F014F9B0
:10F8B000216B41B104F14003994202D0284601F086
:10F8C00089FA00232363B4F90C300022A26162603C
:10F8D0001A063AD423F44A6323F00303B8F1020F63
:10F8E000A3811DD001AB6A462146284601F010FDD8
:10F8F000A3891843A081002E32D1009E3046FFF725
:10F9000031FB074600286BD0A38943F08003A38115
:10F9100028E0A3899905C7D4A06D01F0F5FCC3E7E1
:10F920000025616E002604F1430243F0020301202A
:10F93000A660CE07A38122602261606101D4980590
:10F940003ED5284603B0BDE8F0832169284601F082
:10F9500041FAB4F90C30BDE7284601F015F996E7F5
:10F96000002FCBD0AB6B002B33D0009BB4F90C2015
:10F9700027609E421CBF42F40062A281B8F1010FD1
:10F9800004BF42F00102A28192B212F00803276183
:10F9900066610ED0D1071AD5656E7642002315F048
:10F9A0000105A661A36009D00025284603B0BDE883
:10F9B000F083A360656E15F00105F5D19305C0D401
:10F9C000A06D01F0A3FC284603B0BDE8F083A6605B
:10F9D000F0E7284601F0D8F8C7E74FF0FF35B0E769
:10F9E000DDF80090B14504D04846FFF7BBFA074662
:10F9F00020B9B4F90C304FF0FF3592E74E4683E75B
:10FA0000380200200000000000000000000000009C
:10FA100000000000000000000000000000000000E6
:10FA200000000000000000000000000000000000D6
:10FA300000000000000000000000000000000000C6
:10FA400090F800F06DE9024520F007016FF0000C1E
:10FA500010F0070491F820F040F049804FF00004C6
:10FA60006FF00700D1E9002391F840F000F10800A1
:10FA700082FA4CF2A4FA8CF283FA4CF3A2FA8CF3D9
:10FA80004BBBD1E9022382FA4CF200F10800A4FA40
:10FA90008CF283FA4CF3A2FA8CF3E3B9D1E9042394
:10FAA00082FA4CF200F10800A4FA8CF283FA4CF3CB
:10FAB000A2FA8CF37BB9D1E9062301F1200182FA85
:10FAC0004CF200F10800A4FA8CF283FA4CF3A2FA8B
:10FAD0008CF3002BC6D0002A04BF04301A4612BA99
:10FAE000B2FA82F2FDE8024500EBD2007047D1E99C
:10FAF000002304F00305C4F100004FEAC50514F02B
:10FB0000040F91F840F00CFA05F562EA05021CBFFB
:10FB100063EA050362464FF00004A9E72DE9F84FB8
:10FB20004B6E9C0493462FD59368126853B30E46D0
:10FB3000074602F1080919E920045FEA9A0817D07C
:10FB4000043D002401E0A04510D0324655F8041FC2
:10FB5000384601F0BBF8431C04F10104F3D1002343
:10FB6000CBF80830CBF80430BDE8F88FDBF808306C
:10FB70002AF0030AA3EB0A03CBF8083009F10809BD
:10FB8000002BD8D10020EAE701F00AFA0023CBF8D5
:10FB90000830CBF80430BDE8F88F00BF2DE9F04FF6
:10FBA000ADB01D468B4690460793069018B1836B07
:10FBB000002B00F0F380DBF86430BBF90C00DF07AA
:10FBC00081B202D48E0540F1FC808C040AD4DBF8AB
:10FBD000643040F4005123F40053ABF80C10CBF820
:10FBE000643089B2080740F1B380DBF81030002B95
:10FBF00000F0AE8001F01A030A2B00F0B58000235C
:10FC00000DF170090B93119310930393CDF83C9071
:10FC1000CA46CDF810B098F800304446FBB1252B09
:10FC200002D11CE0252B03D014F8013F002BF9D1A1
:10FC3000A4EB08059DB1109B119ACAF8008001330E
:10FC40002A44072BCAF80450119210937ADD002A37
:10FC500040F0B084039B10922B44CA460393237850
:10FC6000002B00F0E08300204FF000038DF83730C8
:10FC700004F1010862780546064603464FF0FF345A
:10FC800008F10108A2F12001582900F2DE82DFE824
:10FC900011F02102DC02DC022902DC02DC02DC02BF
:10FCA000DC02DC02DC0289029502DC02A200BD0259
:10FCB000DC029F01A401A401A401A401A401A401E8
:10FCC000A401A401A401DC02DC02DC02DC02DC02EF
:10FCD000DC02DC02DC02DC02DC02B201DC02DC025F
:10FCE000DC02DC02DC02DC02DC02DC02DC02DC0224
:10FCF0009701DC02DC02DC02DC02DC029B01DC029C
:10FD0000DC025302DC02DC02DC02DC02DC02DC028C
:10FD1000DC02DC02DC02DC025A021B02DC02DC0236
:10FD2000DC026E021B02DC02DC027302DC02F50163
:10FD300082010902D702DC029A02DC02A700DC027F
:10FD4000DC022E020AF1080A039B2B44039386E788
:10FD50005946069800F0ACFD18BBBBF80C1001F03A
:10FD60001A030A2B7FF44BAFBBF90E30002BFFF6C2
:10FD700046AFDBF86430DB0705D48F0503D4DBF82E
:10FD8000580001F0C3FA2B4642465946069800F047
:10FD90004DFD039003982DB0BDE8F08F00F0F4FE08
:10FDA00009E7DBF86430D90704D4BBF80C309A05B6
:10FDB00040F1AA844FF0FF33039303982DB0BDE8C0
:10FDC000F08FDBF8580001F09FFABBF90C0081B20C
:10FDD000FBE67642079243F0040398F800204FE7D1
:10FDE00008969E0600F150840799DD060A4600F148
:10FDF000EF83580640F1EC830E880431002701227E
:10FE000007914FF000018DF837100025611C00F0BC
:10FE1000168123F08001029156EA070140F0148117
:10FE2000002C40F05C83002A40F0B78313F00103FC
:10FE3000059300F057840DF1B00B30230BF8413DD2
:10FE4000059BA342B8BF234601930DB10133019333
:10FE5000029B13F00203099302D0019B023301932A
:10FE6000029B13F084030A9340F01782089B019AC7
:10FE70009D1A002D40F31182102D40F39084109BA9
:10FE8000119AC44ED6461027A2461946069C07E092
:10FE900001F1020C0EF1080E0146103D102D11DD8E
:10FEA000481C1032072811928EE8C0001090EFDD38
:10FEB000002A40F0E481103D102D11464FF0010C56
:10FEC000CE46EDDC54466146F2462A44072911929B
:10FED000CAF80060CAF80450109100F3EC829DF853
:10FEE00037500AF1080A481C002D40F0DE81099BBA
:10FEF000002B00F0F88102320EA90223072811928C
:10FF000010908AE80A0040F3EA81002A40F08C83CE
:10FF10000A9B802B4FF001001146CA4640F0E78152
:10FF2000089B019D5E1B002E40F3E181102E9A4D2F
:10FF300040F35084D4461027A246069C07E001F106
:10FF4000020E0CF1080C0146103E102E11DD481C6B
:10FF50001032072811928CE8A0001090EFDD002AE3
:10FF600040F09D82103E102E4FF0010E1146CC46FF
:10FF7000EDDC5446E2463244BEF1070F11928AE8A6
:10FF80006000CDF840E000F369830AF1080A0EF141
:10FF900001007146ABE1089613F0200240F08C831B
:10FFA00013F0100140F01A8313F0400200F01683A2
:10FFB00007980A460146043106880791002720E782
:10FFC000089643F01003E7E7089643F0100308E7AC
:10FFD00043F0800398F8002052E6A2F13001002699
:10FFE00018F8012B06EB860601EB4606A2F130015C
:10FFF0000929F5D946E60896002840F0088443F020
:020000040041B9
:1000000010039E0600F14C83DD0600F1F3825806D2
:1000100040F1F082079DB5F900602A46F7170432D7
:10002000304639460792002871F10002C0F25D8324
:10003000611C9DF837504FF001027FF4EAAE56EA9A
:10004000070100F04D820293012A00F08C82022AFF
:1000500040F05C820B98CB46330906F00F0143EA6F
:1000600007733A091E461746435C0BF8013D56EAF2
:100070000703F1D1A9EB0B030593E1E6002840F05B
:10008000C083990600F16783DA0600F1F1805B0610
:1000900040F1EE80079A136804320792BDF80C20F5
:1000A0001A80B8E507983D4A08960B9206687822B0
:1000B000302104308DF8392043F0020307900027E7
:1000C0008DF8381002229CE60896002899D08DF809
:1000D000375096E798F80020002D7FF4D1AD01202D
:1000E0002025CDE543F0010398F80020C8E50896E7
:1000F000002840F0938329490B919F0600F1E88284
:100100000798DE06014600F170825D0640F16D82BF
:100110000431068807910027D80740F1228256EA69
:10012000070100F01E8230218DF8392043F00203D0
:100130008DF83810022264E60896002840F06B83A0
:1001400017490B91D9E7079908960A688DF8482056
:100150004FF000000A468DF837000432012001906C
:10016000079205900DF1480B0293002470E643F0CE
:10017000400398F8002083E598F800206C2A03BF1C
:1001800098F8012043F0200308F1010843F0100320
:1001900076E500BFCC254100DC254100B0254100BB
:1001A0009C25410007990E680A46002E02F10402C0
:1001B000FFF60FAE079298F8002061E598F800204E
:1001C00001202B255CE507990896D1F800B04FF087
:1001D00000028DF837200E1DBBF1000F00F0E58204
:1001E000671C00F0C4822246002158460193FFF7A5
:1001F0007FF9019B002800F0E582A0EB0B0205923D
:10020000079602939DF83750002419E698F80020CD
:100210002A2A08F1010700F0E982A2F13001092938
:10022000B8464FF000043FF62DAD18F8012B04EB53
:10023000840401EB4404A2F130010929F5D921E538
:1002400043F0200398F800201AE50896002840F0B3
:10025000DB82002A00F0E78001218DF848204FF072
:10026000000201918DF8372005910DF1480B7BE7D5
:10027000079A136804320792039A1A60CBE40FAA14
:1002800004992046FFF74AFC002840F03981109974
:10029000119A01F1010CCE46FFE51099119A481C04
:1002A0009DF83750002D3FF422AE01320DF1370595
:1002B0000121072811921090CAF80050CAF80410C2
:1002C00040F30881002A40F0BC81099B002B3FF4D9
:1002D0001FAE0EAB022208461C931D92CA46014671
:1002E0000AF1080A01300A9B802B3FF419AE059BE6
:1002F000E41A002C2EDD102CB34D1EDDD646102640
:10030000069FDDF810A006E0881C0EF1080E1946C5
:10031000103C102C10DD4B1C1032072B11928EE874
:1003200060001093F0DD002A65D1103C102C4FF0D6
:1003300001001146CE46EEDCF24622440728119217
:10034000CAF80050CAF80440109000F385800AF102
:10035000080A01300599CAF800B00A44072811922A
:10036000CAF80410109040F38280002A40F01881EF
:10037000029B1092580735D5089B01995C1A002CF6
:1003800040F3E780CA46102C40F3188210998F4E34
:10039000069FDDF810B0102506E0881C0AF1080A57
:1003A0001946103C102C11DD4B1C1032072B1192FA
:1003B000CAF80060CAF804501093EEDD42BB103C4E
:1003C000102C4FF001001146CA46EDDC22440728EC
:1003D0001192CAF80060CAF80440109051DD002A5A
:1003E00040F09B81039B089A01998A42ACBF9B18FD
:1003F0005B1803934EE00FAA51463846FFF78EFB79
:10040000002840F03F811099119A481CCE467FE7A2
:100410000FAA59463846FFF781FB60B91099119A27
:10042000481CCA46BDE7119BDDF810B0002B40F018
:10043000D48100231093DBF8643013F0010FBBF874
:100440000C3002D19A0540F1DE805B063FF5B2AC7C
:1004500003982DB0BDE8F08F002A40F00681059A80
:100460001D9201231192CDF870B01093CA460AF183
:10047000080A029B590704D5089B01995C1A002CB5
:1004800081DC039B089901988142ACBF5B181B1863
:10049000039372BB00231093CA46FFF7BCBB0FAA9D
:1004A00004992046FFF73AFB50BB1099119A01F1CD
:1004B000010ECC4648E5002A40F040819DF83710F7
:1004C000002900F01B8101220DF1370110461D9219
:1004D0001C91CA4601460AF1080A013007E5029B51
:1004E000012A00F09880022A0DD1029300260027ED
:1004F000B0E50FAA04990698FFF710FB0028C9D0B1
:10050000DDF810B097E7029300260027494600E087
:100510005946F20842EA4772F80806F00703074610
:100520001646303356EA070201F8013C01F1FF3B61
:10053000EED1029AD6077FF59DAD302B3FF49AADF0
:10054000023930230BF8013CA9EB010305938B46DC
:1005500076E4039B089A8A42ACBF9B185B1803930E
:1005600098E702224DE4002F08BF0A2E52D3CB4653
:10057000304639460A22002301F010FB30320BF8D6
:10058000012D3046394600230A2201F007FB0646BA
:100590000F4656EA0703EBD16CE50594CB464FE4D2
:1005A0000FAA04990698FFF7B9FA0028A8D1119A62
:1005B000CA465EE70FAA04990698FFF7AFFA00282B
:1005C0009ED1CA46FFF7C0BBDC254100CC254100C7
:1005D0000431166807910122002712E407980146AA
:1005E00004310668079100270BE40E680431079177
:1005F000002791E507990E680A46F717043207921B
:10060000304639460FE5DBF8580000F07FFEBBF8B6
:100610000C301AE7029B02930DF1B00B3036012328
:100620000BF8416D05930BE40FAA04990698FFF7A8
:1006300075FA00287FF464AF1099119A481CCA46D5
:1006400051E60FAA04990698FFF768FA00287FF48C
:1006500057AF1099119A481CCA4648E4002A40F046
:10066000918001201146CA4641E60FAA04990698D6
:10067000FFF754FA00287FF443AF1098119A013025
:10068000CA4667E6D346D6E6079E073626F0070237
:1006900002F10801D2E9006707910122FFF7B1BB1F
:1006A000079E073626F00706D6E9000106F1080284
:1006B000079206460F46B6E4079E073626F0070265
:1006C00002F10801D2E9006707910022FFF799BB08
:1006D000079E073626F0070101F108000790D1E9CF
:1006E000006719E5CB46FFF7ABBB2D25764267EBDC
:1006F00047078DF837500122FFF788BB099BB3B934
:1007000011460120CA46F2E5DBF8580000F0FEFD74
:100710004FF0FF330393FFF750BB0FAA04990698DD
:10072000FFF7FCF900287FF4EBAE119AA9E60EABB7
:1007300002221C931D920120CA46D0E50FAA0499FB
:100740000698FFF7EBF900287FF4DAAE1099119ABA
:10075000481CCA46A4E5079A03991368CD170846B2
:10076000043229460792C3E90001FFF754BA5846FC
:1007700007960293FFF764F9002405909DF837501F
:10078000FFF75EBB0FAA04990698FFF7C7F9002888
:100790007FF4B6AE1099119A481CCA46A7E5109985
:1007A000119A204E0131FFF790BB062C28BF06247A
:1007B000059407960194DFF870B0D5E41098194EAF
:1007C000013003E605949DF83750079602930446DE
:1007D000FFF736BB8646FFF7CEBB06980FAA5946F1
:1007E000FFF79CF900283FF424AE24E6079998F817
:1007F00001200C68043144EAE474B8460791FFF71D
:100800003FBA8DF837503CE48DF8375021E58DF82C
:100810003750FFF7F4BB8DF8375091E48DF837501F
:1008200069E400BFCC254100C42541002DE9F04119
:100830000C46ADF58D6D8989666EE589199621F0B6
:1008400002010646E069ADF80C1017464FF48061CE
:10085000626AADF80E5098461AAD0023079016A8AC
:1008600009920693009504950291059100F048FDC8
:1008700043463A4669463046FFF790F9051E07DBC6
:100880003046694600F028F9002818BF4FF0FF35C0
:10089000BDF80C305B0603D5A38943F04003A38168
:1008A000169800F02FFD28460DF58D6DBDE8F081FE
:1008B00038B5304B1B6805460C4613B19A6B002ABD
:1008C00038D0B4F90C2093B218070CD52069A8B120
:1008D00013F001021ED0636900225B42A361A26093
:1008E000F0B1002038BDD9063CD5580726D4206980
:1008F00042F00803A3819BB20028E9D103F42072DF
:10090000B2F5007FE4D02846214600F02FFDA389F0
:100910002069DDE7990758BF6269A2600028E0D12D
:10092000B4F90C301A06DDD543F04003A3814FF033
:10093000FF3038BD184600F027F9C2E7216B51B1EE
:1009400004F14003994204D0284600F043FAB4F978
:100950000C200023236300232069636022F024021B
:100960002060C5E742F0400209232B604FF0FF30C2
:10097000A28138BD38020020024B13B1024800F0BA
:1009800005B8704700000000F90B41000023014644
:100990001A46184600F0DABFB1F90C309AB22DE9C8
:1009A000F0410D46110780463AD46A6843F400636B
:1009B000002AAB816FDDAC6A002C49D000229BB2CB
:1009C000D8F80060C8F8002013F4805267D02A6D70
:1009D0005F0705D569682B6B521A0BB1EB6BD21A06
:1009E0000023E9694046A047441C3CD0B5F90C30CF
:1009F0002A692A6023F400630022AB81DB046A6069
:100A000047D4296BC8F8006011B305F1400399423F
:100A100002D0404600F0DEF900202863BDE8F081F6
:100A20002E69AEB12C682E6091070CBF6B69002354
:100A3000A41BAB600AE0234632466F6AE969404670
:100A4000B8470028A4EB0004064404DD002CF2DCC7
:100A50000020BDE8F081AB8943F04003AB814FF04B
:100A6000FF30BDE8F081D8F800401D2CF3D8194BB9
:100A7000E340DB4313F00103EDD1B5F90C206B60CB
:100A800022F400632969AB81DA042960B9D5002C0E
:100A9000B7D12865B5E7EA6B002A8CDCD8E70123DB
:100AA000E9694046A047431C024602D0AB89AC6AC4
:100AB0008EE7D8F80030002BF8D01D2B01D0162B74
:100AC00002D1C8F80060C3E7AB8943F04003AB81B3
:100AD000BDE8F0810100402038B50D46044608B15C
:100AE000836BBBB1B5F90C0088B16B6EDB0701D429
:100AF000810517D520462946FFF74EFF6B6EDA07B2
:100B0000044602D4AB899B0507D5204638BD044670
:100B1000204638BD00F038F8E4E7A86D00F0F6FB99
:100B2000204638BDA86D00F0EFFBE3E7014900F077
:100B3000AFBB00BF351A410010B5002304468181C8
:100B4000C2810360436083604366036143618361E4
:100B5000194608225C30FEF719FE07480749084A83
:100B6000084B2062E4616162A262E36204F1580012
:100B7000BDE8104000F0C4BB791741009D1741004B
:100B8000D9174100F917410010B50446124800F08A
:100B9000BBFBA26BD2B904F53B731048C4F8E83232
:100BA0000321C4F8E022E063C4F8E4126068042181
:100BB000FFF7C2FF01220921A068FFF7BDFF022253
:100BC0001221E068FFF7B8FF0123A3630248BDE8E4
:100BD000104000F09BBB00BFA41E00202D0B410065
:100BE000014800F091BB00BFB81E0020014800F092
:100BF0008DBB00BFB81E002038B50A4C0A4D641BDF
:100C0000A4100AD004F18043013B05EB8305013CAD
:100C100055F804399847002CF9D1BDE8384001F067
:100C200079BD00BF24274100202741002DE9F0476E
:100C300082B080468946144600F054FB012836D025
:100C40004A4604F15C0301A9404600F031FE421C13
:100C5000064625D0A8B39DF804E000250DF1040A4E
:100C600009E023685A1C226083F800E00135B54290
:100C700027D215F80AE0A368013B002BA360F0DA45
:100C8000A769BB4271462246404602DBBEF10A0F0D
:100C9000E7D100F0B5FD431CE8D102B0BDE8F08714
:100CA000A38943F04003A38102B0BDE8F08709F1B6
:100CB000FF33FE2BC4D85FFA89FE06468DF804E0A8
:100CC000CBE7484602B0BDE8F08700BF30B5536EB1
:100CD00013F0010FB2F90C30144683B005469AB2F6
:100CE00001D190051CD5900406D4626E43F40053E4
:100CF00042F40052A381626628462246FFF796FF1F
:100D0000636EDA07054602D4A3899B0502D52846FF
:100D100003B030BDA06D00F0F9FA284603B030BD35
:100D2000A06D019100F0F0FAB4F90C3001999AB27B
:100D3000D9E700BFF8B5244F0C460646FEF774FD10
:100D4000BB685D68C4F57E610F3125F00305294459
:100D500021F47F6121F00F01A1F58054B4F5805F8B
:100D600007DB00213046FEF76BFDBB682B44984241
:100D700004D03046FEF75EFD0020F8BD61423046EB
:100D8000FEF75EFD01300DD0104BBA6819682D1BBF
:100D900045F001053046091B55601960FEF74AFD14
:100DA0000120F8BD00213046FEF74AFDBA68831ADB
:100DB0000F2BDEDD064C0549246843F00103001BC0
:100DC00053600860D5E700BF68060020E40E0020ED
:100DD000700A0020002944D02DE9F0410D468046DC
:100DE000FEF722FD55F8047C694927F00103A5F1BF
:100DF0000804E2188E685068B24220F003005ED00A
:100E0000FE0750600BD455F8087CE41B01F1080E76
:100E1000A56875453B446DD0E768EF60BD60151867
:100E20006D68ED073ED543F001026260E350B3F513
:100E3000007F17D2DB08581C9A104D6851F83070AB
:100E4000A7600123934001EBC0022B43083AE26004
:100E50004B6041F83040FC604046BDE8F041FEF791
:100E6000E9BC70475A0A042A52D89A0902F1390794
:100E7000FF0002F13805C819CA59083890424FD00E
:100E8000516821F003018B4232D292689042F7D12F
:100E9000C368A060E3609C60C4604046BDE8F04168
:100EA000FEF7C8BC95683B4FBD42034440D0D068B4
:100EB000E86043F0010285606260E350B7E7FF0736
:100EC000034407D455F8082CA41A1344A068E26818
:100ED000C2609060304A126843F001009342606043
:100EE0008C60B9D32D4B40461968FFF723FFB3E759
:100EF0001046CDE711184968C90744D49168D268F3
:100F0000CA60034443F0010091606060E350A3E7CE
:100F1000142A16D802F15C07FF0002F15B05AAE76C
:100F2000AA1001234D6893402B434B600346B0E762
:100F300043F001024C610C61E560A5606260E35022
:100F40008AE7542A06D81A0B02F16F07FF0002F154
:100F50006E0590E7B2F5AA7F06D8DA0B02F17807A2
:100F6000FF0002F1770586E740F25450824206D82E
:100F70009A0C02F17D07FF0002F17C057BE74FF43C
:100F80007E777E2577E743F001016160136063E7B8
:100F90006806002070060020740A0020140F00204C
:100FA0009368002B73D02DE9F04F8B8983B00C46EA
:100FB00019070090164626D5226922B313F00200C5
:100FC00035682CD04FF00009B04FC846B246B8453E
:100FD00043464A4628BF3B460098B8F1000F50D020
:100FE000E169666AB047002858DDDAF808301B1A54
:100FF0008144A8EB0008CAF80830002BE7D1002094
:1010000003B0BDE8F08F21460098FFF751FC00289F
:1010100040F03381A389356813F00200D2D113F078
:10102000010945D14F46019637B39A05D4F8088097
:1010300040F183804745C346C0F0AB8013F4906F06
:1010400040F0AC802068BA465A464946FEF73AFB63
:10105000A2682368A2EB08025B44A2602360019AA5
:101060009368A3EB0A03D144A7EB0A079360002B14
:10107000C5D0A389002FD8D1D5F800906F68083566
:10108000D2E7D5F80090D5F8048008359FE7002016
:10109000704721460098FFF71FFD70B3B4F90C307C
:1010A00043F040034FF0FF30A38103B0BDE8F08F61
:1010B000814633464E46A8469A464D464EB380B3C7
:1010C000206823696269B145CB4628BFB346984280
:1010D0005F4604D9A36813449B4500F3A68093455B
:1010E0004BDB1346676AE16900982A46B847071E3A
:1010F000D4DDB9EB0709CCD00120DAF80830DB1BCE
:101100003D44F61BCAF80830002B3FF478AF002EA0
:10111000D5D108F1080313E9600098460833002E82
:10112000F9D032460A212846FEF7E2F9002800F0FD
:10113000A1800130A0EB0509C2E72068236998422D
:1011400002D863699F425DD2B84528BFB84642467F
:101150004946FEF7B7FAA3682268A3EB08034244A6
:10116000A36022600BB1C24679E721460098FFF7E1
:10117000B3FC002892D1C24671E75A462946FEF7D1
:10118000A1FAA2682368A2EB0B025B44A260236071
:10119000AFE72068B846BA46BB4655E762692068A3
:1011A000216902EB4208A0EB010A08EBD8780AF1AA
:1011B00001004FEA680838444045424684BF8046F3
:1011C00042465B0544D511460098FDF7DBFE834699
:1011D000002855D052462169FEF7DAF9A38923F495
:1011E000906343F08003A3810BEB0A00A8EB0A0392
:1011F000C4F810B0C4F814802060A360B846BA46A2
:10120000BB4621E76FF00041B94228BF39464A4644
:1012100091FBF3F10098666A03FB01F3E169B047C3
:10122000B0F1000A3FF71BAF38E71A462946019391
:10123000FEF748FA2268019B00981A442260214672
:10124000FFF74AFC019B00287FF428AF1F4650E7B8
:10125000009800F0EBF883460028C5D1009D216975
:101260002846FFF7B7FDB4F90C300C2223F08003B9
:101270002A6015E706F1010922E74FF0FF30BFE6CB
:10128000009A0C231360B4F90C3009E700FCFF7FCF
:101290002DE9F84310F538771FD0884606464FF001
:1012A00000097D68BC68013D11D4A389012B05F1BB
:1012B000FF3508D9B4F90E3001332146304602D04B
:1012C000C04749EA00096B1C04F16804EDD13F688E
:1012D000002FE6D14846BDE8F883B9464846BDE848
:1012E000F88300BF044B054A1B685B6B002B08BFEB
:1012F000134693F828017047380200207C0A00202A
:10130000704700BF704700BF704700BF704700BF05
:1013100070B50C46B1F90E10002990B015461E4666
:1013200014DB01AA00F0E8FB00280FDB029A02F4AC
:101330007042A2F50052B2FA82F252094FF4806371
:101340004FF4006032602B6010B070BDA2890023A2
:1013500012F08000336004D0402218462A6010B09A
:1013600070BD4FF480632B6010B070BD8A89920706
:101370000B4606D501F1430201211A601A61596139
:101380007047F0B583B001AB6A460C460646FFF7DE
:10139000BFFF009905463046FDF7F4FDB4F90C3067
:1013A000D8B1019A154F0099F76343F08003A381E8
:1013B0002060206161611AB92B43A38103B0F0BDA5
:1013C0003046B4F90E1000F0ABFBA0B1A38923F0B6
:1013D000030343F001031BB2EEE79A05EED423F0BA
:1013E000030304F1430243F002030121A3812260BD
:1013F00022616161E2E7B4F90C30DDE72D0B4100B9
:1014000082B049B15AB16BB113780B601278101CDD
:1014100018BF012002B0704701A9002AF3D110467D
:1014200002B070476FF00100F4E700BF002900F040
:1014300095802DE9F04F0D46164683B0804606F1A3
:101440000B07FEF7F1F955F804EC162F2EF0030404
:10145000A5F108093CD810221746BE423DD8944257
:1014600043DAC44B996809EB0400884200F0B48069
:10147000436823F0010101444968C9074CD51EF0B7
:10148000010F00F09B8031464046FDF77BFD06468C
:1014900000283AD055F8043C23F001034B44A0F156
:1014A00008029A4200F02181221F242A00F20781BB
:1014B000132A00F2DB8003462A461168196051683E
:1014C000596092689A6029464046FFF783FC1CE009
:1014D00027F00707002F3A46BFDA00260C233046D4
:1014E000C8F8003003B0BDE8F08F2E46E31B0F2B89
:1014F0001ED8D9F8043003F0010323434C44C9F843
:101500000430636843F0010363604046FEF792F9DC
:10151000304603B0BDE8F08F23F00303E118914299
:101520001FDBC36882682E46D3600C469A60DDE7F5
:10153000D9F8042009EB070102F001024C4443F002
:1015400001031743C9F804704B60636843F001035B
:10155000083163604046FFF73DFCD6E71146FDF7D2
:1015600011BD1EF0010F8ED155F8081CA9EB010A20
:10157000DAF8041021F003010B442344934225DBE5
:10158000C26881685646CA609160DAF80C1056F855
:10159000080F221F242AC160886000F29480132A59
:1015A0006FD92968CAF808106968CAF80C101B2A94
:1015B00000F2A28008350AF1100263E055F8083CF9
:1015C000A9EB030ADAF8041021F00301631893422F
:1015D000FFF659AF5646D8E7416821F0030BA34404
:1015E00007F11000834556DA1EF0010F7FF44BAF70
:1015F00055F8081CA9EB010ADAF8041021F00301E0
:101600008B445845E2DC5646DAF80C1056F8080FC1
:10161000221F242AC160886000F28F80132A40F2C2
:101620008A802968CAF808106968CAF80C101B2A51
:1016300000F28A8008350AF1100229681160696891
:101640005160A96891600AEB0701ABEB070242F019
:10165000010299604A60DAF8043003F001031F4385
:101660004046CAF80470FEF7E5F851E72B680360BE
:101670006B6843601B2A2DD800F1080305F10802AE
:101680001BE732462968116069685160A96891605A
:101690001C46D1462AE709EB0701ABEB070B4BF0E1
:1016A000010299604A6055F8043C03F001031F43AE
:1016B000404645F8047CFEF7BDF82E4628E729464B
:1016C000FEF700F8FFE6294630461C46D146FDF7F6
:1016D000F9FF0BE7AB688360EB68C360242A17D07F
:1016E00000F1100305F11002E7E650F8043C23F086
:1016F00003031C442E46F9E6A968CAF81010E968ED
:10170000CAF81410242A0CD010350AF11802B9E7CF
:101710002B6903616B69436105F1180200F118033D
:10172000CBE62A69CAF818206A69CAF81C2018355D
:101730000AF12002A6E732467FE7294630460193A8
:10174000FDF7C0FF019B7EE7A968CAF81010E968A1
:10175000CAF81410242A03D010350AF118026CE7D5
:101760002A69CAF818206A69CAF81C2018350AF1D3
:10177000200262E76806002010B50C46B1F90E1091
:1017800000F0F6F9002803DB236D0344236510BD48
:10179000A38923F48053A38110BD00BF2DE9F0413C
:1017A0001646B1F90C201F46D3050C46054607D551
:1017B00000220223B1F90E1000F0C4F9B4F90C2094
:1017C000B4F90E1022F48052A2813B4632462846DC
:1017D000BDE8F04100F0A4B810B50C46B1F90E1008
:1017E00000F0B0F9A389421C0EBF23F4805343F4E8
:1017F00080532065A38110BDB1F90E1000F008B927
:10180000F8B50D461446064610B1836B002B4BD03D
:10181000B4F90C20A369A36091B2080739D52369F4
:10182000002B36D0EDB289042F4615D522686169A8
:10183000D31A8B421CDA0133A168501C0139A16014
:101840002060157062699A421AD0A389DB0701D51E
:101850000A2D15D03846F8BD616E42F4005221F4CD
:101860000051A281226861666169D31A8B42E2DB72
:1018700021463046FFF730F940B922680123DBE703
:1018800021463046FFF728F90028E3D04FF0FF3714
:10189000E0E721463046FFF70BF80028F6D1B4F90F
:1018A0000C20236991B2BDE7FFF76EF9B0E700BFE6
:1018B000F0B5064685B01F4689B1104C104D24681E
:1018C000646B002C08BF2C46D4F8E040A047431CB2
:1018D00003D100228A233A60336005B0F0BD0C4684
:1018E0000649074A0968496B002908BF1146224684
:1018F000D1F8E04001A9A047E9E700BF3802002085
:101900007C0A002021B1FF2A04D80A700120704708
:10191000084670478A2303604FF0FF30704700BFCE
:1019200070B50D46084C114606461A462846002357
:101930002360FAF76FFA431C00D070BD2368002BB8
:10194000FBD0336070BD00BFBC1E00202DE9F84302
:101950002C4D0646286898460F469146FFF7D4FC62
:10196000294B1C68D4F84831002B3ED05A681F2AF6
:101970001CDC02F1010E76B103EB82010124C1F8F7
:101980008890D3F8880194402043022EC3F8880140
:10199000C1F8088123D00232C3F804E0286843F874
:1019A0002270FFF7B3FC0020BDE8F883174B0BB3A0
:1019B0004FF4C870FDF7D6FA0346D8B1D4F84821E1
:1019C0000260002141600A46C4F848014FF0010E50
:1019D000C0F88811C0F88C11002EDCD0CCE7D3F809
:1019E0008C110C43C3F88C41D5E704F5A673C4F8F9
:1019F0004831BBE72868FFF789FC4FF0FF30BDE8AE
:101A0000F88300BF780A00209825410065EF400068
:101A100038B5074C0023054608462360FAF7FCFD5D
:101A2000431C00D038BD2368002BFBD02B6038BD91
:101A3000BC1E002070B559B105460C4610B1836B31
:101A4000002B3CD0636ED80705D5B4F90C302BB908
:101A50000026304670BDA38999053CD5214628460D
:101A6000FEF79AFFE36A064633B1E16928469847D4
:101A70000028B8BF4FF0FF36A3891A0622D4216B85
:101A800041B104F14003994202D02846FFF7A2F980
:101A900000232363616C21B12846FFF79BF90023E3
:101AA0006364FFF79DF8636E0022DB07A2810ED509
:101AB000A06DFFF727FCFFF799F8304670BDFFF7E0
:101AC00063F8BFE721692846FFF784F9D7E7A06DDF
:101AD000FFF71CFCECE7A06DFFF716FCB4F90C3027
:101AE000002BBBD1666E16F00106B1D1A06DFFF7D9
:101AF0000DFC304670BD00BF38B50B46074C05469F
:101B00001146184600232360FAF789FD431C00D0D4
:101B100038BD2368002BFBD02B6038BDBC1E0020D5
:101B200038B5074C0023054608462360FAF77CFDCC
:101B3000431C00D038BD2368002BFBD02B6038BD80
:101B4000BC1E002070B50D46084C114606461A46CC
:101B5000284600232360FAF769FD431C00D070BDBE
:101B60002368002BFBD0336070BD00BFBC1E00207B
:101B700070B50D46084C114606461A462846002305
:101B80002360FAF72DF9431C00D070BD2368002BA9
:101B9000FBD0336070BD00BFBC1E002053B94AB9F2
:101BA000002908BF00281CBF4FF0FF314FF0FF3065
:101BB00000F07AB9ADF1080C6DE904CE00F006F83A
:101BC000DDF804E0DDE9022304B070472DE9F047B9
:101BD0008C460D460446089E002B51D18A4217467A
:101BE0006DD9B2FA82FEBEF1000F0BD0CEF1200CFF
:101BF00001FA0EF520FA0CFC02FA0EF74CEA050C7D
:101C000000FA0EF44FEA174A250CBCFBFAF81FFA4B
:101C100087F90AFB18CC45EA0C4508FB09F3AB42EF
:101C20000AD9ED1908F1FF3280F02381AB4240F26E
:101C30002081A8F102083D44ED1AA4B2B5FBFAF0E8
:101C40000AFB105544EA054400FB09F9A14509D9EE
:101C5000E41900F1FF3380F00A81A14540F20781C9
:101C600002383C44A4EB090440EA08400021002E5D
:101C700061D024FA0EF4002334607360BDE8F0876D
:101C80008B4207D9002E54D0002186E82100084657
:101C9000BDE8F087B3FA83F1002940F08E80AB42B3
:101CA00002D3824200F2FA80841A65EB0305012018
:101CB000AC46002E3FD086E81010BDE8F08712B980
:101CC0000127B7FBF2F7B7FA87FEBEF1000F34D158
:101CD000EB1B3A0C1FFA87FC0121B3FBF2F8250C31
:101CE00002FB183345EA03450CFB08F3AB4207D966
:101CF000ED1908F1FF3002D2AB4200F2D1808046EC
:101D0000ED1AA3B2B5FBF2F002FB105543EA05440D
:101D10000CFB00FCA44507D9E41900F1FF3302D203
:101D2000A44500F2B8801846A4EB0C0440EA084031
:101D30009DE731463046BDE8F087CEF1200405FA34
:101D40000EF307FA0EF720FA04F83A0C25FA04F419
:101D500048EA0308B4FBF2F14FEA184502FB1144CC
:101D60001FFA87FC45EA044501FB0CF3AB4200FA7D
:101D70000EF409D9ED1901F1FF3080F08A80AB42F1
:101D800040F2878002393D44EB1A1FFA88F5B3FB15
:101D9000F2F002FB103345EA034500FB0CF3AB42C3
:101DA00007D9ED1900F1FF386FD2AB426DD9023877
:101DB0003D44EB1A40EA01418FE7C1F1200722FAC6
:101DC00007F88B4005FA01F448EA030320FA07FEFE
:101DD0004FEA134CFD404EEA040EB5FBFCF94FEA06
:101DE0001E440CFB19551FFA83F844EA054509FB0C
:101DF00008F4AC4202FA01F200FA01FA08D9ED182F
:101E000009F1FF3043D2AC4241D9A9F102091D4486
:101E10002D1B1FFA8EFEB5FBFCF00CFB10554EEA95
:101E2000054400FB08F8A04507D9E41800F1FF3588
:101E300029D2A04527D902381C4440EA0940A4EB26
:101E40000804A0FB02894C45C6464D4615D312D066
:101E500056B1BAEB0E0364EB050404FA07F7CB4066
:101E60001F43CC40376074600021BDE8F0871846FE
:101E7000F8E69046E0E6C245EAD2B8EB020E69EB1E
:101E800003050138E4E72846D7E7404691E7814655
:101E9000BEE7014678E702383C4445E7084608E7D4
:101EA000A8F102083D442BE7704700BF0100000085
:101EB0000200000004000000080000001000000004
:101EC00020000000400000008000000000008000B2
:101ED00000000001000000020000000400000008F3
:101EE00000000010000000000000000000000000E2
:101EF00000000000000000000000000000000000E2
:101F00000000000000000000000000000128011097
:101F10000203800253290351FF01026902026B1080
:101F2000058000404011088102560009000F00089A
:101F30008202560009000F0002350002250103F05D
:101F4000AA1104C00040000AC2010A010A010A00E5
:101F5000900203FF5A8102650B0EF9585F666D749B
:101F60007B828990979EA5AC03F0AA1202D320032E
:101F7000BF37BE02360003F0AA1104C500014000BD
:101F8000012801100253290351FF01026902026B6B
:101F90001005800140401103F0AA1104C000400068
:101FA0000AC2010A010A010A0090022D7011000004
:101FB000891080078003C0078003C003C0020003AC
:101FC000580020C637000D000F001100081800103F
:101FD000F0030C2000060B0B3308810256000B00A7
:101FE000110008820256000B001100023500022584
:101FF0000103F0AA1002D10203F0AA110AC2010AD9
:10200000010A010A00900203FF5A8102650B0EF9D2
:10201000585F666D747B828990979EA5AC03F0AA89
:102020001202D32003BF37BE02038102360003F041
:10203000AA1104C50001400001280110020380021A
:1020400053290351FF01026900026B100580004013
:102050004011088104AC0010001000088204AC009C
:102060001000100002350002250103F0AA1002D171
:102070000203F0AA110AC2010A010A010A009082B1
:1020800003F0AA1202D32003BF07BE03FF5A810246
:10209000650B0EF9585F666D747B828990979EA5DB
:1020A000AC0236000000000001280110020381028A
:1020B00053290351FF01026900026B102D701100BA
:1020C0000089108009F004F804F804F804F802000C
:1020D000041B002091BF0011000F00190009180017
:1020E00010F0030C2000060B0B330580013E3E115F
:1020F000088101E10010001000088201E1001000D9
:10210000100002250103F0AA1002D10203F0AA1167
:102110000AC2010A010A010A00900203F0AA12028F
:10212000D32003BF07BE03FF5A8102650B0EF95887
:102130005F666D747B828990979EA5AC000000005D
:102140005658523030000000302E322E3000000041
:1021500055534152540000004661696C6564207417
:102160006F20637265617465207573617274207489
:1021700061736B0D0A00000048494420436F6D6D88
:10218000616E6473000000004661696C65642074D0
:102190006F206372656174652048494420636F6DE8
:1021A0006D616E642070726F636573736F722074FB
:1021B00061736B0D0A000000484944205265706F3E
:1021C000727400004661696C656420746F206372EC
:1021D000656174652048494420706572696F64695F
:1021E00063207265706F7274207461736B0D0A00E6
:1021F000302E322E3000000000FFFFFFFFFFFF00F7
:1022000009279550D2040000021E0104A5000078A1
:10221000E7000000000000000000000000000101D5
:102220000101010101010101010101010101CAB422
:102230000080F080187040209200FFFF0000001E18
:10224000A5510080A00020A040200204FFFF000054
:10225000001E000000000000000000000000000060
:10226000000000000000001000000000000000005E
:1022700000000000000001757012790000030014D6
:10228000689F0080FF137F003F801F00FF091F0031
:102290000F800100000000000000000000000000AE
:1022A000000000000000000000000000000000002E
:1022B000000000000000000000000000000000001E
:1022C000000000000000000000000000000000000E
:1022D00000000000000000000000000000000000FE
:1022E00000000000000000000000000000000000EE
:1022F000000000000000B19000FFFFFFFFFFFF00A3
:1023000009273412D2040000021E0104A50000783F
:10231000E7000000000000000000000000000101D4
:10232000010101010101010101010101010100009F
:1023300000000000000000000000FFFF0000001887
:10234000000000000000000000000000000000008D
:10235000000000000000000000000000000000007D
:1023600000000000000000FC004265796F6E640010
:10237000000000000000010D7020790000220928F3
:102380001EF50A00FF0EFF003F801F007F071B00A5
:102390000E80010039540F80DF137F003F801F0043
:1023A000EF0917000E8001007E00073A02928100BB
:1023B0000800000000000000000000000000000015
:1023C000000000000000000000000000000000000D
:1023D00000000000000000000000000000000000FD
:1023E00000000000000000000000000000000000ED
:1023F000000000000000F890766964656F5F7072FD
:102400006F6300004661696C656420746F206372BD
:102410006561746520766964656F2070726F6365AD
:1024200073736F72207461736B0D0A00FF00FF00FD
:10243000493243004661696C656420746F206372A1
:102440006561746520493243207461736B0D0A0025
:1024500054494D45445F5354415254004661696CA0
:10246000656420746F206372656174652074696DA2
:1024700065642073746172747570207461736B0D80
:102480000A000000414443004661696C65642074A1
:102490006F206372656174652041444320746173E9
:1024A0006B0D0A00313233342020202020202020E0
:1024B000202020200000000049444C45000000007E
:1024C00000C20100C0000000000800000000000081
:1024D0002D2D2042696773637265656E20426579B0
:1024E0006F6E64202D2D0A00444953504C415942CF
:1024F0004F4152442056302E342E32002D2D2025AF
:1025000073202D2D0A0000002D2D20566572736951
:102510006F6E202573202D2D0A00000031343A31D2
:10252000313A3036000000004A616E2033302032EC
:10253000303233002D2D20436F6D70696C65643A25
:10254000202573202573202D2D0A00005553424C61
:102550006F6164004661696C656420746F2063720A
:102560006561746520555342204C6F61646572202B
:102570007461736B0D0A0000737461636B206F7676
:102580006572666C6F772025782025730D0A000030
:102590006C6F67660000000040020020303132336B
:1025A000343536373839414243444546000000004F
:1025B00030313233343536373839616263646566B9
:1025C00000000000286E756C6C290000202020207F
:1025D00020202020202020202020202030303030BB
:1025E0003030303030303030303030304300000068
:1025F000504F5349580000002E00000000202020BA
:1026000020202020202028282828282020202020A2
:102610002020202020202020202020202088101072
:1026200010101010101010101010101010040404CE
:10263000040404040404041010101010101041418C
:10264000414141410101010101010101010101017A
:10265000010101010101010110101010101042428E
:10266000424242420202020202020202020202024A
:1026700002020202020202021010101020000000EA
:10268000000000000000000000000000000000004A
:10269000000000000000000000000000000000003A
:1026A000000000000000000000000000000000002A
:1026B000000000000000000000000000000000001A
:1026C000000000000000000000000000000000000A
:1026D00000000000000000000000000000000000FA
:1026E00000000000000000000000000000000000EA
:1026F00000000000000000000000000000000000DA
:10270000F8B500BFF8BC08BC9E4670477909410087
:1027100029444000F8B500BFF8BC08BC9E4670478D
:1027200005444000A8F4FF7F0100000030B482B0EF
:10273000049C5BB31D46036843F480330360C9B255
:1027400041F0B441416083680193019B13F0010F94
:10275000F9D1002306E0990001F58001096845F8E8
:1027600023100133A342F6D3D2B242F0B442426006
:1027700083680193019B13F0010FF9D0036823F4E0
:1027800080330360002002B030BC70470220FAE7BB
:102790000160704782B0416083680193019B13F030
:1027A000010FF9D0019800F00E0002B07047000050
:1027B0007144400075444000774440007B44400031
:1027C0007F444000B9444000094540008144400036
:1027D00085444000914440000100FFFFFFFF0000DE
:1027E0000110FFFF0210FFFF0310FFFF0120FFFF9A
:1027F0000220FFFF05000000F822410001474700CA
:1028000080010020F000002000000000F8000020FF
:102810009401002009028500030100C032080B006A
:102820000201010002090400000001010002092464
:102830000100011E0001010C24020101020002033B
:102840000000000924030201010001000904010045
:102850000001020002090401010101020002072433
:1028600001020101000B2402010202100180BB00E1
:102870000905840500010100000725010000000092
:1028800009040200010300000009211101000122D6
:102890002600070581034000040000001201000229
:1028A00000000040BD3501010001010203010000EC
:1028B00094000020A8000020A00100202D944000DA
:1028C0004D944000A59440004F944000000000004B
:1028D00006FFFF0901A10109020903150026FF00F7
:1028E00075089540810209060907150026FF007545
:1028F000089540B102C00000000300000000000085
:1029000000000000000000000000000000000000C7
:1029100000000000000000000000000000000000B7
:10292000000000000403090447656E6572696300D6
:102930005553422053746572656F204D6963726F01
:1029400070686F6E6500010000127A00AAAAAAAA38
:102950000100000040020020000000000000000014
:102960002C05002094050020FC050020000000003C
:102970000000000000000000000000000000000057
:102980000000000000000000000000000000000047
:102990000000000000000000000000000000000037
:1029A0000000000000000000000000000000000027
:1029B0000000000000000000000000000000000017
:1029C0000000000000000000000000000000000007
:1029D00000000000000000000000000000000000F7
:1029E00000000000000000000000000000000000E7
:1029F00000000000000000000000000000000000D7
:102A00000000000001000000000000000E33CDAB0C
:102A100034126DE6ECDE05000B0000000000000043
:102A200000000000000000000000000000000000A6
:102A30000000000000000000000000000000000096
:102A40000000000000000000000000000000000086
:102A50000000000000000000000000000000000076
:102D800000000000000000000000000068060020B5
:102D900068060020700600207006002078060020DB
:102DA000780600208006002080060020880600208B
:102DB000880600209006002090060020980600203B
:102DC00098060020A0060020A0060020A8060020EB
:102DD000A8060020B0060020B0060020B80600209B
:102DE000B8060020C0060020C0060020C80600204B
:102DF000C8060020D0060020D0060020D8060020FB
:102E0000D8060020E0060020E0060020E8060020AA
:102E1000E8060020F0060020F0060020F80600205A
:102E2000F806002000070020000700200807002007
:102E300008070020100700201007002018070020B6
:102E40001807002020070020200700202807002066
:102E50002807002030070020300700203807002016
:102E600038070020400700204007002048070020C6
:102E70004807002050070020500700205807002076
:102E80005807002060070020600700206807002026
:102E900068070020700700207007002078070020D6
:102EA0007807002080070020800700208807002086
:102EB0008807002090070020900700209807002036
:102EC00098070020A0070020A0070020A8070020E6
:102ED000A8070020B0070020B0070020B807002096
:102EE000B8070020C0070020C0070020C807002046
:102EF000C8070020D0070020D0070020D8070020F6
:102F0000D8070020E0070020E0070020E8070020A5
:102F1000E8070020F0070020F0070020F807002055
:102F2000F807002000080020000800200808002002
:102F300008080020100800201008002018080020B1
:102F40001808002020080020200800202808002061
:102F50002808002030080020300800203808002011
:102F600038080020400800204008002048080020C1
:102F70004808002050080020500800205808002071
:102F80005808002060080020600800206808002021
:102F900068080020700800207008002078080020D1
:102FA0007808002080080020800800208808002081
:102FB0008808002090080020900800209808002031
:102FC00098080020A0080020A0080020A8080020E1
:102FD000A8080020B0080020B0080020B808002091
:102FE000B8080020C0080020C0080020C808002041
:102FF000C8080020D0080020D0080020D8080020F1
:10300000D8080020E0080020E0080020E8080020A0
:10301000E8080020F0080020F0080020F808002050
:10302000F8080020000900200009002008090020FD
:1030300008090020100900201009002018090020AC
:10304000180900202009002020090020280900205C
:10305000280900203009002030090020380900200C
:1030600038090020400900204009002048090020BC
:10307000480900205009002050090020580900206C
:10308000580900206009002060090020680900201C
:1030900068090020700900207009002078090020CC
:1030A000780900208009002080090020880900207C
:1030B000880900209009002090090020980900202C
:1030C00098090020A0090020A0090020A8090020DC
:1030D000A8090020B0090020B0090020B80900208C
:1030E000B8090020C0090020C0090020C80900203C
:1030F000C8090020D0090020D0090020D8090020EC
:10310000D8090020E0090020E0090020E80900209B
:10311000E8090020F0090020F0090020F80900204B
:10312000F8090020000A0020000A0020080A0020F8
:10313000080A0020100A0020100A0020180A0020A7
:10314000180A0020200A0020200A0020280A002057
:10315000280A0020300A0020300A0020380A002007
:10316000380A0020400A0020400A0020480A0020B7
:10317000480A0020500A0020500A0020580A002067
:10318000580A0020600A0020600A0020FFFFFFFFAD
:1031900000000200981E0020430000000000000014
:1031A000000000000000000000000000000000001F
:1031B00000000000000000004300000000000000CC
:1031C00000000000000000000000000000000000FF
:1031D00000000000000000004300000000000000AC
:1031E00000000000000000000000000000000000DF
:1031F000000000000000000043000000000000008C
:1032000000000000000000000000000000000000BE
:10321000000000000000000043000000000000006B
:10322000000000000000000000000000000000009E
:10323000000000000000000043000000000000004B
:10324000000000000000000000000000000000007E
:10325000000000000000000043000000000000002B
:10326000000000000000000000000000000000005E
:103270000000000000000000051941000114410099
:1032800000000000FC254100F8254100B424410065
:10329000B4244100B4244100B4244100B4244100CA
:1032A000B4244100B4244100B4244100B4244100BA
:1032B000FFFFFFFFFFFFFFFFFFFFFFFFFFFF00001C
:1032C0000100415343494900000000000000000094
:1032D00000000000000000000000000000000000EE
:1032E0000000415343494900000000000000000075
:1032F00000000000000000000000000000000000CE
:1033000000000000FFFFFFFFFFFFFFFFFFFFFFFFC9
:10331000FFFFFFFFFFFFFFFFFFFFFFFF5088D7BE4C
:00000001FF
